:020000040800F2
:10000000000001105DE10308F5B2020865D70008A1
:1000100061E2030861E2030861E2030800000000F6
:100020000000000000000000000000003DB90208D0
:1000300039B902080000000035B9020801ED0008D6
:1000400061E2030861E2030861E2030861E2030878
:1000500061E2030861E20308559B0008819C0008E7
:10006000459C0008099C0008CD9B00084DBC000879
:100070003DBC00082DBC00081DBC00080DBC0008DC
:10008000F9BB0008E5BB000861E2030861E2030870
:1000900061E2030861E2030861E20308919B000842
:1000A00061E2030861E2030861E2030861E2030818
:1000B0004DDE00083DDE000861E2030869C4000867
:1000C00071C400085DC4000865C4000861E203084B
:1000D00061E20308C990000861E2030829EE000804
:1000E000199B000861E2030841B9020861E20308B4
:1000F0000DDE000861E203081DDE0008D1BB000828
:1001000061E2030861E203082DDE000861E20308F2
:1001100061E2030861E20308ADA8010891A80108A3
:10012000BDBB0008A9BB000895BB000881BB000847
:100130006DBB000861E2030861E2030861E20308A5
:1001400061E2030861E2030861E20308F9B2020810
:1001500059BB000845BB000831BB00088DED000805
:1001600051C4000859C4000861E2030861E20308B1
:1001700061E2030861E2030861E2030861E2030847
:0801800061E2030861E20308DB
:1001880016000800A4250020AC250020000000006F
:100198004C06000803000100302B0020382B0020FB
:1001A8000000000000000000010104007C2B00207A
:1001B800A03A00200000000000000000080209002A
:1001C800E2390020A43A002000000000298200083B
:1001D80006020C00583A0020B03A00200000000047
:1001E800F98E0008070202007C3A0020BC3A002081
:1001F800000000005406000802000C00643A0020C9
:10020800C03A00200000000000000000F7010600CE
:10021800DC390020CC3A0020000000005606000817
:100228000A020A000C2C0020D43A0020000000002A
:100238005C0600082C001000904000208040002040
:100248000000000015F801082B002400C44000201D
:10025800A040002000000000E5F70108230010007E
:1002680014400020E840002000000000E1EE0108F2
:1002780028000C00CC460020104700200000000099
:100288006606000829005000604600201C47002030
:100298000000000000000000140002005C4600207E
:1002A8006C470020000000007206000801020500EB
:1002B800A84C00201851002000000000AD300208B2
:1002C80000020500704700202051002000000000B7
:1002D800000000001E000400B44A0020285100203D
:1002E800000000007406000822000C00344A0020B8
:1002F8002C5100200000000078060008031233008B
:10030800AB5200207852002000000000840600084C
:1003180025005A00C45100201E5200200000000091
:1003280000000000F6110C00B8510020AC5100206C
:1003380000000000B806000801200800BC53002097
:100348000854002000000000C40600081A00080035
:10035800A05300201054002000000000CC06000824
:100368001D00010034590020C85900200000000079
:10037800D40600081900050020590020CC59002097
:1003880000000000D606000800010400BC59002047
:10039800D459002000000000DC06000827000400F3
:1003A80054590020D859002000000000E006000839
:1003B8001B00F400505A0020D05B00200000000011
:1003C800BD3002082F001100B45B0020C45C00207F
:1003D80000000000E406000810000300FC5C002098
:1003E800045D002000000000F6060008F901040082
:1003F8009463002098630020000000001182000828
:1004080018102C00646300209C630020000000008A
:1004180039040208FB01010030630020C863002092
:100428000000000065C50008FC010900FC6100200F
:10043800CC6300200000000031C500080A1012003B
:10044800D0610020D863002000000000FA060008F0
:1004580006001600A05E0020EC63002000000000EB
:10046800094D0208340010000C5D002004640020CF
:1004780000000000195F03080D003400886B00209D
:10048800BC6B002000000000896E020812100C00EE
:100498006C6B0020F06B0020000000000C070008C7
:1004A8000C020100686B0020FC6B002000000000BB
:1004B80018070008020203007C6B0020006C002073
:1004C8000000000000000000FA010200B8640020EB
:1004D800046C00200000000089C50008FD0124000C
:1004E80084640020086C002000000000A18100083E
:1004F800FE010800706400202C6C00200000000041
:100508006DC500081F000E004C6D0020286F0020EC
:10051800000000001A07000805020100346D0020E1
:10052800386F0020000000002807000809020100B9
:10053800A06F0020F86F0020000000002A070008C4
:100548000C0024006A6F0020FC6F002000000000EF
:10055800519E01080E20EA00A2700020C07E0020F3
:1005680000000000E94C020813000400D0710020CC
:10057800AC7F0020000000002C07000802010300E7
:100588008D700020B07F002000000000799E0108D7
:10059800F811010030860020B48600200000000019
:1005A800300700082A00600018870020B88600205D
:1005B80000000000F15E030815007000E8800020CC
:1005C80078870020000000000000000026000E00D0
:1005D800EC890020DC8900200000000095780308E1
:1005E8000B20100060880020FC890020000000001B
:1005F80032070008030106004C8A0020608A0020A8
:1006080000000000420700080400800098A60020AF
:100618004CA80020000000000000000005000600B3
:10062800CCA90020F0A9002000000000480700081D
:10063800F511620064A90020F8A90020000000005C
:04064800C9BC03081E
:10064C00C409000019012828013C390100000000F0
:10065C0000004A01B400D6010000000000010000B7
:10066C00000000000000030000000100C800141E80
:10067C00010064002C0128000000000000000000B4
:10068C00000000000000000000000000000000005E
:10069C00000000000000000000000000000000004E
:1006AC00000000000000000000000100000000003D
:1006BC000000000000000000E8036400040A0001D0
:1006CC007E05EA05B4053200000000002801000098
:1006DC00900100002003000000000000000000005A
:1006EC0000000000000000000000000105000030C8
:1006FC000100005A0000000090012C01C8006400A9
:10070C000000000100054B545631000001000000B0
:10071C000000000001000000000500000000370090
:10072C000804040004002B21231E640102000000B5
:10073C0001000A012900040101000000200003004F
:02074C000100AA
:10074E000100000050010000070000000200000040
:10075E000000803F0000803F0000803F000000004E
:10076E000000000001020304060708090101000051
:10077E0020430408E06104080000000000000000AF
:10078E003043040838430408000000000120000034
:10079E003C430408444304080000000001400000EC
:1007AE0048430408E0550408000000000120000042
:1007BE0054430408604304080000000004000000D5
:1007CE006443040850850408000000000400000083
:1007DE00704304088C6F0408000000000100000044
:1007EE000201FF000000803F1012040805080400FB
:1007FE00000000004037040818320408FC110408F9
:10080E00000000003C12040805080A000000000069
:10081E004037040818320408C039040800000000EC
:10082E00FFFFFFFF0101000061F40108000000005E
:10083E00000000000001010101000000E0010000C5
:10084E000000803F080000000000803F5DAD020800
:10085E0015AD020865AC02080000000081A8020870
:10086E001DAA0208DDAA020885A9020800000000E0
:10087E000000000075A8020859A8020855A8020831
:10088E0051A8020845A8020841A802084DA802086E
:10089E0049A8020869A802085DA802085DA9020815
:1008AE0071A9020849A9020835A9020821A902085E
:1008BE000000803F303030302D30312D303154300B
:1008CE00303A30303A30300004030904120100028D
:1008DE00020200408304405700020102030100009F
:1008EE0009024300020100C03209040000010202A5
:1008FE000100052400100105240100010424020258
:10090E000524060001070582030800FF0904010003
:10091E00020A0000000705010240000007058102DF
:10092E0040000000FF000000E9AB020809AB02081E
:10093E0045AE0208DDA80208F1AD0208EDA80208D6
:10094E0009A90208B5A80208A5A80208000000001F
:10095E000000000000000101FFFF010100600240E5
:10096E001060024000000000000B0000000020009C
:10097E0000000000000000000060024028600240FD
:10098E0000000000060C0000000020000000000027
:10099E0000000000006002404060024000000000C5
:1009AE00100D0000000020000000000000000000FC
:1009BE00006002405860024000000000160E000069
:1009CE000000200000000000000000000060024057
:1009DE007060024000000000200F000000002000A8
:1009EE00000000000000000000600240886002402D
:1009FE000000000026100000000020000000000093
:100A0E000000000000600240A060024000000000F4
:100A1E003011000000002000000000000000000067
:100A2E0000600240B860024000000000362F000057
:100A3E0000002000000000000000000000640240E2
:100A4E00106402400000000000380000000040006A
:100A5E000000000000000000006402402864024014
:100A6E0000000000063900000000400000000000F9
:100A7E0000000000006402404064024000000000DC
:100A8E00103A0000000040000000000000000000CE
:100A9E00006402405864024000000000163B000053
:100AAE000000400000000000000000000064024052
:100ABE007064024000000000203C00000000400076
:100ACE000000000000000000006402408864024044
:100ADE00000000002644000000004000000000005E
:100AEE000000000000640240A0640240000000000C
:100AFE003045000000004000000000000000000033
:100B0E0000640240B8640240000000003646000057
:100B1E000000400000000000000000000000000186
:100B2E0000000000000000000000000008000000AF
:100B3E0000FFFF0000000000AA5503009FAA550504
:100B4E00010000AA550701000001AA550B01000083
:100B5E00AA5509020000000001000000C0120000AA
:100B6E0001010100687A04080F000000B94A030869
:100B7E000000000000000000A40500202C7A0408EC
:100B8E000000000000000000000000000000000057
:100B9E00E0610408000000000000000030060020A4
:100BAE0004000000B87904080D000000E5510308A8
:100BBE00440A002000000000847D04080D0000009F
:100BCE00B5510308380A0020000000004C7A0408D2
:100BDE0008000000000000002C0A002004000000A5
:100BEE003C7A04080D000000CD500308200A0020B6
:100BFE0000000000D078040803000000B19503083F
:100C0E00080A002000000000447A040803000000D7
:100C1E00B1950308F009002000000000D478040804
:100C2E0001000000000000000000000000000000B5
:100C3E00000000000E000000000000000000000098
:100C4E00000000002C7A04080000000000000000E4
:100C5E000000000000000000E06104080000000039
:100C6E000000000030060020040000005C7904083B
:100C7E000300000071500308D8090020080000008E
:100C8E003C7A04080D000000CD500308200A002015
:100C9E0000000000D078040803000000B19503089E
:100CAE00080A002000000000447A04080300000037
:100CBE00B1950308F009002000000000D478040864
:100CCE000100000000000000000000000000000015
:100CDE00000000000E0000000000000000000000F8
:100CEE0000000000547A040800000000000000001C
:100CFE000000000000000000E06104080000000099
:100D0E000000000030060020040000006479040892
:100D1E0003000000B1950308500A002000000000F7
:100D2E00D47804080100000000000000000000005C
:100D3E0000000000000000000E0000000000000097
:100D4E00000000000000000020700020702D7200D6
:100D5E002D202D2D202D2D2D2D202D2D2D2D000036
:100D6E000000000000000000000000000000000075
:100D7E002D202D2D202D2D2D2D202D2D2D00000043
:100D8E000000000000000000000000000000000055
:100D9E002E70002088130C17010000003070002008
:100DAE0088130C1700000000A8780408000000004B
:100DBE00000000000000000000000000B8780408E9
:100DCE0008000000000000005C0600200400000087
:100DDE00C47804080800000000000000500600203F
:100DEE0000000000D078040804000000B150030891
:100DFE000000000000000000D4780408010000008C
:100E0E0000000000000000000000000000000000D4
:100E1E000E000000000000000000000000000000B6
:100E2E002C70002088130C17010000002A7000207F
:100E3E0088130C17000000000C7904080F00000046
:100E4E00114B03080000000000000000680600209F
:100E5E00CE71002001000000003704082970002028
:100E6E00010000000C370408306D00200200000065
:100E7E00143704085EA700200000000000000000E8
:100E8E005CA7002000000000000000005AA7002010
:100E9E00000000000000000058A700200000000025
:100EAE000000000056A70020000000000000000017
:100EBE0054A7002000000000000000001C040020C9
:100ECE00000000000000000028700020020000005A
:100EDE002037040814790408000000000000000008
:100EEE000000000000000000B878040808000000B0
:100EFE0000000000EC06002004000000C478040886
:100F0E000800000000000000E006002000000000C5
:100F1E00D078040804000000F14A03080000000025
:100F2E0000000000D478040801000000000000005A
:100F3E000000000000000000000000000E00000095
:100F4E0000000000000000000000000024790408EA
:100F5E000000000000000000000000000000000083
:100F6E00347904080D0000005551030828070020AD
:100F7E0004000000407904080D000000354B030802
:100F8E001C070020040000004C7904080D0000002E
:100F9E0015510308100700200000000058790408BE
:100FAE000300000091500308F8060020080000001E
:100FBE006479040803000000B1950308500A00206C
:100FCE0000000000D47804080100000000000000BA
:100FDE000000000000000000000000000E000000F5
:100FEE000000000000000000000000006C79040802
:100FFE0000000000000000000000000000000000E3
:10100E007479040804000000155203080000000063
:10101E0000000000D4780408010000000000000069
:10102E000000000000000000000000000E000000A4
:10103E00000000000000000000000000C07904085D
:10104E000000000000000000000000000000000092
:10105E00F86804080D00000000000000880700205A
:10106E0004000000D0790408080000000000000011
:10107E007C07002004000000DC7904080800000052
:10108E00000000007007002004000000E47904084E
:10109E0008000000000000006407002004000000AB
:1010AE00EC7904080800000000000000580700203A
:1010BE0004000000F479040808000000000000009D
:1010CE004C07002004000000FC7904080800000012
:1010DE00000000004007002004000000047A04080D
:1010EE00080000000000000034070020040000008B
:1010FE00D478040801000000000000000000000089
:10110E0000000000000000000E00000000000000C3
:10111E0000000000000000000C7A04080F00000020
:10112E00014B03080000000000000000940700209F
:10113E00147A04080F0000000000000000000000F8
:10114E00000000000C0800201C7A04080F000000AC
:10115E00000000000000000000000000AC080020AD
:10116E00CD710020040000002C37040824700020EC
:10117E00E0150C170000000027700020080000008A
:10118E0018320408267000200500000040370408BD
:10119E00247A04080F000000000000000000000088
:1011AE0000000000FC080020846604080000000017
:1011BE00000000008D9E0108A086010004000000C2
:1011CE000000000000000000000000000000000011
:1011DE000000000000000000000000000C7E04086B
:1011EE002C60040800000000715801087D0000000A
:1011FE0006000000000000000000000000000000DB
:10120E0000000000000000000000000000000000D0
:10121E00A87A04080000000000000000A5B603082C
:10122E00E8030000030000000000000000000000C2
:10123E0000000000000000000000000000000000A0
:10124E0000000000B07A040800000000000000005A
:10125E00114E0208102700000300000000000000DD
:10126E000000000000000000000000000000000070
:10127E000000000000000000787C04080000000060
:10128E006DF60108F9360108204E00000500000039
:10129E000000000000000000000000000000000040
:1012AE00000000000000000000000000F8670408C5
:1012BE00000000000000000061B1030810270000CC
:1012CE00010000000000000000000000000000000F
:1012DE000000000000000000000000000000000000
:1012EE00BC7A04080000000000000000FDC40008E5
:1012FE00E8030000050000000000000000000000F0
:10130E0000000000000000000000000000000000CF
:10131E0000000000C87A0408000000000000000071
:10132E00B5A00108204E00000300000000000000E0
:10133E00000000000000000000000000000000009F
:10134E000000000000000000D87A04080000000031
:10135E0000000000BD9E0108204E000003000000AA
:10136E00000000000000000000000000000000006F
:10137E00000000000000000000000000E87A0408F1
:10138E00000000000000000001560108400D03009F
:10139E00030000000000000000000000000000003C
:1013AE00000000000000000000000000000000002F
:1013BE003867040800000000000000007D8302086A
:1013CE0010270000010000000000000000000000D7
:1013DE0000000000000000000000000000000000FF
:1013EE00000000004860040800000000000000003B
:1013FE0079410208102700000300000000000000E1
:10140E0000000000000000000000000000000000CE
:10141E000000000000000000F87A04080000000040
:10142E00000000006DD50308A08601000100000039
:10143E00000000000000000000000000000000009E
:10144E0000000000000000000000000038600408EA
:10145E0000000000000000008DD4030850C30000FF
:10146E00010000000000000000000000000000006D
:10147E00000000000000000000000000000000005E
:10148E00208504080000000000000000F5CF0308CE
:10149E00A861000001000000000000000000000034
:1014AE00000000000000000000000000000000002E
:1014BE0000000000007B0408000000000000000097
:1014CE005D480208A0860100010000000000000037
:1014DE0000000000000000000000000000000000FE
:1014EE00000000000000000000680408000000007A
:1014FE0000000000F50D0108A00F00000100000023
:10150E0000000000000000000000000000000000CD
:10151E000000000000000000000000000C7B04082A
:10152E00000000000000000041BD0208102700006E
:10153E00010000000000000000000000000000009C
:10154E00000000000000000000000000000000008D
:10155E0078820408000000000000000051BE03085D
:10156E001A41000001000000000000000000000011
:10157E00000000000000000000000000000000005D
:10158E000000000064680408000000000000000075
:10159E00E1230308102700000100000000000000F6
:1015AE00000000000000000000000000000000002D
:1015BE00000000000000000070750408000000002C
:1015CE0000000000D99603081A4100000100000037
:1015DE0000000000000000000000000000000000FD
:1015EE00000000000000000000000000187B04084E
:1015FE000000000000000000656E0208400D0300B0
:10160E0000000000000000000000000000000000CC
:10161E0000000000000000000000000000000000BC
:10162E00207B04080000000000000000216E02086C
:10163E00400D03000000000000000000000000004C
:10164E00000000000000000000000000000000008C
:10165E0000000000287B04080000000000000000CD
:10166E00BDA20108A08601000300000000000000DA
:10167E00000000000000000000000000000000005C
:10168E000000000000000000000000000102030442
:10169E000102030406070809D48204080F000000A3
:1016AE00000000000000000000000000F4220020F6
:1016BE00FFFFFFFFFA000000010000000100000024
:1016CE00487B0408507B04086C7904080000000075
:1016DE00000000000000000000000000407B040835
:1016EE00040000000350030800000000000000008A
:1016FE00D478040801000000000000000000000083
:10170E0000000000000000000E00000000000000BD
:10171E00000000000000000002A800200100C40923
:10172E000000000000A800200100C4090000000015
:10173E00FEA700200100C40900000000FCA7002045
:10174E000100C40900000000F8A700200100C40930
:10175E0000000000FAA700200100C40900000000EC
:10176E00F6A700200100C40900000000F4A7002025
:10177E000100C409000000003E7000200100C800F6
:10178E00010000003C700020320030753200000075
:10179E003B700020055A05003670002000FF010046
:1017AE003A70002001000000800F002038700020E9
:1017BE0002000000704204083570002000FF010096
:1017CE003970002001000000800F002037700020CB
:1017DE000200000070420408707B04080F00000035
:1017EE00000000000000000000000000880F002034
:1017FE00488A00209CFF2C010000000022040020DB
:10180E000A000000C039040820700020E0150C17F3
:10181E000000000021040020080000001832040817
:10182E00200400200500000040370408227000202C
:10183E0002000000D8390408BE7100200100FF7FAD
:10184E0001000000BC71002002000000E439040811
:10185E009670002003000000F439040895700020F3
:10186E0003000000F4390408947100200000F40114
:10187E0001000000927100200000F4010100000040
:10188E00907100200000F401010000008E71002014
:10189E000000F401010000008C71002000FF010027
:1018AE00A8710020E803D0070A000000A6710020EE
:1018BE00006401000A000000A7710020006401000E
:1018CE000A000000A0710020006401000A00000060
:1018DE00A5710020006401000A000000A471002020
:1018EE00006401000A000000A371002000640100E2
:1018FE000A0000009F71002000FF01000A00000096
:10190E009E71002000FF01000A0000009E70002062
:10191E000000F401010000009C7000200000F401A2
:10192E00010000009A7000200000F4010100000088
:10193E00987000200000F401010000009B7100204F
:10194E0000C801009A71002000C8010099710020A2
:10195E0000C8010098710020006401000A00000018
:10196E009771002000FF01000A000000B3710020F3
:10197E0000C80100B271002000C80100B171002042
:10198E0000C80100B071002000C80100AF71002036
:10199E0000C80100AE71002000C80100AD7100202A
:1019AE0000C80100AC71002000C80100AB7100201E
:1019BE0000C80100787B0408000000000000000051
:1019CE000000000000000000887B040809000000F1
:1019DE00000000002C10002004000000907B040882
:1019EE00090000000000000020100020040000008C
:1019FE0030810408090000000000000014100020CF
:101A0E0004000000607404080900000000000000DB
:101A1E000810002004000000987B04080900000054
:101A2E0000000000FC0F002004000000A07B040852
:101A3E000900000000000000F00F0020040000006C
:101A4E00A87B04080900000000000000E40F00203D
:101A5E0004000000B07B0408090000000000000034
:101A6E00D80F002004000000D47804080100000004
:101A7E000000000000000000000000000000000058
:101A8E000E0000000000000000000000000000003A
:101A9E00887C040800000000000000000000000028
:101AAE0000000000FC840408070000000000000095
:101ABE005010002000000000987C04080800000070
:101ACE00000000004410002000000000A47C040868
:101ADE000800000000000000381000200000000088
:101AEE00D47804080100000000000000000000008F
:101AFE0000000000000000000E00000000000000CA
:101B0E000000000000000000AC7C04080000000093
:101B1E00000000000000000000000000BC7C040873
:101B2E000D000000000000008C10002000000000DE
:101B3E00C47C04080D00000000000000801000208E
:101B4E0000000000CC7C040807000000000000002C
:101B5E007810002000000000D47C04080D00000066
:101B6E00000000006C10002000000000DC7C040867
:101B7E000D000000000000006010002000000000BA
:101B8E00E47C04080700000000000000581000204C
:101B9E0000000000D47804080100000000000000DE
:101BAE000000000000000000000000000E00000019
:101BBE00000000000000000000000000EC7C0408A3
:101BCE000000000000000000000000000000000007
:101BDE00FC8404080C00000000000000407000208F
:101BEE0000000000007D04080C0000000000000052
:101BFE004270002000000000107D04080C00000060
:101C0E00000000007870002000000000207D040815
:101C1E000C000000000000006C70002000000000AE
:101C2E00347D04080C000000000000004470002009
:101C3E0000000000407D04080C00000000000000C1
:101C4E004670002000000000487D04080C000000D3
:101C5E000000000048700020000000005C7D0408B9
:101C6E000C000000000000004A7000200000000080
:101C7E00647D04080C000000000000004C70002081
:101C8E00000000006C7D04080C0000000000000045
:101C9E004E70002000000000787D04080C0000004B
:101CAE0000000000507000200000000024750408A1
:101CBE000C00000000000000527000200000000028
:101CCE00807D04080C00000000000000547000200D
:101CDE00000000008C7D04080C00000000000000D5
:101CEE005670002000000000987D04080C000000D3
:101CFE00000000005870002000000000A47D0408C1
:101D0E000C000000000000005A70002000000000CF
:101D1E00B07D04080C000000000000005C70002084
:101D2E0000000000BC7D04080C0000000000000054
:101D3E007070002000000000C47D04080C0000003C
:101D4E00000000006E70002000000000CC7D040832
:101D5E000C000000000000007C700020000000005D
:101D6E00D87D04080C000000000000007E700020EA
:101D7E0000000000E47D04080C00000000000000DC
:101D8E008470002000000000208504080C00000074
:101D9E00000000005E700020000000003C7A040885
:101DAE000C00000000000000667000200000000023
:101DBE00F07D04080C0000000000000060700020A0
:101DCE0000000000FC7D04080C0000000000000074
:101DDE006270002000000000087E04080C00000065
:101DEE00000000006470002000000000107E040857
:101DFE000C000000000000006870002000000000D1
:101E0E00D46004080C000000000000007270002076
:101E1E00000000001C7E04080C0000000000000002
:101E2E006A70002000000000D47404080C0000004A
:101E3E00000000007A70002000000000287E0408D8
:101E4E000C00000000000000747000200000000074
:101E5E00307E04080C0000000000000076700020A8
:101E6E0000000000387E04080C0000000000000096
:101E7E008070002000000000407E04080C0000006E
:101E8E00000000008270002000000000D4780408DA
:101E9E000100000000000000000000000000000033
:101EAE00000000000E000000000000000000000016
:101EBE0000000000487E0408000000000000000042
:101ECE000000000000000000587E0408050000001D
:101EDE00000000009470002000000000D478040878
:101EEE0001000000000000000000000000000000E3
:101EFE00000000000E0000000000000000000000C6
:101F0E0000000000607E04080000000000000000D9
:101F1E000000000000000000E06104080000000066
:101F2E000000000010060020040000005C7404088D
:101F3E000D00000049500308EC10002000000000C6
:101F4E00B87904080D000000654A0308E01000206F
:101F5E0000000000847D04080D000000314A0308D3
:101F6E00D4100020000000004C7A04080800000085
:101F7E0000000000C8100020040000003C7A040895
:101F8E000D0000001D4A0308BC10002000000000D8
:101F9E006C7E04080900000000000000B010002054
:101FAE0004000000D078040803000000B195030877
:101FBE009810002000000000D478040801000000F2
:101FCE000000000000000000000000000000000003
:101FDE000E000000000000000000000000000000E5
:101FEE00747E0408000000000000000000000000E5
:101FFE0000000000847E04080D00000000000000B8
:10200E0004110020000000008C7E04080A0000006D
:10201E0000000000D471002000000000987E04082B
:10202E000A00000000000000DC710020000000002B
:10203E00A07E04080A00000000000000E4710020E9
:10204E0000000000A87E0408080000000000000048
:10205E00F810002000000000B07E0408040000000C
:10206E00895403080000000000000000D478040822
:10207E000100000000000000000000000000000051
:10208E00000000000E000000000000000000000034
:10209E0000000000BC7E04080000000000000000EC
:1020AE000000000000000000D07E04080D000000BB
:1020BE00000000001C11002000000000E07E04085B
:1020CE0004000000E15203080000000000000000C0
:1020DE00E87E04080D000000000000001011002032
:1020EE0000000000FC7E040804000000BD5203083E
:1020FE000000000000000000D47804080100000079
:10210E0000000000000000000000000000000000C1
:10211E000E000000000000000000000000000000A3
:10212E00047F040800000000000000000000000012
:10213E0000000000187F04080700000000000000E7
:10214E005811002000000000247F04080800000041
:10215E00000000004C11002000000000307F040839
:10216E0008000000000000004011002000000000E8
:10217E003C7F04080800000000000000341100201D
:10218E0000000000487F0408080000000000000066
:10219E002811002000000000D4780408010000007F
:1021AE000000000000000000000000000000000021
:1021BE000E00000000000000000000000000000003
:1021CE00547F040800000000000000000B060020F1
:1021DE0000000000607F04080B00000000000000FB
:1021EE00C011002000000000687F04080B000000F2
:1021FE0000000000B411002000000000747F0408ED
:10220E000B00000000000000A811002000000000DC
:10221E00807F04080B000000000000009C110020CD
:10222E00000000008C7F04080B000000000000007E
:10223E009011002000000000987F04080B000000A1
:10224E00000000008411002000000000A07F0408A0
:10225E000B000000000000007811002000000000BC
:10226E00AC7F04080B000000000000006C11002081
:10227E0000000000B87F0408080000000000000005
:10228E006011002000000000D47804080100000056
:10229E000000000000000000000000000000000030
:1022AE000E00000000000000000000000000000012
:1022BE00C47F0408000000000000000000000000C1
:1022CE0000000000D87F0408080000000000000095
:1022DE00F011002000000000E47F04080800000058
:1022EE0000000000E411002000000000F07F040850
:1022FE000800000000000000D811002000000000BF
:10230E00FC7F04080800000000000000CC11002033
:10231E0000000000D4780408010000000000000056
:10232E000000000000000000000000000E00000091
:10233E0000000000000000000000000004800408FF
:10234E000000000000000000080600200000000051
:10235E00148004080B000000000000002012002072
:10236E0000000000208004080B00000000000000A8
:10237E0014120020000000002C800408070000004A
:10238E00000000000C12002000000000388004083D
:10239E0007000000000000000412002000000000F2
:1023AE00448004080700000000000000FC1100201B
:1023BE0000000000D47804080100000000000000B6
:1023CE000000000000000000000000000E000000F1
:1023DE000000000000000000000000005080040813
:1023EE0000000000000000000806002000000000B1
:1023FE005C80040807000000000000006C12002042
:10240E0000000000648004080700000000000000C7
:10241E0064120020000000006C8004080700000019
:10242E00000000005C120020000000007480040810
:10243E000700000000000000541200200000000001
:10244E007C80040807000000000000004C120020F1
:10245E000000000084800408070000000000000057
:10246E0044120020000000008C80040807000000C9
:10247E00000000003C1200200000000094800408C0
:10248E0007000000000000003412002000000000D1
:10249E009C80040807000000000000002C120020A1
:1024AE0000000000D47804080100000000000000C5
:1024BE000000000000000000000000000E00000000
:1024CE00000000000000000000000000A4800408CE
:1024DE000F00000000000000314D03080000000056
:1024EE00741200209270002017000000043A0408B5
:1024FE00917000200A3201009070002001FA010054
:10250E008C70002000C801008A700020E803D007FC
:10251E00010000004B414B5554454634000000006D
:10252E00347000200003010033700020000301000E
:10253E00AC8004080F000000554C0308314C030812
:10254E000000000050130020B88004080F000000A7
:10255E00F94B0308B94B030800000000C813002014
:10256E00C48004080F000000914C0308794C030846
:10257E00000000007C140020D08004080F00000032
:10258E00474D0308000000008D5203087417002009
:10259E00D88004080F0000007D49030800000000E9
:1025AE0000000000C4170020E08004080F000000A7
:1025BE0065540308A54F0308A14F0308A018002077
:1025CE00E88004080F0000006D4D030800000000B5
:1025DE000000000054190020F08004080F000000D5
:1025EE00114E0308E14D030800000000E019002021
:1025FE00F88004080F0000008D4E0308D54E030826
:10260E0000000000801A00209C71002001030100D0
:10261E00048104080F000000AD4D0308814D03082E
:10262E0000000000701B00200C8104080F00000049
:10263E00414E03080553030800000000FC1B002058
:10264E00188104080F000000054F030851530308BA
:10265E00000000009C1C0020967100200103010068
:10266E0020810408000000000000000000000000AF
:10267E00000000002C81040808000000000000008B
:10268E00C81D00200000000034810408070000006F
:10269E0000000000C01D002000000000448104085E
:1026AE000700000000000000B81D00200000000020
:1026BE00508104080700000000000000B01D00203B
:1026CE00000000005C8104080D0000000000000006
:1026DE00A41D002000000000688104080300000013
:1026EE00B19503088C1D002000000000D47804086A
:1026FE0001000000000000000000000000000000CB
:10270E00000000000E0000000000000000000000AD
:10271E0000000000708104080000000000000000AE
:10272E000000000000000000808104080A00000084
:10273E0000000000B8420408000000008881040870
:10274E000A00000000000000004304080000000022
:10275E00908104080A00000000000000B4710020FF
:10276E0000000000988104080A000000000000002C
:10277E00D41D002000000000D478040801000000E1
:10278E00000000000000000000000000000000003B
:10279E000E0000000000000000000000000000001D
:1027AE00A0810408000000000000000000000000EE
:1027BE0000000000AC81040803000000B19503087E
:1027CE00201E002000000000BC8004080300000052
:1027DE00B1950308081E002000000000B080040818
:1027EE0003000000B1950308F01D0020000000005A
:1027FE00B8810408050000000000000032700020BF
:10280E0000000000C0810408070000000000000066
:10281E00E81D002000000000CC8104080700000025
:10282E0000000000E01D002000000000D478040825
:10283E000100000000000000000000000000000089
:10284E00000000000E00000000000000000000006C
:10285E0000000000D8810408000000000000000005
:10286E000000000000000000EC81040803000000DE
:10287E00B1950308681E002000000000F8810408CE
:10288E0003000000B195030824040020000000009E
:10289E000082040803000000B1950308501E0020BA
:1028AE00000000000882040803000000B195030830
:1028BE00381E002000000000D4780408010000003B
:1028CE0000000000000000000000000000000000FA
:1028DE000E000000000000000000000000000000DC
:1028EE001482040800000000000000000000000038
:1028FE000000000020820408070000009D5303081A
:10290E00181F0020000000000C7E040803000000C9
:10291E00B1950308001F0020000000002C8204085F
:10292E0003000000B1950308E81E0020000000001F
:10293E003482040803000000B1950308D01E002065
:10294E00000000003C8204080700000081530308C9
:10295E00C81E002000000000D47904080300000007
:10296E00B1950308B01E0020000000004882040844
:10297E0003000000B1950308981E0020000000001F
:10298E005482040803000000B1950308801E002045
:10299E0000000000D47804080100000000000000D0
:1029AE000000000000000000000000000E0000000B
:1029BE00000000000000000000000000608204081B
:1029CE000F000000ED4C0308A94C030800000000A6
:1029DE00201F0020688204080F000000754F0308B6
:1029EE000000000000000000D41F002074820408C4
:1029FE000F0000009D4B0308814B030800000000F0
:102A0E00602000207C8204080F00000000000000FF
:102A1E000000000000000000142100208C82040839
:102A2E000F0000004D4F0308B953030800000000CB
:102A3E00A021002094820408000000000000000085
:102A4E000000000000000000BC600408030000004D
:102A5E00B1950308DC2200200000000080820408EB
:102A6E0003000000B1950308C422002000000000FE
:102A7E007882040803000000B1950308AC22002000
:102A8E0000000000A082040803000000B1950308B6
:102A9E009422002000000000AC8204080300000015
:102AAE00B19503087C22002000000000B4820408C7
:102ABE0002000000C994030800000000000000009E
:102ACE00BC82040802000000C99403080100000043
:102ADE0000000000C882040802000000C994030828
:102AEE000200000000000000000000000E000000C8
:102AFE0000000000000000000000000001000000C7
:102B0E00685E0C00430000000000000000000000A2
:102B1E0000000000000000000000000000000000A7
:102B2E000000000043000000000000000000000054
:102B3E000000000000000000000000000000000087
:102B4E000000000043000000000000000000000034
:102B5E000000000000000000000000000000000067
:102B6E000000000043000000000000000000000014
:102B7E000000000000000000000000000000000047
:102B8E0000000000430000000000000000000000F4
:102B9E000000000000000000000000000000000027
:102BAE0000000000430000000000000000000000D4
:102BBE000000000000000000000000000000000007
:102BCE0000000000430000000000000000000000B4
:102BDE0000000000000000000000000000000000E7
:102BEE0000000000C5E4030805E303080000000030
:102BFE00708504083B7B0408CA760408CA7604086C
:102C0E00CA760408CA760408CA760408CA76040886
:102C1E00CA760408CA760408CA760408FFFFFFFFC6
:102C2E00FFFFFFFFFFFFFFFFFFFF0000010041530B
:102C3E0043494900000000000000000000000000B1
:102C4E0000000000000000000000000000004153E2
:102C5E004349490000000000000000000000000091
:102C6E000000000000000000000000000000000056
:102C7E0034250020000000000000000000000000CD
:102C8E000000000000000000000000000000000036
:102C9E000000000000000000000000000000000026
:102CAE000000000000000000000000000000000016
:102CBE000000000000000000000000000000000006
:102CCE0000000000000000000000000000000000F6
:082CDE000000000001000000ED
:1080000070B4EFF31186502383F31288436B1A6820
:10801000D20720D45D686DB9446A826A944217D051
:1080200081691144D9600ED9A21A5A608462002273
:1080300080F858201A6842F00102F1B21A6081F308
:10804000118870BC704701698A1A5A608562EEE730
:10805000012380F85830F3B283F3118870BC704765
:10806000436A8269D154436A0169426B01338B428E
:1080700028BF00234362002A2FD0EFF31182502340
:1080800083F31288436B1968C9072CD470B45E68F7
:108090006EB9456A816A8D4217D084690C44DC60F0
:1080A0000ED9691A59608562002180F85810196844
:1080B00041F00101D2B2196082F3118870BC70479F
:1080C0000469611A59608662EEE7012380F858302E
:1080D000D2B282F3118870BC7047426DD36843F00E
:1080E0008003D3607047D2B282F31188704700BF1B
:1080F000026B10B462B1836CC2684469D11A013B4F
:10810000615C5DF8044B08BF13468364C8B27047D6
:10811000016A4369C4685B5C0131A14228BF114612
:1081200001625DF8044BD8B2704700BF436B13B1D6
:1081300090F858007047836A406A181AB0FA80F0C5
:1081400040097047416A836A99420AD3CB1A416B4E
:10815000026961B14968501E0B4483420AD2C01AB9
:10816000704702691144CB1A416B0029F2D1501EAD
:10817000C01A704700207047036B43B1826C5B6884
:1081800093422FBF981AC0689B1AC0187047C269E3
:10819000036A9A422FBFD01AC0688018C01A70476D
:1081A0000A4B30B503F1140493F900205D78072AD7
:1081B000C8BF143A811804330D7313F8025C855458
:1081C00013F8012C0A76A342EED130BDBC0A040894
:1081D00003682DE9F041DF691FB13B46BDE8F0417E
:1081E0001847002A164611DD04460D460E4400E0ED
:1081F00023689B68204698470028F9D0236815F823
:10820000011B1B6820469847AE42F1D1BDE8F081C2
:1082100010B424212524262200230470417082708A
:10822000C3705DF8044B7047152303701623C370A9
:10823000172383713A2383703B2343713C230372DA
:10824000704700BF40F2E93300E0A3B10289013B6F
:1082500012F0020F9BB2F8D089B2818140F2E9336B
:1082600000E043B10289013B12F0010F9BB2F8D04C
:108270008089C0B27047094A904205D0084B9842A5
:1082800001D0FF2070470223064A02EB03135A89EC
:10829000013292B25A815889C0B270470030014011
:1082A000003C004068AA002030B4846814B1236800
:1082B000A5885D83436840F2E93001E0002832D0B0
:1082C0001D89013815F0020F80B2F7D089B299816B
:1082D00040F2E93101E0002947D01889013910F056
:1082E000010F89B2F7D0998940F2E93100E059B322
:1082F0001889013910F0020F89B2F8D092B29A8130
:1083000040F2E93201E0002A3FD01989013A11F028
:10831000010F92B2F7D09B8914B12368A2881A8307
:10832000012030BC704721498B4204D0A1F5744133
:108330008B42D9D102201E4901EB00104189013145
:1083400089B241814189CFE7184A934204D0A2F50E
:1083500074429342E0D10221154B03EB01114B898A
:1083600001339BB24B814B89D6E71048834203D03F
:1083700010498B42B8D102210D4800EB0111488908
:10838000013080B248814989AEE708498B4203D069
:10839000084A9342C0D10222054B03EB02125389D3
:1083A00001339BB253815389B6E700BF00300140CF
:1083B00068AA0020003C0040F0B484894FF6FF76A4
:1083C0004FF47A7443B3002938D00F78013101E0BB
:1083D000B4421AD00589013C15F00205A4B2F7D0C9
:1083E000BCB284814FF47A7402E0BCB2B4420CD0C7
:1083F000058915F0010504F1FF37F6D08589ADB286
:108400000AB115700132013BDCE70D4B984207D0F1
:10841000A3F57443984202D00120F0BC70470225B6
:10842000084B03EB05156B8901339BB26B8168899F
:1084300080B2003018BF0120F0BC7047FF27C9E7A9
:108440000030014068AA002070B50546806810B170
:1084500004688088608341F08001686840F2E934F4
:1084600000E0E4B10689013C16F0020FA4B2F8D096
:1084700089B2818140F2E93100E009B30489013910
:1084800014F0010F89B2F8D081890021FFF794FF21
:10849000AB6813B11A689B881383012070BD104923
:1084A000884204D0A1F574418842EED102240D49DE
:1084B00001EB04146189013189B261816189E4E7CA
:1084C000074CA04203D008498842DED10221054C66
:1084D00004EB01114C890134A4B24C814989D4E7E1
:1084E0000030014068AA0020003C0040002870B520
:1084F0001EDB0928044620DD012303EB83035B0018
:10850000B0FBF3F2092AF8D87BB10E4EB4FBF3F0BE
:108510000928CCBF57223022A6FB03E5024403FB07
:108520001044EB0801F8012BF0D100230B7070BD53
:108530002D230B7040420131DBE7303001F8010B95
:10854000F3E700BFCDCCCCCC884230B44FF001046F
:108550002ED301FB04F4B0FBF4F58D42F9D284B1C3
:10856000AAB901E0B0FBF4F5092DCCBF57223022A7
:108570002A4404FB150003F8012BB4FBF1F4002C92
:10858000F0D100221A7030BC7047B0FBF4F5092D11
:10859000CCBF372230222A4404FB150003F8012BFC
:1085A000B4FBF1F4002CF0D100221A7030BC7047FB
:1085B0000546002AEBD1D7E703685A1C0260197000
:1085C000704700BF2DE9F047089C2578002B8046B6
:1085D00089460CBF4FF0200A4FF0300A661C35B3B5
:1085E000002A29DD334601E0024698B113F8011B49
:1085F000501E0029F8D1971E60B13D46013D5146FD
:108600004046C8476B1C002BF8DC257827EAE7704A
:10861000013055B1041B29464046C847301916F8A9
:10862000015B002DF7D1BDE8F087BDE8F087002A97
:1086300004DC2846BDE8F0870020EBE7571EDCE7A6
:1086400083684268D0ED037A00EB830101339342E3
:1086500081ED040A836004BF0023836000EB830381
:1086600093ED047A036870EE277A9A42C0ED037A9C
:1086700077EEC77AC0ED037A0CDA013307EE103AD1
:10868000F8EEC76AB7EE007A87EEA60A036030EE0E
:10869000070A704707EE102AB8EEC77A87EE870AF6
:1086A000704700BF90ED057A90ED004AD0ED066A64
:1086B000D0ED014AD0ED047A90ED035AD0ED025A84
:1086C000A4EE007AB0EE406AB0EE470AB0EE667AE9
:1086D000A6EE247A67EEC07AA0EE457AE6EE257A19
:1086E00080ED057AC0ED067A704700BFD0ED057ABF
:1086F00090ED013AD0ED003AD0ED064A90ED024AF5
:1087000090ED077A90ED035A90ED086AD0ED045A87
:10871000C0ED067AF0EE406A27EE830AC0ED056AE6
:10872000A3EEA60A80ED087AA4EE240AA5EE470A75
:10873000A5EEC60A80ED070A704700BFD0ED007AAB
:1087400090ED017A30EE670AE7EE007AB0EE670A44
:10875000C0ED007A704700BF704700BF0A449142E5
:1087600014D030B40139551E41F2210211F8014FE5
:10877000082380EA042004044CBF82EA4000400041
:10878000013B80B2F7D18D42F0D130BC704700BFC1
:108790002DE9F04FDFF8F8C1DFF8F8E1BCF80A7016
:1087A000DEF80060BCF80C30BCF808A03C028BB0CE
:1087B000361B4FF00004CDE90034009CBCF80630B5
:1087C0004FEA17654FF0000767EB0507B946B0465B
:1087D000A4FB06670024CDE90634009C002304FBBB
:1087E00009770024CDE90034AAFB0823CDE9022350
:1087F000039AF30D00930AFB09230393009B43EABA
:1088000047230093029B4FEAD31AFB150193039B66
:108810004AEA436ADDE9002344464D46CDE908456E
:10882000069C12F5FA62A4FB086743F1000304FBFF
:108830000977CDE90623BCF80440039BBCF802206D
:108840004FEAE31B230C059323040493340A44EA00
:1088500007643D12DDE904674FEAC23816EB0A06E9
:1088600047EB0B0718EB0408DDE906344FEA5249E1
:1088700049EB0509B3F5FA6F74F10004B246BB4643
:108880003CDADDE90067BC00B20044EA9673B41834
:1088900047EB030522463C462B4602FB04F406FB4D
:1088A0000344A2FB06232344940844EA83749D10E6
:1088B0005B104FEA3202B8EB040869EB0509BAEB2A
:1088C000020A6BEB030BDDE90623304C4FF0FF355A
:1088D000A242AB412CDBDDE90856A5FB052305FBD5
:1088E00006F403EB4403D40F44EA4304DD17DDE947
:1088F0000623121B63EB0503CDE90623DEF80440D3
:10890000A4FB082304FB0933540D44EAC3245D157A
:10891000B4EB0A0A65EB0B0B4FEADA3343EA4B433D
:1089200000B1036009B1069B0B600BB0BDE8F08F8E
:1089300040F6AC52B4184FF0000347EB0305224653
:10894000A2FB022304FB05F403EB4403941843EB5E
:108950000305A4185D414FEA850CA6004CEA947CFF
:10896000B41A6CEB0305DF00D6006D104FEA340437
:1089700047EA5277921B63EB0703B8EB040869EBF5
:1089800005091AEB020A4BEB030BA4E724FAFFFFDD
:10899000DC4600209825002050F8043C012280F895
:1089A0004520103803B11847704700BF4FF40063EB
:1089B00083827047BFF34F8F0549064BCA6802F4A4
:1089C000E0621343CB60BFF34F8F00BFFDE700BFF2
:1089D00000ED00E00400FA05F8B5057B4669036880
:1089E0001F2D29D9A5F120045F682021A1400F4245
:1089F0002A4613D01022A240D960DA605A68E240B9
:108A0000D10703D5012202FA04F4DC6004463046A3
:108A1000FFF7F6FA227B23681F2A20D9A2F1200053
:108A200008215A688140114200D0D9600422596857
:108A300082400A4221D1F8BD20211C68A9400C4285
:108A40002A460CD01022AA4099609A601A68EA401F
:108A5000D207DBD5012202FA05F59D60D6E7082191
:108A600018689140014200D099600421186801FA09
:108A700002F2024203D09A60F8BDDA60F8BDF8BD98
:108A800070B4037B04681F2B08D9203B2021626847
:108A900001FA03F31A421CD170BC704720212268EE
:108AA00001FA03F31A42F7D042691449582000FB37
:108AB000021251685689CD680868296821F00101C1
:108AC0002960828992B222EA06028281A36070BC88
:108AD000704742690949582000FB021251685689C3
:108AE000CD680868296821F001012960828992B265
:108AF00022EA06028281E36070BC7047C85E0020F3
:108B000030B4094B1C786CB1084A002502EBC40450
:108B1000116893884D628889083203439BB2A24250
:108B20008B81F5D130BC7047886100208C610020BA
:108B300010B4037B01681F2B09D9203B20224C680D
:108B400002FA03F31C4214D15DF8044B7047202253
:108B50000C6802FA03F31C42F6D00C4A4068002469
:108B6000147002685DF8044B22F0010202608B6011
:108B70007047064A40680024147002685DF8044B90
:108B800022F001020260CB60704700BF535B0020FF
:108B9000F0B5C40022189200AE498B585B689D8ADC
:108BA000ADB2EEB2F7070A445CD4B70732D5BFF3D3
:108BB0005F8F167EF6B2012E00F0C780A64D1A8B8D
:108BC000BFF35F8F221801EB8202167E022E00F0A7
:108BD000D580221801EB8202167E032E00F08880D9
:108BE0009A8895F9086092B242F480629A802218BD
:108BF00001EB8202127E013296425BD1AA7A0026F4
:108C00006E72002A40F09580204401EB8000002322
:108C10004375F0BD77074ED416F0400600F0C980CA
:108C20008D4D1E8A95F908E0176AF6B207F80E60B6
:108C30005FFA8EFE0EF1010C4FFA8CFC177E85F860
:108C400008C00CF103029742664600F01C8122180E
:108C500001EB8202127E9445C9D10EF1020676B272
:108C60002E72C4E71E887C4D26F400663604360C4E
:108C70001E801E88B6B246F480661E80967E00274F
:108C80002F72002E48D06E7A002E42D0221801EBAF
:108C900082020126127E6E72022A00F0B98022182A
:108CA00001EB8202927D42F001021A82204401EB24
:108CB0008000037EF0BD684D967E0127AF72002EC6
:108CC00073D06E7A002E7BD1221801EB8202527E85
:108CD000002A00F0A3801A882E7A92B2013642F45C
:108CE000007276B21A802E721A88D205FCD47EE702
:108CF000927E002A3FF474AF6A7A002A3FF470AF84
:108D00009A8895F9086022F480621204120C9A8005
:108D10006DE7D27DFF2AB9D0221801EB8202967D41
:108D200006F0FE061E82D37DFF2BBFD0FF232B72E1
:108D3000BCE79A8822F4407212042044120C01EB22
:108D400080009A8000234375F0BD927E424D002A38
:108D50003FF435AF6A7A002A3FF431AF1A8822F423
:108D600080621204120C1A80BFF35F8F1A8B1A886C
:108D7000AE7292B242F400721A8031E7927E002AFB
:108D80003FF427AF6A7A002A3FF423AF1A8895F997
:108D9000086022F480621204120C1A809A8822F46D
:108DA00080621204120C9A8021E76A7A002A8BD022
:108DB00091E715F0800F284D3AD195F9086016E734
:108DC000167ED2F820E01F88022E95F9086045D95A
:108DD00027F480673F043F0C1F801F8AFFB20EF804
:108DE00006701F88D2F820E0BFB247F400771F80DA
:108DF000F2B21F8A561C76B2FFB20EF806709F8838
:108E0000961CBAB276B242F480622E729A806BE7F8
:108E10001A8892B242F400621A8040E71A8895F9E3
:108E2000086092B242F4807201271A806F725BE789
:108E300095F90870B7F1FF3F2CD0D669F65D1E8218
:108E400092F818E001377AB2964516462A727FF4F6
:108E5000CEAEA3E7EC39002098250020BFB247F43E
:108E600000771F801F8AFFB20EF80670F6B21F8AC5
:108E7000D2F820E0721C52B20336FFB276B20EF87E
:108E800002702E7230E79A8822F480621204120C6B
:108E90009A80DCE6D77D1F822E72957E1DB9127EE8
:108EA000002A7FF403AF9A8822F480621204120C25
:108EB0009A80FBE670B5044682B00830656A0623E6
:108EC0006A463B21A847A8B19DF804009DF80060C0
:108ED0009DF801109DF802509DF803209DF8053083
:108EE00041EA062143EA002342EA0522E182228385
:108EF0006383012002B070BD00232622036002704C
:108F00002722C270012243608360827143727047DE
:108F1000F8B50468C4F30D0405460E4604B32F6883
:108F20002FF0FCFF092840F08880454C236923F48A
:108F300040732361236943F400732361236943F081
:108F4000010323613E602FF0E9FF2369092823F024
:108F50000103236171D12B6804332B600020F8BD1D
:108F6000384B394A93422BD902F58042934226D995
:108F700002F5804293422AD902F58042934228D9D1
:108F800002F58032934226D902F50032934224D969
:108F900002F50032934222D902F50032934220D9E1
:108FA00002F5003293421ED902F5802293421CD969
:108FB000B3F1016F1BD3052005F058F9FBE7082436
:108FC0002FF0ACFF092814D04FF0FF30F8BD10246B
:108FD000F6E71824F4E72024F2E72824F0E7302409
:108FE000EEE73824ECE74024EAE74824E8E7582491
:108FF000E6E7134F3B6923F440733B613B6943F45D
:1090000000733B613B6923F0F8033B613B6943F02C
:1090100002031C433C613B6943F480333B612FF006
:109020007DFF3B6923F002033B613B69092823F084
:10903000F8033B613FF473AFC6E76FF00100F8BD82
:10904000003C024000400008FF3F0008F8B504461D
:109050000D468E180027B54201D12069F8BDE3689E
:10906000591CE160234415F8012B1A720429F2D12E
:10907000206918B9A1682046FFF74AFF2061E76020
:10908000E9E700BF70B582B004466946143028F0A5
:1090900079F8B0B19DF805009DF801609DF80210C7
:1090A0009DF803509DF804209DF8063041EA062102
:1090B00043EA002342EA0522A187E287A4F8403070
:1090C000012002B070BD00BF38B5254B1C68236B72
:1090D00073B1636D626BCAB1998A1A88C90592B27D
:1090E00001D5D20700D438BD4FF6F7721A8038BDCB
:1090F000636D99891A88890692B2EBD59206E9D5F3
:10910000E26ACAB1988880B29047E2E799891A88E2
:109110000D0692B2E0D51006DED5A26A616A8A42D7
:1091200019D0A1692569885C98800132B2FBF5F1FC
:1091300005FB1122A262CFE79B88E2696169DBB27D
:109140008B54E269E068636D0132B2FBF0F100FB21
:109150001122E261BEE7DA6822F08002DA60BBE742
:10916000C439002003685B6A03B11847704700BF29
:1091700003681B6A03B11847704700BF03682DE9F5
:10918000F041DF691FB13B46BDE8F0411847002AB6
:10919000164611DD04460D460E4400E023689B6828
:1091A000204698470028F9D0236815F8011B1B6852
:1091B00020469847AE42F1D1BDE8F08103689B6933
:1091C000184700BF03685B69184700BF03681B6945
:1091D000184700BF0368DB68184700BF03689B6837
:1091E000184700BF03685B68184700BF03681B6827
:1091F000184700BF014B1868F8E700BFCCA8002053
:1092000038B50C46097849B1054601342B68284623
:109210001B68984714F8011B0029F7D138BD00BF1F
:10922000064B53F820302BB11A689B8851690B42CA
:1092300001D1138370475383704700BF04B40020EB
:1092400003682DE9F04F03F13F4404F57E04604EBE
:10925000A40A0125345D04F01F066409032C05FAF5
:1092600006F500F0AF80042C00F0A780022C54D04B
:109270008588B5FA85F0C0F11F0080B2C40803EB01
:10928000840400F00700266A80000F27874026EA42
:1092900007062662276A01F0030602FA00F0721E32
:1092A0003843012AC1F3810CC1F300182062C1F3D5
:1092B000411137D90024224601274FF0030E03E065
:1092C000102A04F1020426D007FA02F0A84302F1A2
:1092D0000102F5D1D3F800C00EFA04F0C04300EA51
:1092E0000C0CC3F800C0D3F8008006FA04FC4CEA6A
:1092F000080CC3F800C0D3F80CC000EA0C00D8601A
:10930000D3F80CC001FA04F040EA0C00102AD8602F
:1093100004F10204D8D1BDE8F08F2E4C666C3543C1
:109320006564A5E7002002464FF0010E4FF00309E7
:1093300004E00132102A00F102003CD00EFA02F7DC
:1093400037EA0504F5D1D3F800A009FA00F4E443A4
:109350000AEA040AC3F800A0D3F800B006FA00FA3B
:109360004AEA0B0AC3F800A0D3F808A004EA0A0AE4
:10937000C3F808A0D3F808B00CFA00FA4AEA0B0ABE
:10938000C3F808A0D3F804A02AEA07075F60D3F85F
:1093900004A008FA02F747EA0A075F60DF683C406A
:1093A000DC60DF6801FA00F401323C43102ADC6023
:1093B00000F10200C2D1BDE8F08F064C266B3543A8
:1093C000256355E7034C266C3543256450E700BF01
:1093D0007C42040800380240026802F13F4303F572
:1093E0007E032DE9F04F9B0A544DEB5C03F01F0503
:1093F0005B090124032B04FA05F400F09980042B87
:1094000000F09180022B3ED001F00306731E012B69
:10941000C1F3810CC1F300188588C1F3411137D91C
:109420000024234601274FF0030E03E0102B04F124
:10943000020426D007FA03F0A84303F10103F5D193
:10944000D2F800C00EFA04F0C04300EA0C0CC2F8D7
:1094500000C0D2F8008006FA04FC4CEA080CC2F8FE
:1094600000C0D2F80CC000EA0C00D060D2F80CC0EA
:1094700001FA04F040EA0C00102BD06004F1020461
:10948000D8D1BDE8F08F2E4B5D6C2C435C64BBE7FC
:10949000002003464FF0010E4FF0030904E00133B2
:1094A000102B00F102003CD00EFA03F737EA050456
:1094B000F5D1D2F800A009FA00F4E4430AEA040A5C
:1094C000C2F800A0D2F800B006FA00FA4AEA0B0A85
:1094D000C2F800A0D2F808A004EA0A0AC2F808A05C
:1094E000D2F808B00CFA00FA4AEA0B0AC2F808A04F
:1094F000D2F804A02AEA07075760D2F804A008FAB5
:1095000003F747EA0A075760D7683C40D460D7683A
:1095100001FA00F401333C43102BD46000F1020047
:10952000C2D1BDE8F08F064B1D6B2C431C636BE76B
:10953000034B1D6C2C431C6466E700BF7C4204088F
:109540000038024010B50409013C022C17D80D4B1D
:1095500033F8142000F00F0042FA00F313F0010377
:109560000DD0012303FA00F00138104034F0E2FD81
:10957000054A064B125D104403EBC00010BD0020ED
:1095800010BD00BF884204088442040880B2002055
:10959000754B76487649774A2DE9F04F1860986008
:1095A00018619861186298621863986318649864E7
:1095B0001865986518669866186798674FF04000B8
:1095C00098864FF0800098874FF48070A3F844008D
:1095D0004FF40070A3F84C004FF480604FF0010B83
:1095E0004FF0020A4FF004094FF008084FF0100C3A
:1095F0004FF0200E4FF400674FF480564FF40055A3
:109600004FF48044A3F8540048F20000A3F804B0DB
:10961000A3F80CA0A3F81490A3F81C80A3F824C00E
:10962000A3F82CE0A3F85C70A3F86460A3F86C5076
:10963000A3F87440A3F87C004FF04000A3F8B400F6
:109640004FF08000A3F8BC004FF48070C3F8801086
:10965000C3F88810C3F89010C3F89810C3F8A0108E
:10966000C3F8A810C3F8B010C3F8B810C3F8C010FE
:10967000A3F8C400C3F8C8104FF40070C3F8D010AA
:10968000C3F8D810C3F8E010C3F8E810C3F8F0101E
:10969000C3F8F81048F20001A3F8CC00A3F8FC10BE
:1096A0004FF480604FF04001A3F884B0A3F88CA081
:1096B000A3F89490A3F89C80A3F8A4C0A3F8ACE00E
:1096C000A3F8D400A3F8DC70A3F8E460A3F8EC508E
:1096D000A3F8F440C3F80021A3F834114FF080013F
:1096E000A3F83C114FF48071C3F80821C3F810218E
:1096F000C3F81821C3F82021C3F82821C3F830216A
:10970000C3F83821C3F84021A3F84411C3F8482115
:109710004FF40071C3F85021C3F85821C3F86021F9
:10972000C3F86821C3F87021C3F8782148F2000219
:10973000A3F804B1A3F80CA1A3F81491A3F81C8119
:10974000A3F824C1A3F82CE1A3F84C11A3F8540109
:10975000A3F85C71A3F86461A3F86C51A3F8744199
:10976000A3F87C21BDE8F08F80B200200000024009
:10977000000402400008024000286AD003682DE976
:10978000F04F03F13F4404F57E045F4EA40A012527
:10979000345D04F01F066409032C05FA06F559D060
:1097A000042C00F0AC80022C59D08588B5FA85F0E5
:1097B000C0F11F0080B2C40803EB840400F007006E
:1097C000266A80000F27874026EA07062662276A56
:1097D00001F003068240701E3A430128C1F3810C58
:1097E000C1F300182262C1F341113DD90024224681
:1097F00001274FF0030E03E0102A04F1020426D0E3
:1098000007FA02F0A84302F10102F5D1D3F800C033
:109810000EFA04F0C04300EA0C0CC3F800C0D3F801
:10982000008006FA04FC4CEA080CC3F800C0D3F828
:109830000CC000EA0C00D860D3F80CC001FA04F0A8
:1098400040EA0C00102AD86004F10204D8D1BDE827
:10985000F08F70472D4C266C35432564A5E72B4CC3
:10986000666C35436564A0E7002002464FF0010EA8
:109870004FF0030904E00132102A00F102003CD04D
:109880000EFA02F737EA0504F5D1D3F800A009FA79
:1098900000F4E4430AEA040AC3F800A0D3F800B0D5
:1098A00006FA00FA4AEA0B0AC3F800A0D3F808A0A7
:1098B00004EA0A0AC3F808A0D3F808B00CFA00FAC0
:1098C0004AEA0B0AC3F808A0D3F804A02AEA07075B
:1098D0005F60D3F804A008FA02F747EA0A075F605E
:1098E000DF683C40DC60DF6801FA00F401323C4391
:1098F000102ADC6000F10200C2D1BDE8F08F034CF9
:10990000266B3543256350E77C420408003802404B
:10991000002855D0026802F13F4303F57E032DE98C
:10992000F04F9B0A544DEB5C03F01F055B090124CB
:10993000032B04FA05F444D0042B00F09780022B8B
:1099400044D001F00306731E012BC1F3810CC1F357
:1099500000188588C1F341113DD900242346012711
:109960004FF0030E03E0102B04F1020426D007FA97
:1099700003F0A84303F10103F5D1D2F800C00EFAB9
:1099800004F0C04300EA0C0CC2F800C0D2F800801A
:1099900006FA04FC4CEA080CC2F800C0D2F80CC06D
:1099A00000EA0C00D060D2F80CC001FA04F040EAE2
:1099B0000C00102BD06004F10204D8D1BDE8F08F68
:1099C00070472E4B1D6C2C431C64BAE72B4B5D6C0F
:1099D0002C435C64B5E7002003464FF0010E4FF0C6
:1099E000030904E00133102B00F102003CD00EFA11
:1099F00003F737EA0504F5D1D2F800A009FA00F41C
:109A0000E4430AEA040AC2F800A0D2F800B006FA59
:109A100000FA4AEA0B0AC2F800A0D2F808A004EA49
:109A20000A0AC2F808A0D2F808B00CFA00FA4AEA0A
:109A30000B0AC2F808A0D2F804A02AEA0707576068
:109A4000D2F804A008FA03F747EA0A075760D76874
:109A50003C40D460D76801FA00F401333C43102B3A
:109A6000D46000F10200C2D1BDE8F08F034B1D6B42
:109A70002C431C6365E700BF7C42040800380240A9
:109A800010B1036882885A83704700BF10B1036821
:109A900082881A83704700BF10B5014600BF074C8B
:109AA00023689868FFF7ECFF23685868FEF7CAFB45
:109AB00023689868FFF7EAFF00BF10BDA864002084
:109AC00018B10368828809B95A8370471A837047AE
:109AD00010B40A4B0A4A1C7801238340234052F8F1
:109AE000200029B9B3FA83F149095DF8044BE7E78F
:109AF000191C18BF01215DF8044BE1E700B40020F8
:109B000004B4002030B1036882881B691A4214BF74
:109B100001200020704700BF2DE9F0410B4E346852
:109B200073691C400FD0DFF828800127B4FA84F352
:109B3000C3F11F0307FA03F558F823000368984799
:109B4000AC437561F2D1BDE8F08100BF003C01403B
:109B5000146400202DE9F0410B4E346873691C40F9
:109B60000FD0DFF828800127B4FA84F3C3F11F0374
:109B700007FA03F558F8230003689847AC4375616A
:109B8000F2D1BDE8F08100BF003C01401464002028
:109B90002DE9F0410B4E346873691C400FD0DFF89B
:109BA00028800127B4FA84F3C3F11F0307FA03F5F1
:109BB00058F8230003689847AC437561F2D1BDE8BB
:109BC000F08100BF003C0140146400202DE9F04109
:109BD0000B4E346873691C400FD0DFF828800127D2
:109BE000B4FA84F3C3F11F0307FA03F558F823000E
:109BF00003689847AC437561F2D1BDE8F08100BFBE
:109C0000003C0140146400202DE9F0410B4E346803
:109C100073691C400FD0DFF828800127B4FA84F361
:109C2000C3F11F0307FA03F558F8230003689847A8
:109C3000AC437561F2D1BDE8F08100BF003C01404A
:109C4000146400202DE9F0410B4E346873691C4008
:109C50000FD0DFF828800127B4FA84F3C3F11F0383
:109C600007FA03F558F8230003689847AC43756179
:109C7000F2D1BDE8F08100BF003C01401464002037
:109C80002DE9F0410B4E346873691C400FD0DFF8AA
:109C900028800127B4FA84F3C3F11F0307FA03F500
:109CA00058F8230003689847AC437561F2D1BDE8CA
:109CB000F08100BF003C014014640020084A0948BC
:109CC00008B5536C43F4804353640021402236F0BE
:109CD00040FE054B4FF0FF321A60C3F8032008BD69
:109CE00000380240146400205464002003685B6A5A
:109CF000184700BF2DE9F041044618460D461646A8
:109D0000984633F04DFD2768E6722844A072294634
:109D10007D69434632462046AC46BDE8F041604787
:109D2000036810B504461B689847236820469B6863
:109D30009847A37B0133A37310BD00BF10B5036820
:109D400004469B689847FF2301226373227310BD6A
:109D500008B5FFF7F7FB38B12C2282710022C271DF
:109D60002021BDE80840D3E508BD00BF144B984250
:109D700024D003F58063984220D0028822F040026C
:109D80001204120C0280028822F038031B041B0C00
:109D900059B141F48071002991FAA1F2B2FA82F12D
:109DA00008BF4FF0FF310139C9000B439BB203805C
:109DB00003889BB243F04003038070474908DCE707
:109DC0000038004038B5044690F85900002857D1B3
:109DD00004F11405A0694FF48071FFF7C7FF236EEB
:109DE00080226B2128469847642004F0EBFE236E06
:109DF0000322682128469847642004F0E3FE236E7E
:109E000001226B21284698470F2004F0DBFE94F8CE
:109E10005320236E032A8CBF1A2218221B212846A6
:109E200098470F2004F0CEFE236E18221C212846EE
:109E300098470F2004F0C6FE236E94F852201A2192
:109E4000284698470F2004F0BDFE236E94F8542056
:109E5000192128469847642004F0B4FE236E10228E
:109E60003721284698470F2004F0ACFE2846236E81
:109E7000382101229847A0690821BDE8384075E7DC
:109E8000FFF760FB0546FFF73DFE014600289FD126
:109E9000D5B12023E871AB712846FFF739FD214683
:109EA0000F4B41F8103F284627F002F9AB88B3FA70
:109EB00083F3C3F11F03012212FA03F388D0094987
:109EC0000A6813430B6083E72946FFF721FD21460B
:109ED000034B41F8103F284627F0EAF878E700BF27
:109EE00099890008003C0140F8B5654C0601A719A6
:109EF0000546387A32F006FD3B7A03F01F015B0914
:109F00000122032B02FA01F26DD0042B66D0022B42
:109F10005CD0A31901351879FFF714FBEDB20746A1
:109F200010B11223C5718371A3195879FFF70AFB89
:109F300010B11323C5718371A3199879FFF702FB40
:109F400010B11423C5718371A5190A21EA79384625
:109F5000FFF712FC6879FFF7F5FAEA790A21FFF7B3
:109F60000BFCA879FFF7EEFAEA790A21FFF704FC67
:109F7000A359444A934247D0434A934250D0434A5C
:109F8000934259D0424A934262D0424A93426BD0A4
:109F9000414A93422CD03444227BE2B90120022270
:109FA000198801F4415141F445710A4302431A8072
:109FB0009A8B22F400621204120C07219A831982F0
:109FC0001A8892B242F040021A80F8BD334B596AA7
:109FD0000A435A629DE700200246E1E72F4B1969C8
:109FE0000A431A6195E72D4B196A0A431A6290E7F2
:109FF00002F564424FF40010536A43F400135362B5
:10A000002EF086FEA359C6E702F584324FF4805045
:10A01000536A43F4805353622EF07AFEA359BAE791
:10A0200002F500324FF48040136A43F48043136218
:10A030002EF076FEA359AEE702F5FE324FF4004053
:10A04000136A43F4004313622EF06AFEA359A2E799
:10A0500002F582324FF40050536A43F400535362C6
:10A060002EF056FEA35996E702F568424FF4801091
:10A07000536A43F4801353622EF04AFEA3598AE7D1
:10A0800068AA00200030014000380040003C004039
:10A0900000340140005001400054014000380240AB
:10A0A000427A02B9704710B504460368406804F16B
:10A0B0000A0198470023637210BD00BF437A5A1CFF
:10A0C0000344D2B242729972037A934200D802B921
:10A0D000704710B504460368406804F10A019847C8
:10A0E0000023637210BD00BF302827D0312827D04D
:10A0F000322827D0332827D0342827D0352827D016
:10A10000202827D0212827D0102827D0112827D071
:10A11000122827D0132827D0142827D0152827D075
:10A12000162805D0172808BF0F2202D0002070473C
:10A130000E22104B03EB4203587D70470022F8E7D4
:10A140000122F6E70222F4E70322F2E70422F0E715
:10A150000522EEE70622ECE70722EAE70822E8E715
:10A160000922E6E70A22E4E70B22E2E70C22E0E715
:10A170000D22DEE7BC0A040870B5448806460D4689
:10A18000C4F30B0422460021284636F0E2FB336973
:10A19000094A934209D3094A934206D222462846E5
:10A1A0001946BDE8704034F0BFB823B121462846B7
:10A1B000BDE87040184770BD4C0600084E07000807
:10A1C000064B07498B4202D30023184670471A8872
:10A1D000C2F30B029042F8D01433F3E78801000871
:10A1E0004C060008024A136823EA0000106070471A
:10A1F000D0710020F8B5174D2B78A32B28D16B78A0
:10A20000BE2B25D1022229464FF6FF70FEF7A6FA93
:10A21000114FAC1C22884AB1A618BE4218D2052A9A
:10A2200016D92146FEF79AFA3446F3E72146022270
:10A23000FEF794FA0222A118FEF790FA0634074BB3
:10A24000641B1C8041F60F53C31A58425841F8BD95
:10A250000020F8BD0040000800800008E23A00201D
:10A260002DE9F04FDFF84C914D4F8BB00326A7EB53
:10A2700009071822002104A836F06BFB494BCDF8E2
:10A28000109005971A69002A04DA474A5A6002F1C9
:10A2900088325A6001228DF82420F322DA60434B81
:10A2A000434C1B88ADF800300222694604A8FEF733
:10A2B000CDFE022269464FF6FF70FEF74FFADFF837
:10A2C000F8A080464FF0000B544539D30AAC002566
:10A2D00024F8245D0222214604A8FEF7B7FE0222DC
:10A2E00021464046FEF73AFA40BAC043ADF80800AE
:10A2F000022202A904A8FEF7A9FE079878B106ABCE
:10A30000C0F104022946184436F023FB089818B916
:10A31000069904A8FEF7FCFD0023089007939DF81A
:10A320002430089A23B11F490B6943F000430B61A5
:10A33000013E2DD0002A9CD1FFF75CFF50B32CE0EA
:10A3400065888DF80DB0C5F30B05AB1DADF8083071
:10A350002388C3F30B02ADF80A201B0B062202A9C7
:10A3600004A88DF80C30FEF771FE062202A94046C3
:10A37000FEF7F4F9616880462A4604A8FEF766FEF7
:10A38000616840462A46FEF7E9F9143480469BE7A7
:10A39000002AD1D0052003F069FF0BB0BDE8F08F93
:10A3A00000800008003C024023016745F00A0408D1
:10A3B00088010008004000084C0600080378202BA4
:10A3C000024600F10100F9D0092BF7D02D2B2CD03B
:10A3D0002B2B03BF5378B7EE000A0246B7EE000AF4
:10A3E000A3F13001C8B209289FED467A10D8F2EEE9
:10A3F000046A07EE901AF8EEE77A12F8013FE7EEEA
:10A40000267AA3F13001C8B20928B0EE677AF0D9F4
:10A410002E2B4CD003F0DF03452B0BD0F7EE007A48
:10A4200067EE276A20EE260A70475378BFEE000ACF
:10A430000246D5E710B451782D2959D02B290ABFEF
:10A440009178501C901C0024A1F13003092B53D8A3
:10A45000002303EB830301EB430310F8011FA1F179
:10A460003002092AA3F13003F3D9B3F59A7F28BF4C
:10A470004FF49A73072B42D9DFED236A1A46F7EEA1
:10A48000007A083A072A67EEA67AFAD803F007039B
:10A490002BB1F2EE046A013B67EEA67AFBD124B33E
:10A4A000C7EE276A5DF8044B20EE260A7047537802
:10A4B000A3F13001C8B2092802F10102AAD8F2EED4
:10A4C000046AF0EE665A07EE901AF8EEE77A12F890
:10A4D000013F87EEA66AA3F13001C8B2092866EEF3
:10A4E000A56A37EE067AEED994E767EE276AD9E7D0
:10A4F000901C91780124A7E7F7EE007ACFE7F7EEFA
:10A50000007AC5E70000000020BCBE4CB5EEC00AD2
:10A51000DFED317AF1EE10FACCBF30EE270A30EEE3
:10A52000670ADFED2E7A20EE270A30B5FDEEC07AFD
:10A5300087B017EE904A054684EAE470002303A929
:10A54000A0EBE4700193009302932FF0A7FF002C7F
:10A55000ACBF20232D2303A88DF8003033F020F961
:10A56000012803A924D002282DD0032805BF3023B9
:10A57000684668468DF8013036F011FA684633F0C7
:10A580000FF90338C4B222466946284636F065FA08
:10A5900000232B55284633F003F92E22431C2A545E
:10A5A0000DEB0401E81836F017FA284607B030BD65
:10A5B000302368468DF801308DF802308DF8033075
:10A5C00036F0EDF9DAE7302368468DF801308DF882
:10A5D000023036F0E4F9D1E76F12033A00007A4412
:10A5E0002DE9F041064615460846B6FBF2F43CB9A3
:10A5F00005FB1464124B1B5D00F8013BBDE8F081C4
:10A60000B4FBF2F767B90E4B05FB174705FB146463
:10A61000DA5D00F8012B1B5D00F8013BBDE8F0811D
:10A62000B7FBF2F8B8F1000F02D04046FFF7D8FFB1
:10A6300005FB1878024B13F8082000F8012BE3E71C
:10A640009042040830B402681146531C036011F8AC
:10A65000024B0160D31C517803609378151D05608F
:10A660001B0443EA0123D078234343EA006030BC53
:10A67000704700BF0368591C1A46016012F8021B9C
:10A680000260587841EA0020704700BF03685A1CF6
:10A6900002601878704700BF38B504460068154658
:10A6A00033F042FE22682A44226038BD036810B4A9
:10A6B0000A0E5C1C04601A7003680A0C5C1C0460BF
:10A6C0001A7003680A0A5C1C04601A7003685A1C3A
:10A6D000026019705DF8044B704700BF036810B446
:10A6E0000A0A5C1C04601A7003685A1C0260197024
:10A6F0005DF8044B704700BF03685A1C026010B439
:10A70000197003680A0A5C1C04601A7003680A0C5A
:10A710005C1C04601A700368090E5A1C02601970F0
:10A720005DF8044B704700BF03685A1C0260197043
:10A730000368090A5A1C0260197070472DE9F04736
:10A74000002488B080460F461E46A14605AD531C26
:10A750000393117839B3252933D1931CCDF8109088
:10A760000393507830284ED04FF0000AA0F1300308
:10A77000DBB2092B42D96C2819D0642800F09380F1
:10A7800024D825281CD063D9582876D063281BD11B
:10A7900031784046B847039A531C03931178043626
:10A7A00001340029D7D1204608B0BDE8F087039BCB
:10A7B0005A1C03921B78642B7CD02AD8252B54D1A9
:10A7C000252140460134B847039AC0E7732833D0A7
:10A7D00044D975284FD106F1040E30682B4600226B
:10A7E0000A217646FDF7B0FE049A00955346394695
:10A7F0004046FDF7E7FE039A0444A8E704AA03A92C
:10A8000027F010FCB7E7D31C039390784FF0010AB0
:10A81000ACE7732B10D05BD9752B3AD0782B96D13F
:10A82000A3F15802B2FA82F2306852092B46102185
:10A830000436FDF789FED7E73368049A009339465A
:10A8400000234046FDF7BEFE04360444039A7EE72B
:10A850000028B9D1204608B0BDE8F0876E28B3D1F2
:10A86000039A336804361C6071E72AD9582BD7D075
:10A87000632B8DD06BE77828A6D1A0F15802B2FAED
:10A8800082F2306852092B461021FDF75DFE043636
:10A89000AAE706F1040E30682B4600220A2176460C
:10A8A000FDF752FEA0E7331D306829461E46FDF72E
:10A8B0001DFE99E7331D306829461E46FDF716FE3A
:10A8C00092E7002B7FF443AF204608B0BDE8F08745
:10A8D0006E2BC6D03BE700BF0EB400B584B005AB0D
:10A8E000019053F8042B0649039301A8FFF726FFB4
:10A8F000019B00221A7004B05DF804EB03B07047AE
:10A90000B98500080FB430B583B006AB0A490B48CF
:10A9100053F8042B096800680193FFF70FFF084CF8
:10A9200005462068FEF74EFC0028FAD0284603B002
:10A93000BDE8304004B07047B8390020BC39002071
:10A94000CCA80020DFED2B7AB4EEE70AF1EE10FA86
:10A950004ADDDFED296A9FED297A01E0B0EE670A52
:10A96000B4EEC70AF1EE10FA70EE667AF6DC9FEDEF
:10A97000247AF4EEC77AF1EE10FA38D5DFED1E6ACC
:10A980009FED207A01E0F0EE407AF4EEC77AF1EE26
:10A9900010FA37EEA60AF6D4DFED1B7AB4EEE70A1A
:10A9A000F1EE10FA14DDDFED137A37EEC00A60EE37
:10A9B000006A9FED166A9FED167ADFED167AA6EE15
:10A9C000867A20EE266AE6EE877AA6EE270A704798
:10A9D000DFED117AB4EEE70AF1EE10FA44BFDFEDD5
:10A9E000087A37EEC00AE2E7F0EE407ABFE7B0EE51
:10A9F000670AD1E7DB0F4940DB0FC940E4CB1641C2
:10AA0000DB0F49C0E4CB16C1DB0FC93F92E741B968
:10AA10009730083C15A82ABEDB0FC9BF80EAE07357
:10AA2000A3EBE0738B4205DB002801DD401A704781
:10AA300002D17047002070470844704709B909E007
:10AA4000194690FBF1F301FB13030846002BF7D1E5
:10AA5000084670470146FBE7F0EEC07AB0EEE07AB8
:10AA6000B4EEE77AF1EE10FAB4BFB0EE676AB0EE7A
:10AA7000476AB5EE406AF1EE10FA46D0B4EEE77AD6
:10AA8000F1EE10FA8CBFF0EE675AF0EE475AC5EEC1
:10AA9000866A9FED1F3A9FED1F6A9FED1F4A9FED4B
:10AAA0001F5ADFED1F3ADFED1F4ADFED1F5AA6EEFA
:10AAB000C36AE6EEA34AA6EE864AB7EE006AA6EEA1
:10AAC000845AA6EEA46AE6EE855AC5EE866AB4EE0E
:10AAD000E77AF1EE10FA48BFDFED147AF5EEC00A1E
:10AAE00048BF77EEE66AF1EE10FA48BFDFED107A64
:10AAF000B5EEC00A48BF77EEE66AF1EE10FA48BF3D
:10AB0000F1EE666AB0EE660A7047DFED076ADEE7CF
:10AB100039094E3DE3B59E3E88FA163E45FE7F3F1D
:10AB200099FB243F69A2163EA7DFA834DB0FC93F7B
:10AB3000DB0F4940DFED317A30EE277AFDEEC76A50
:10AB400016EE903A2033402B02D99FED2D0A704724
:10AB5000B4EEE70AF1EE10FA4DDD9FED2A6ADFED63
:10AB60002A6A01E0B0EE677AB4EEE67AF1EE10FA06
:10AB700077EE467AF6DC9FED257AF4EEC77AF1EEB1
:10AB800010FA35D5DFED1F6A9FED217A01E0F0EE76
:10AB9000407AF4EEC77AF1EE10FA37EEA60AF6D450
:10ABA000DFED167AB4EEE70AF1EE10FA1BDCDFED0A
:10ABB000197AB4EEE70AF1EE10FA44BFDFED137A2A
:10ABC00037EEC00A60EE006A9FED136A9FED137ABC
:10ABD000DFED137AA6EE867A20EE266AE6EE877A15
:10ABE000A6EE270A7047DFED0F7A37EEC00AE9E7D5
:10ABF000B0EE670AD4E7F0EE477ABCE7DB0FC93F57
:10AC000000000000DB0FC940E4CB1641DB0F49C058
:10AC1000E4CB16C1DB0FC9BF92E741B99730083CBE
:10AC200015A82ABEDB0F4940FDEEC07A17EE903A18
:10AC30002033402B51D8DFED2D7AB4EEE70AF1EE48
:10AC400010FA50DDDFED2A6A9FED2A7A01E0B0EEBE
:10AC5000670AB4EEC70AF1EE10FA70EE667AF6DC17
:10AC60009FED257AF4EEC77AF1EE10FA38D5DFEDD4
:10AC7000206A9FED227A01E0F0EE407AF4EEC77A86
:10AC8000F1EE10FA37EEA60AF6D4DFED1D7AB4EE37
:10AC9000E70AF1EE10FA1BDCDFED1A7AB4EEE70AF0
:10ACA000F1EE10FA44BFDFED147A37EEC00A60EE21
:10ACB000006A9FED156A9FED157ADFED157AA6EE15
:10ACC000867A20EE266AE6EE877AA6EE270A704795
:10ACD000DFED067A37EEC00AE9E79FED0E0A70470E
:10ACE000B0EE670AD1E7F0EE407AB9E7DB0F4940F2
:10ACF000DB0FC940E4CB1641DB0F49C0E4CB16C1E2
:10AD0000DB0FC93FDB0FC9BF92E741B99730083C61
:10AD100015A82ABE0000000010B507EE901A2DED10
:10AD2000028BB8EE678ADFED217A28EE008A0446AE
:10AD300028EE278AB0EE480A33F04AFDF0EE408A4A
:10AD4000B0EE480A33F0A6FCF7EE007A9FED187AD1
:10AD5000F0EE675AE8EE875A0023A361B0EE676A07
:10AD6000C7EEA56A63612362E361A8EEC76ABDEC22
:10AD7000028B77EEC07AB6EE007AF8EE005A27EE34
:10AD8000877A20EE250A27EE267A26EE266A67EED7
:10AD9000A67A20EE260A84ED046AC4ED017A84EDD9
:10ADA000007A84ED027A84ED030A10BD27D4D236EE
:10ADB000F304353F10B44C09012250F8243001F05F
:10ADC0001F0102FA01F10B4340F824305DF8044BF7
:10ADD000704700BF4B0901F01F0150F823200123E9
:10ADE00003FA01F1114214BF18460020704700BF5A
:10ADF000054B06480021012210B4202499715A7194
:10AE000004815DF8044B70474C6D0020886B002076
:10AE1000074A084B10781B78074A834296BFC31A2B
:10AE2000C3F180030020126818441044704700BF2B
:10AE3000788B0020F58A002058460020064A074BF0
:10AE400010781B7883428ABFC3F18003C01AC018F0
:10AE5000C0F17F00704700BF788B0020F58A00208A
:10AE600030B5144C237883B01BB90120237003B094
:10AE700030BD052200238DF800208DF8013000BF81
:10AE80000D4D2B689868FEF7FBFD2B6801AA6946FB
:10AE9000586831F04BFE2B689868FEF7F7FD00BF4D
:10AEA0009DF8053003F0010383F00100237003B027
:10AEB00030BD00BFBA640020A864002070B5064C05
:10AEC0000646256803E023685B1BB34203D8FFF7FF
:10AED000C7FF0028F7D070BD60AA00202DE9F04F11
:10AEE00089B0B2F1000A02900491039340F3B0805C
:10AEF0000B46002201EB8A0153F8040B8B420244FB
:10AF0000FAD1039B0592002B00F09A80059B002B41
:10AF10006AD0544B059A1B68DFF85C910092009947
:10AF2000DAB25118B1F5807F8CBFC2F58072009AF9
:10AF300001924D4A92689A426DD9190C1A0A4FF043
:10AF4000020406208DF81F308DF81E208DF81D108C
:10AF50008DF81C40FFF7B2FF0620FEF79DFD434A27
:10AF60000123137000BFD9F800309868FEF788FD00
:10AF7000D9F8003007A95868002231F08FFD00246D
:10AF8000049D029E019FA34629684FEA840800227F
:10AF90000B46013471B1B9422AD2D9F800003168A8
:10AFA0004068FDF709FA2A68336813443360BF1A12
:10AFB000C5F800B0A24505F1040506F10406E3D189
:10AFC000D9F800309868FEF761FD00BF254B019964
:10AFD00000981B68421A0092224A0B441360039A9D
:10AFE00032B3009A002A9AD1059809B0BDE8F08FD3
:10AFF000029CD9F8003054F80810586800223B46EB
:10B00000FDF7DAF954F808202B683A44DF1B44F8BE
:10B0100008202F60D4E70598009C1549154A001BAD
:10B020000590059800230B70137009B0BDE8F08FF0
:10B03000059B009A9B1A0593059809B0BDE8F08F0F
:10B04000FFF70EFF00287FF461AF039B0593CBE76A
:10B05000039C1CB9FFF704FF0594C5E70023059383
:10B06000C2E700BF58460020DC030020BA6400207D
:10B07000788B0020F58A0020A864002070B5104D60
:10B08000104E2B7831788B4284B016D00E4A039242
:10B090001A4402928CBF0C46CA1A04A98CBFC3F191
:10B0A00080020024012341F8102D02A802220194FD
:10B0B000FFF714FF002333702B7004B070BD00BF86
:10B0C000F58A0020788B0020F88A002070B5194C92
:10B0D000194D23782978994284B027D0174A0392D2
:10B0E0001A44029234BF0E46CA1A04A934BFC3F1EF
:10B0F00080020026002341F8102D02A802220196AA
:10B10000FFF7ECFE23781844C0B203062B7848BF43
:10B1100080F080008342207002D0002004B070BD17
:10B12000002301202B70237004B070BD012004B0F7
:10B1300070BD00BFF58A0020788B0020F88A0020BF
:10B1400008B545F20820FFF7B9FE0620FEF7A4FC7B
:10B15000064B0122C7201A70FEF79EFC04480549E1
:10B16000054A002303700B70136008BDBA64002009
:10B17000788B0020F58A0020584600202DE9F04108
:10B1800082B00346060C050A032406208DF807301A
:10B19000884617468DF805608DF806508DF80440F6
:10B1A000FFF78CFEC0B100BF0D4C23689868FEF716
:10B1B00067FC236801A95868002231F06FFC2368FE
:10B1C0004246002158683B46FDF7F6F82368986828
:10B1D000FEF75CFC00BF384602B0BDE8F08100BF5E
:10B1E000A8640020F0B5124B9D6885B00DB905B07C
:10B1F000F0BDED0A14D0002704AE7C196410E00203
:10B2000010226946FFF7BAFF0F2809DD6B4653F895
:10B21000042B01320AD1B342F9D12546AF42ECDB0F
:10B22000FFF72CFF034BED021D60E0E7671CF5E71D
:10B23000DC030020584600202DE9F84FDFF8A880F5
:10B24000DFF8A8A0D8F80000DFF8A490234E01236F
:10B250008AF80030FEF714FC052031F0AFFC002026
:10B2600031F0ACFC062031F0A9FC002031F0A6FC46
:10B2700099F80040042044F0010431F09FFC20467E
:10B2800031F09CFC33888BB1154D164F002415F816
:10B2900004B0072031F092FC584631F08FFC2A5D53
:10B2A00033883A550134A4B2A342F0D8072031F0D4
:10B2B00085FCFF2031F082FC99F80040042031F039
:10B2C0007DFC204631F07AFCD8F80000FEF7DEFB6A
:10B2D00000238AF80030BDE8F88F00BFFC00002092
:10B2E00078470020BC4C0020606B0020A54C00205B
:10B2F000AD4C00202DE9F041474E3068FEF7C0FB11
:10B30000464B1B78012B78D05FD3022B0AD1DFF894
:10B310002C81082388F800300D254FF4C373404F6B
:10B320003B8010E0DFF814813D4F98F8003003F0C7
:10B330004003002B14BF4FF4F0734FF4C3733B80F2
:10B3400014BF10250D25002404F11000C0B231F007
:10B3500035FC0134012031F031FCA3B2AB42F3D310
:10B3600098F800402F4D002031F028FC204631F0A5
:10B3700025FC2D4B1C78022031F020FC204631F0BA
:10B380001DFC2A4B1C78032031F018FC204631F0BC
:10B3900015FC274B1C780420044331F00FFC204699
:10B3A00031F00CFC3068FEF771FB3A88214800212F
:10B3B00035F0CFFA2B7833B11F4B1B7833B3002312
:10B3C0002B70BDE8F081BDE8F081A02031F0F6FBE4
:10B3D000002031F0F3FB00F00603022BDFF85C8065
:10B3E00007D000F00500012803D1482388F8003079
:10B3F00008E0082388F800308EE7DFF84080482313
:10B4000088F8003010254FF4F07388E7FFF714FF39
:10B4100000232B70BDE8F081606B0020786B00206A
:10B42000FC000020000000207F6B0020806B0020CB
:10B43000AD4C0020BC4C0020A54C00200401002095
:10B440000C4B984213D0A3F5806398420FD003F5BC
:10B45000804398420BD003F58063984207D003F5F0
:10B460008063984203D0044B186840087047024B31
:10B470001868704700040140DC5D0020F0B5774B90
:10B48000774A87B01968914200AF00F0DB80002353
:10B49000744A3B607B60136843F48033136003E0BD
:10B4A0003B68B3F5A04F09D0136803F400337B6009
:10B4B0003B6801333B607B68002BF1D0694B1B6814
:10B4C00013F4003318BF01237B607B68012B7BD012
:10B4D000654D644B654AEA606549586F654A086086
:10B4E000AA605E6B644C654A654826F080065E6320
:10B4F0005E6F46F080765E67196B0C431C63596B78
:10B500005963996B9963196C41F05B5141F47B115C
:10B5100041F41F6141F00F011964596C07F11804DF
:10B520000A4348F2FF715A6444F8101D0026214670
:10B530000123FB733E737E73BE732DF0B5FA214673
:10B540004FF6FF734F48BB602DF0AEFA4FF6FF7316
:10B5500021464D48BB602DF0A7FA21464B482DF0FF
:10B56000A3FA21464A482DF09FFA214649482DF07A
:10B570009BFA214648482DF097FA214647482DF07E
:10B5800093FA214646482DF08FFA20462DF07EFC96
:10B59000444B454C1B68BA6844484549A4FB0343E7
:10B5A0009B09A0FB0202013B920CB3F1807F0A6071
:10B5B00007D2404AF0200721536085F823009660A7
:10B5C00011601C37BD46F0BD264B3B4C1A6C3B4905
:10B5D00042F080521A6420688A684D68C96840F455
:10B5E00040402060986898609868120640F40040D7
:10B5F000986042EA8512986842F48002490842F055
:10B600000802013942EA014240F4A05098605A60B1
:10B610001A6842F080721A601A689201FCD52849B3
:10B62000104A40F205700860996821F003019960A2
:10B63000996841F002019960936803F00C03082BAC
:10B64000FAD145E700221A6062B61E4B1B6883F3ED
:10B6500008881D4B1B689847FEE700BFFCFF0120D0
:10B66000EFBEADDE0038024000ED00E00005FA0557
:10B670009063002000000008FF916700335F07001F
:10B68000000002400004024000080240000C02409A
:10B69000001002400014024000180240001C02404A
:10B6A00000200240DC5D0020D34D621083DE1B438E
:10B6B00064AA002010E000E00070004000000020BC
:10B6C000003C02400000FF1F0400FF1F08B5054BAF
:10B6D0001B6803B19847044B044A1A6072B6FDF721
:10B6E00069F900BF88410020FCFF0120EFBEADDEFC
:10B6F00008B5034B1B6803B1984772B6FDF75AF9BA
:10B7000088410020084B10B507281B68C8BF1438B3
:10B7100018440C46007EFDF715FF20B12146BDE818
:10B720001040FEF7CDB910BD8064002030B504464E
:10B73000406D61718389A26823F400531B041B0CC4
:10B74000838185B0A379009213F0040230D04FF4C6
:10B75000805213F00203ADF8042056D1ADF8063044
:10B760004FF480630022ADF8083011F00103ADF80A
:10B770000C2028D1ADF80A3008238D07694648BF50
:10B78000ADF80A302DF016FCA279636DD10724D4F0
:10B7900012F0080F9A8A1BD122F008021204120C30
:10B7A0009A829A8992B242F400529A8105B030BDD1
:10B7B00013F00203ADF8042024D04FF400551346D3
:10B7C000ADF80650CEE70423ADF80A300C23D4E7D9
:10B7D00092B242F008029A82E3E70D498B420FD001
:10B7E000A1F548418B4209D00A498B42D0D10520AE
:10B7F0000121FFF787FFA279636DC9E70220F7E710
:10B800000020F5E7ADF80630ACE74FF40053A5E7AC
:10B81000001001400014014010B50446406DA160C5
:10B82000838923F400531B041B0C8381A37984B008
:10B8300013F00402009135D04FF4805213F002034C
:10B84000ADF8042056D1ADF806304FF4806362792C
:10B85000ADF80830D1074FF00003ADF80A30ADF86D
:10B860000C3045BF0423ADF80A3008230C23694689
:10B87000920748BFADF80A302DF09CFBA279636DAA
:10B88000D1071FD412F0080F9A8A16D122F00802AD
:10B890001204120C9A829A8992B242F400529A814E
:10B8A00004B010BD13F00203ADF804201FD04FF414
:10B8B00000511346ADF80610C9E792B242F00802F3
:10B8C0009A82E8E70D498B420FD0A1F548418B429F
:10B8D00009D00B498B42D5D105200121FFF712FF7A
:10B8E000A279636DCEE70220F7E70020F5E7ADF817
:10B8F0000630ACE74FF40053A5E700BF001001404D
:10B900000014014038B50C4B07281B68CCBFA0F1D0
:10B910001404044623440546187EFDF713FE50B177
:10B9200001342722C471827131F058F82846002171
:10B93000BDE83840E6E638BD8064002070B50F4CA5
:10B940000F4DC0EBC00004EB8004286B2669304328
:10B95000286382B09209667BA1600025012101A8BD
:10B9600063618DF804608DF805208DF806508DF820
:10B9700007102DF0E7FA02B070BD00BF1C020020D6
:10B9800000380240074BC0EBC00030B403EB80002E
:10B99000054C0569236B2B4323630176427630BC4B
:10B9A000704700BF1C020020003802402DE9F04F14
:10B9B0005B4C54F8204083B0002C00F0AC80E66D66
:10B9C000002E00F0AA809046564A356922609946BA
:10B9D00004F2622204F162036361A2614FF4007316
:10B9E0007268A1600746E36023616265A246B5B153
:10B9F0004D4B00205A68954203F11C0376D001306C
:10BA00001028F7D100207A1CD2B20C21FFF7BAFF20
:10BA1000636DB168326922630433A1632365F06802
:10BA2000E8B1414B00215A68904203F11C035BD0FE
:10BA300001311029F7D100257A1CD2B20B212846FA
:10BA4000FFF7A0FF2346F27F38492846FFF776FF2D
:10BA5000636DB168F26862630433E163E36494F890
:10BA60006100FDF76FFD054694F86000FDF76AFD83
:10BA70008346307F00284BD119F0080F38D118F0D9
:10BA8000020F09D045B10B227B1CAA71EB7128462D
:10BA9000727F2221FDF770FE18F0010F15D1A36B04
:10BAA0007BB996F82020B17F8DF8063001A8930964
:10BAB00001228DF805308DF804108DF807202DF047
:10BAC00041FA504603B0BDE8F08FBBF1000FE6D05D
:10BAD00001370C238BF807708BF806305846727FBD
:10BAE0002221FDF749FEDAE7CDB2A5E7C0B28AE729
:10BAF0000137FFB215B10B23EF71AB7119F0100FC5
:10BB0000284614BF02211221727FFDF735FEC6E7D9
:10BB100030F0F8FEB0E7A246D3E7B246D1E700BF67
:10BB2000C4390020F40A04081C020020D989000846
:10BB30000348D0F8AC3113B100F5D2701847704704
:10BB40001C0200200348D0F8903113B100F5C470F6
:10BB5000184770471C0200200348D0F8743113B115
:10BB600000F5B670184770471C0200200348D0F853
:10BB7000583113B100F5A870184770471C02002017
:10BB80000348D0F83C3113B100F59A70184770475C
:10BB90001C0200200348D0F8203113B100F58C704E
:10BBA000184770471C0200200348D0F804310BB13D
:10BBB000FC301847704700BF1C0200200348D0F833
:10BBC000E8300BB1E0301847704700BF1C0200207E
:10BBD0000348D0F8CC300BB1C4301847704700BFD1
:10BBE0001C0200200348D0F8B0300BB1A830184731
:10BBF000704700BF1C0200200348D0F894300BB1FE
:10BC00008C301847704700BF1C0200200248836F29
:10BC10000BB17030184770471C0200200248C36DFA
:10BC20000BB15430184770471C0200200248036CC7
:10BC30000BB13830184770471C0200200248436A95
:10BC40000BB11C30184770471C0200200248836863
:10BC500003B11847704700BF1C020020431C00F0CE
:10BC60000E812DE9F04F4FEAC00808EB00039B005E
:10BC7000DFF8E8A25AF803B087B00AEB0304BBF17F
:10BC8000000F00F0F98014330AEB03010022DBF807
:10BC900004704AF803204A608A60CA600346A568B7
:10BCA00001900133D4F80C90DBB2002D00F0E88055
:10BCB0001522EB71AA71B9F1000F00F0FA8016227B
:10BCC00089F8062089F807309BF80E0030F01AFE3C
:10BCD000BB8823F440731B041B0CBB802846FDF774
:10BCE000D5FE4846FDF7D2FE11212846FDF774FB2C
:10BCF00011214846FDF770FB0826642403E03CB19F
:10BD000030F01EFE013C2846FDF7FCFE0028F6D070
:10BD10002846FDF7B5FE30F013FE2846FDF7B6FEC7
:10BD200030F00EFE013EEED14846FDF7A9FE30F0A0
:10BD300007FE2846FDF7A4FE30F002FE2846FDF778
:10BD4000A5FE30F0FDFD4846FDF7A0FE019B08EB87
:10BD500003040AEB84042846637C002B0CBF1221E9
:10BD600032210422FDF708FD637C002B0CBF122159
:10BD7000322148460422FDF7FFFC704B9F4200F041
:10BD8000B7806F4B9F4200F0BD806E4B9F4200F02A
:10BD9000A580BB8801996C4A6C4C23F440731B044A
:10BDA0001B0CBB803B8888440AEB880A9BB243F09B
:10BDB00001039AF810103B80BD8802A8002918BF23
:10BDC00014462DF063F8049A6148B2FBF4F325F0B1
:10BDD0003F05A0FB02122D04900C2D0C0543BD80E5
:10BDE0005C4C39884FF4967202FB00F284FB0240EF
:10BDF0009BB2D217002BC2EBA01221F0010108BFA9
:10BE000001230904013243F40043090C92B2398042
:10BE10003A84BB833B889BB243F001033B803B8861
:10BE200023F4816323F002031B041B0C43F480639F
:10BE30004FF480423B803A813B8823F080031B040F
:10BE40001B0C3B809BF810308DF808300024012338
:10BE500002A88DF80B308DF809408DF80A402DF0BE
:10BE600071F89BF80F308DF8083002A88DF8094062
:10BE70008DF80A402DF08CF807B0BDE8F08F7047C0
:10BE8000B9F1000F48D0162289F8073089F806204A
:10BE90009BF80E0030F036FDBB8823F440731B0482
:10BEA0001B0C2846BB80FDF7F1FD4846FDF7EEFD73
:10BEB0001EE79BF80E0030F025FDBB8823F440738D
:10BEC0001B041B0CBB802846FDF7E0FD4846FDF730
:10BED000DDFD11212846FDF77FFA0DE71E4A136AA2
:10BEE00043F4000313624FF400002CF019FF50E7F5
:10BEF000194A136A43F4001313624FF400102CF034
:10BF00000FFF46E7144A136A43F4800313624FF4A9
:10BF100080002CF005FF3CE79BF80E0030F0F2FCAF
:10BF2000BB8823F440731B041B0C4846BB80FDF701
:10BF3000ADFD4846FDF7AAFDDEE600BF0054004017
:10BF400000580040005C0040009F2400804F120019
:10BF500083DE1B43D34D621000380240EC390020D1
:10BF6000F8B54FEAC00E274F069C0EEB000507EB15
:10BF700085056E68002E42D04900C9B2A9754FF000
:10BF8000000C0121EA7585F819C0A9762B76697530
:10BF900085F814C0B3882C629905EC6114D43388F9
:10BFA000DA050CD44FF4805401E0013C1ED03388F4
:10BFB0009B05FAD433889BB243F480733380B388F3
:10BFC0009BB243F44073B3800EEB000107EB810298
:10BFD0004FF4805401E0013C08D0537D002BFAD18E
:10BFE00007EB81073C7D84F00100F8BD064A138809
:10BFF00001339BB21380FFF731FE2046F8BD304677
:10C00000F8BD00BFEC390020E03A002070B590F98F
:10C0100004506C1C82B00AD0032D08DC16460A4678
:10C02000417900962846FFF79BFF02B070BD0020C3
:10C0300002B070BD00B50378012B83B004D1032397
:10C0400001AA0021FFF7E2FF9DF805309DF80420CA
:10C050009DF806001B0243EA0243184303B05DF853
:10C0600004FB00BF08B5FFF7E5FF014B586008BDB2
:10C070009825002008B5FFF7DDFF014B186008BDCB
:10C0800098250020F0B585B002AB0446009303224A
:10C0900006231E210020FFF763FF00283CD09DF8F7
:10C0A00008509DF809109DF80A709DF80B209DF826
:10C0B0000C609DF80D3041EA052142EA072243EA6F
:10C0C000062309B212B21BB2144D06EE901A07EE07
:10C0D000102A07EE903AF8EEE66A95ED045AD5ED8F
:10C0E000065A95ED056AB8EEC77AF8EEE77A66EE7D
:10C0F000856A27EE257A67EE867AFDEEE66ABDEE62
:10C10000C77AFDEEE77A16EE901A17EE102A17EEB0
:10C11000903A2180A280638005B0F0BD000000202D
:10C1200000B583B0002000920A466821FFF718FF8F
:10C1300003B05DF804FB00BFF0B5C60033189B00E8
:10C14000254DEA585468A28A83B092B20192019AAE
:10C150002B4412F4706F1CBF01221A75019B13F45B
:10C16000E06F07460CD1A38A3E4423F4706305EBCD
:10C1700086051B041B0C0022A3826A7503B0F0BD68
:10C18000238BA38823F480631B041B0CA380019BD7
:10C190009B05E8D423889805E5D42388D9050ED5D6
:10C1A0002388DA05FCD423889BB243F400732380F0
:10C1B00023889B05FCD43846FFF750FDD3E723883E
:10C1C0009BB243F400732380A38823F440731B04C1
:10C1D0001B0CA380C7E700BFEC390020F0B583B08B
:10C1E000441C8DF8073001D0032802DD002003B085
:10C1F000F0BDC700244E3B1806EB83035D68002D9D
:10C20000F4D04900C9B2997501240021DA755C7631
:10C2100099761C765C751975A9880DF10702890558
:10C22000DA611A6214D42B88DA050CD44FF48054E6
:10C2300001E0013C1ED02B889B05FAD42B889BB2D1
:10C2400043F480732B80AB889BB243F44073AB8084
:10C25000074406EB87024FF4805401E0013C09D00B
:10C26000537D002BFAD106EB87073C7D84F001005B
:10C2700003B0F0BD054A138801339BB21380FFF76A
:10C28000EDFC2046B3E700BFEC390020E03A002087
:10C290002DE9F043322083B002F094FC00221046D6
:10C2A00011231E21FFF79AFF602301221E21002087
:10C2B000FFF794FF642002F085FC6846FFF7E2FE7A
:10C2C0000024DFF85481254626460A27012302224E
:10C2D0001E210020FFF782FF322002F073FC684627
:10C2E000FFF7D0FEBDF902E0BDF90410BDF9002052
:10C2F0008E457346A8BF0B469342A8BF13464345DD
:10C300004FF0010075440C44164479DBFCF788FFBC
:10C31000013FDBD14FF001090022104612231E21FC
:10C32000FFF75CFFDFF8F0800A27012302221E21BD
:10C330000020FFF753FF322002F044FC6846FFF76D
:10C34000A1FEBDF902E0BDF90410BDF900208E4543
:10C350007346A8BF0B469342A8BF134643454FF010
:10C360000100A5EB0E05A4EB0104A6EB02064ADBD7
:10C37000FCF756FF013FD8D107EE906AF8EEE76A66
:10C3800007EE905AB8EEE77A07EE904ADFED1F5AB3
:10C390009FED1F5A1F4EF8EEE77A85EEA66A00223F
:10C3A000104670231E21C5EE876A85EE277AB0EE0F
:10C3B000C66AF0EEE66AF0EEC77A86ED046AC6ED6C
:10C3C000056AC6ED067AFFF709FF202301221E2128
:10C3D0000020FFF703FF0023184602221E21FFF76B
:10C3E000FDFE642002F0EEFBB9F1000F04D14FF026
:10C3F0007E5333617361B361012003B0BDE8F08304
:10C400004FF0000988E74FF00009B5E700406F469C
:10C4100001C05E460000002001F0FFFF0378012B01
:10C4200000D07047417990F904005822D6E600BF49
:10C430000378012B00D07047417990F9040048221D
:10C44000CCE600BF134600200A466821C6E600BFBE
:10C450000220FCF79DBB00BF02206DE60120FCF727
:10C4600097BB00BF012067E60020FCF791BB00BF2F
:10C47000002061E61549164B16484A6810B4CC688E
:10C480001549B2FBF4F203FB02F30360D1F88820F4
:10C49000124B134C42F47002C1F888201A68002035
:10C4A00042F001021A6098601A6822F0847222F445
:10C4B00080321A605C601A684FF0006422F48022B7
:10C4C0001A60D8608C605DF8044B70470000002053
:10C4D00040420F00DC5D002000ED00E0003802402B
:10C4E00010300024044B4FF4F07002210A225860EF
:10C4F000D9609A60FFF7BEBF0000002038B50B4C32
:10C5000023688BB15A68821A002A054604DA0CE0C7
:10C510005A68AA1A002A07DB9A68226018461A6825
:10C5200090472368002BF3D138BD38BDA43E0020CE
:10C530000B4B002210B4027203F1A804012102E0A7
:10C54000072A09DC9979890702D5197981540132C2
:10C550009C4203F11803F3D15DF8044B704700BF10
:10C56000EC32040837230370704700BF012310B476
:10C5700032213324312244704171C270037003713F
:10C5800083705DF8044B70472322032302704370CD
:10C59000704700BF08B519F07DFFFFF7A9F800BF8D
:10C5A000024A034B1278197827F07EBFB425002089
:10C5B000B5250020038A2DE9F0478589ADB21D40DD
:10C5C00029D00F4606464FF000484FF00009B5FA53
:10C5D00085F328FA03F2D24391B21B3B1540318216
:10C5E000042B16D8DFE803F03129211903007B6AF8
:10C5F000002B32D003F1FF3A1FFA8AFAC7F82490D1
:10C600003C6A34B123682046514698476468002C40
:10C61000F8D1002DDBD1BDE8F0873868716B036875
:10C6200089B29847002DD2D1F5E77868B16B0368DD
:10C6300089B29847002DCAD1EDE7B868F16B03685D
:10C6400089B29847002DC2D1E5E7F868316C0368DC
:10C6500089B29847002DBAD1DDE7F36A1FFA83FA51
:10C66000CEE700BF2DE9F04F2DED028BA0F10A03BC
:10C6700089B00C46E72B00F22B87DFE813F01C0192
:10C68000290729072907290729072907290729072A
:10C69000290729072907290729072907290729071A
:10C6A00029072907290729072907290729078001B9
:10C6B0002907290729077101290729072907640183
:10C6C00029076F0229072C022907210229071902CD
:10C6D0002907F4012907E001290729072907DA01B9
:10C6E000D30129078803290729078103290759034B
:10C6F0002907290729073D032907290729072907AA
:10C70000E4022907FC002907260303032907290758
:10C7100029072907290729072907F0042907C2043F
:10C7200029078E0429073A0429072604290729071F
:10C7300029072907D00396038F03B302E8000A06EE
:10C74000F5052F06E8052907B005930529072907F0
:10C7500029072907750529072907530529072907E7
:10C760002907B7069F068A064706290729072907CA
:10C77000DF06C706190732052907290729072907F0
:10C780002907290729072907290729072907290729
:10C79000290729072907D003290729072907290776
:10C7A0002907290729072907290729072907290709
:10C7B00029072D01290729072907290729072907FB
:10C7C00029072907290729072907290729072907E9
:10C7D00029072907290729072907290729072907D9
:10C7E00029072907290729072907290729072907C9
:10C7F00029072907290729072907290729072907B9
:10C8000029072907290729072907290729072907A8
:10C810002907290729072907290729072907290798
:10C820002907290729072907290729072907290788
:10C830002907290729072907290729072907290778
:10C84000290729072907290729079E01A901AE4EB3
:10C85000337853B1AD4F002537F8021F2046FDF75E
:10C8600063FF33780135AB42F6DC012009B0BDEC43
:10C87000028BBDE8F08FA44E3378002BF5D0A44F87
:10C880000025B846236817F81520591C21601A7036
:10C8900098F8011001EB810101EB810101F2EE2119
:10C8A00089B22046FDF740FF33780135AB4208F1ED
:10C8B0000208E7DCD9E7974D284630F071FF0028E1
:10C8C000D3DD2B460544226813F8011B501C9D4202
:10C8D00020601170F7D1C8E70B68DFF87CC2591CE3
:10C8E0009CF8002021601A709CF80030002BBCD00E
:10C8F000894E8A4D8A488B490023226816F8017FA9
:10C9000002F1010EC4F800E01770226815F8017FEB
:10C9100002F1010EC4F800E01770226810F8017FE0
:10C9200002F1010EC4F800E01770226811F8017FCF
:10C9300002F1010EC4F800E017709CF800200133EA
:10C940009A42DADC91E70B68774A581C117820602C
:10C95000197023685278591C216001201A7085E7EC
:10C96000724D08462988FDF7DFFEA9882046FDF7AD
:10C97000DBFE20462989FDF7D7FE012076E76C4DC6
:10C9800005F1500628782FF085F92368027A591CA2
:10C9900021601A7023686A78591C21601A70236814
:10C9A000AA78591C21601A702368EA780435591C4A
:10C9B000AE4221601A70E5D157E75E4D0846E9891D
:10C9C000FDF7B2FE2046A989FDF7AEFE01204DE736
:10C9D000594B03F1700522681978501C20601170C2
:10C9E00022685978501C2060117022689978501C78
:10C9F000206011702268D978501C20601170226864
:10CA00001979501C2060117022685979501C2060DF
:10CA10001170226899790733501C9D422060117073
:10CA2000D9D122E70B6801229918216010461A70AB
:10CA30001CE708460021FDF75FFE012016E73F4D89
:10CA40003F4E05F1300795F902103E4B93F9062051
:10CA50008A4203F1080300F03E859E42F6D1083574
:10CA6000BD42F0D101E7384B03F15A0522685979EC
:10CA7000501C2060117022681978501C20601170C1
:10CA800022685978501C2060117022689978501CD7
:10CA9000206011702268D978501C206011702268C3
:10CAA00019790633501C9D4220601170DED1DCE6FE
:10CAB0000B68264A591C527D216001201A70D5E668
:10CAC000234D05F1800655F8041F2046FDF714FE9E
:10CAD000AE42F8D1C9E61F4D05F14006B5F8801009
:10CAE0002046FDF721FE236895F88220591C21601D
:10CAF0001A70236895F883200435591CB5422160CB
:10CB00001A70EBD1B1E600BF946F0020F2A70020AD
:10CB1000C4400020B45B0020CF4A0020DF4A002040
:10CB2000FF4A0020EF4A00205C460020643A0020C3
:10CB30006046002014400020E8800020886B002020
:10CB40006463002034630020C4510020646300202B
:10CB50004C5A0020505A0020CD4A0020B74D0B6897
:10CB60002A7A591C21601A70A98B2046FDF7DCFD3A
:10CB7000298B2046FDF7D8FD698B2046FDF7D4FDB3
:10CB80002368EA7C591C21601A70A98C2046FDF7A5
:10CB9000CBFDE98C2046FDF7C7FD2368AA7F591C11
:10CBA00021601A70236895F82020591C21601A70A2
:10CBB000698C2046FDF7B8FD2368EA7A591C21608C
:10CBC0001A70E9682046FDF797FD23682A7C591CF6
:10CBD00021601A70236895F82120591C21600120DA
:10CBE0001A7043E6964D974E9FED978ADFF8A48220
:10CBF000DFED968A05F120070EE0FCEEE77ACDED39
:10CC0000017ABDF8041020460435FDF78DFDBD42C4
:10CC100006F118063FF429AE717C0029F3D08C4B45
:10CC2000D5ED007A1B78012BE7D18A4B1B68DB041A
:10CC300040F10F85F5EE407AF1EE10FA40F03B85B9
:10CC400040F2DC51DFE70B68834D591C2A792160E3
:10CC50001A7023686A79591C21601A702988204645
:10CC6000FDF762FD2368AA79591C21601A70698852
:10CC70002046FDF759FD2368EA79591C21600120FF
:10CC80001A70F3E50B68754E01255A1C0A601D7079
:10CC90000B68B278591921601A7015F0B5F923683C
:10CCA0006F4A70495F1927601870B1F90010B2F926
:10CCB0000000FDF7C3FE23685A19226018703188FE
:10CCC0002046FDF731FD2846D0E50B6800255A1CAB
:10CCD0000A601D700B685A1C0A601D700B685A1C94
:10CCE0000A60204629461D70FDF706FD20462946AC
:10CCF000FDF702FD0120B9E5FEF7B2F823685A4DB1
:10CD0000002803F101010CBF0222032221601A70E6
:10CD100029882046FDF7F0FCA9682046FDF7ECFCC9
:10CD2000FEF776F801462046FDF7E6FC01209DE57A
:10CD30000B684E4A4E4D11784E4A581C20601970AF
:10CD400011682046FDF7D8FC23683C4A591C127A2A
:10CD500021601A7029882046FDF7E6FCA988204644
:10CD6000FDF7E2FC29892046FDF7DEFC0021204684
:10CD7000FDF7DAFC20460021FDF7D6FC012075E521
:10CD8000084608222D49FDF787FC01206EE50B6857
:10CD9000394A581C917820601970DAE5084610224B
:10CDA0003649FDF779FC012060E5354B9B8AB3F5E8
:10CDB000006F00F26384B3F5806F00F27984B3F5FD
:10CDC000007F34BF012702272E4D05F10C0655F8D0
:10CDD000041B91FBF7F1204689B2FDF7A5FCAE429A
:10CDE000F5D1294D294F05F10C06B5EC010AD7ED17
:10CDF000087A80EE270A31F09FFC81B22046FDF7C9
:10CE000093FCAE42F1D1224D05F10C0655F8041BFE
:10CE1000204689B2FDF788FCAE42F7D125E5002512
:10CE20008146DFF87480DFF874B0059504950695A7
:10CE3000079501214FF6FF7A38E000BF64630020B8
:10CE400064410020E05D00200000404200E0824498
:10CE5000C45E0020F4610020BC530020CCA9002057
:10CE6000D2440020D4440020DC0300205C46002093
:10CE7000643A0020D0710020FC5C00205441002066
:10CE80000088002038880020E861002098AA00204F
:10CE9000546F0020DB9B91414C0B04087C5B00200D
:10CEA00001350B2D00F0358318F9011F4F1C4AFA8C
:10CEB00005F3F5D0DE07F3D5BBF800302B41D807DA
:10CEC000EED506A8FDF776FFEAE70B68AC4AAD4958
:10CED000D078AD4A5D1C2560187023684979581CCC
:10CEE000206019702368D278591C216001201A70C3
:10CEF000BCE400212046FDF717FC00212046FDF789
:10CF000013FC00212046FDF70FFC23689F4D0026EF
:10CF10005A1C22601E7023682A68591C92F82C2023
:10CF200021601A7023682A68591C92F83620216003
:10CF30001A7023682A68591C92F8372021601A70E9
:10CF400023685A1C22601E7023685A1C22601E70BF
:10CF500023685A1C22601E702B682046598FFDF7EB
:10CF6000E3FB2B682046198FFDF7DEFB23682A6858
:10CF7000591C92F82E2021601A7023685A1C2260D6
:10CF80001E702B682046598EFDF7CEFB2B6820467D
:10CF9000998EFDF7C9FB012068E47D4E0B6872791C
:10CFA0007A4D591C21601A702B682046198CFDF7A8
:10CFB000BBFB2B682046D98BFDF7B6FB7189204659
:10CFC000FDF7B2FBB1892046FDF7AEFB2B6820468A
:10CFD000598CFDF7A9FB2B682046998CFDF7A4FB23
:10CFE000F1892046FDF7A0FB318A2046FDF79CFB26
:10CFF0002A68236892F82620591C216001201A70A3
:10D0000034E4634EF378002B00F02C830B68082285
:10D01000591C21601A7023680122991821601A7026
:10D0200023685C4D591C2A7921601A702368AA78FC
:10D03000591C21601A7029882046FDF775FBE98983
:10D040002046FDF771FB2368F279591C21601A70A4
:10D050002368EA78591C216001201A7006E427F041
:10D0600007FAFF28064600F00C8308A9002501F8FE
:10D07000125D0DF10D008DF80D5027F0D9F908A8BB
:10D0800000F8115D27F0C8F908A800F8105D27F036
:10D09000B7F908A820F8085D27F0A6F923685A1CFC
:10D0A00022601E7023689DF80D20591C21601A70A3
:10D0B00023689DF80E20591C21601A7023689DF882
:10D0C0000F20591C21601A7023689DF81020591CEC
:10D0D00021601A702046BDF81810FDF725FBFFF7F8
:10D0E000C4BB0B682C4F591C3A7821601A703B78EE
:10D0F000002B3FF4BAAB0025EEB2304625F07CFEA3
:10D1000023684278591C216030461A7025F074FE5D
:10D1100001892046FDF708FB3B780135AB42EBDC8B
:10D12000FFF7A3BB1D4D05F16006A9882046FDF75A
:10D13000FBFAE9882046FDF7F7FA29892046FDF732
:10D14000F3FA2368AA7A591C21601A702368EA7AD4
:10D15000591C21601A7055F80C1B2046FDF7CCFABB
:10D16000AE42E2D1FFF781BB0D4952232268501C29
:10D170002060137011F8013F002BF7D1FFF775BB4A
:10D1800014400020EC890020CC460020CC5B00201D
:10D19000D0610020A05E0020596C0020188700207C
:10D1A0001C0B0408AD4800232268056803EB43010B
:10D1B000561C6D5C26601570026825680A446E1C5A
:10D1C000527826602A70026825680A4401339278F2
:10D1D000691C0A2B21602A70E6D1FFF746BBA04DDF
:10D1E0000B682A68591C127821601A702B68226813
:10D1F0009978531C2360002311702A6821681A440F
:10D2000001335279481C032B20600A70F5D1236842
:10D210002A68591C127A21601A7023682A68591CDE
:10D22000D27821601A7023682A68591C127921600B
:10D230001A702B6820465989FDF776FA2A68236808
:10D24000527A591C21601A702A68FFF782BB854BFD
:10D2500008461968FDF750FA834B20461988FDF7F8
:10D2600063FA0120FFF702BB804B08461988FDF7DF
:10D270005BFA7F4B20461988FDF756FA7D4B2268F2
:10D280001B78511C03F00103216001201370FFF78C
:10D29000EDBA794B0A681B78784D511C03F00203F4
:10D2A0002160137023682A7D591C21601A70296837
:10D2B0002046FDF721FA69682046FDF71DFA298905
:10D2C0002046FDF731FAE9892046FDF72DFA204680
:10D2D000298AFDF729FA0120FFF7C8BA684D0846E8
:10D2E0002988FDF721FA69882046FDF71DFAB5F96E
:10D2F0000430644AD91782FB0323C1EBA301204603
:10D3000089B2FDF711FA0120FFF7B0BADFF89CE10E
:10D310000027FEB2714600232268501C2060167060
:10D320002268501C20601370226811F8010F01332D
:10D33000551C062B25601070EED10137062F0EF11B
:10D34000060EE6D1504900232268501C2060177059
:10D350002268501C20601370226811F8010F0133FD
:10D36000551C0B2B25601070EED12368474A581CC2
:10D3700007212060197023680021581C2060197053
:10D38000236892F8F020591C216001201A70FFF7E1
:10D390006DBA0B683E4A3F4910783F4A5D1C2560D4
:10D3A000187023688978581C206019702368927857
:10D3B000591C216001201A70FFF758BA0A68374BD0
:10D3C00037491878551C2560107022685878551C0C
:10D3D0002560107022689B78501C206013702046D6
:10D3E000C988FDF7A1F90120FFF740BA2C4D084686
:10D3F0002988FDF799F969882046FDF795F92046B7
:10D40000A988FDF791F90120FFF730BA0A68254B8A
:10D41000501C19782060117022685978501C2060C7
:10D42000117022689978501C206011702268DB7896
:10D43000511C216001201370FFF718BA1A4D0846DD
:10D44000298AFDF771F9698A2046FDF76DF92046B2
:10D45000A98AFDF769F90120FFF708BACC5B002023
:10D46000D85C00205488002048880020D6A90020DD
:10D47000B25B00209C490020788800207C88002036
:10D480005888002067666666335B0020505A00208B
:10D49000D061002014400020CC46002020590020FC
:10D4A000A0530020B44A0020A05E00200F5B0020A3
:10D4B000A04BA149B3F9003081FB0321DB17C3EB7B
:10D4C000A101204689B2FDF72FF90120FFF7CEB95F
:10D4D0000020FFF7CBB923685A1C226019702988F5
:10D4E0002046FDF721F92368EA78591C21601A705B
:10D4F00023682A79591C21601A702368AA79591C5B
:10D5000021601A7023686A79591C21601A70FFF72C
:10D51000A6BADFF84CA200254FF008080135C5F186
:10D52000200208FA02F2A5F120032AFA05F61643B2
:10D5300028FA03F31E43252D06F001024FF00003E5
:10D540000BD01343EAD0E8B221F090FA0028E5D0DE
:10D55000294606A8FDF72EFCE0E7784B1B78DA0792
:10D5600000F196800025764E2F4602E00135252DEC
:10D570000DD029463046FDF72DFC0028F6D029466F
:10D5800006A8FDF727FC00285ED10137EEE76D4BBA
:10D590006D4DB3F850102046FDF7C6F86B4B198857
:10D5A000204689B2FDF7C0F8694B19684B0103F0BA
:10D5B0002002C1F340031343C1F3800243EA420354
:10D5C000C1F3C00243EA8203C1F3401243EAC2033B
:10D5D00001F0100119432046FDF7A6F804A9042222
:10D5E0002046FDF759F8236829785A4A581C2060CC
:10D5F000197011886429A8BF64212046FDF794F8AA
:10D60000B9F1960F49D000212046FDF78DF8216829
:10D61000B7F1190348BFA7F11203A3F3C4034A1CCF
:10D62000226020461A460B7005A9FDF735F82368DD
:10D63000494A581C10212060197020461188FDF7B6
:10D640005BF80120FFF712B9394604A8FDF7B2FBD9
:10D650009BE7F4EEC87AF1EE10FA49DA4FF47A71EA
:10D66000FFF7D1BA0B68B1783C4A581C206019709A
:10D6700023681278591C21601A70D1E40827FFF73B
:10D68000A3BB23685A1C226001201E70FFF7EEB86E
:10D69000069B43F00103069364E723680322591CA9
:10D6A00021601A7023686A78591C21601A70AEE7ED
:10D6B0000427FFF789BBF4EEC87AF1EE10FA3FF5C4
:10D6C000BFAAF4EEE87AFDEEE77AF1EE10FA17EE73
:10D6D000901A20D86FF4F973303903FB01F140F24E
:10D6E000E73391FBF3F101F2DB5189B2FFF78BBA1B
:10D6F000FDEEE77A40F2E73217EE903A303B02FB5C
:10D7000003F388FB0312D917C1EB622101F2E9315F
:10D7100089B2FFF778BA40F2F313A1F5836103FBF6
:10D7200001F140F2E73391FBF3F101F2DD5189B2EF
:10D73000FFF769BACC46002067666666288A002033
:10D7400044A90020680A00206C6B0020E03A002009
:10D7500074880020E43A0020ECA9002030860020E4
:10D7600090E33FF408B501210220FCF7B1F9094B21
:10D770001B7803F00503052B08D000210120FCF7DE
:10D78000A7F900210846FCF7A3F9FEE718F014FFFB
:10D79000F3E700BFC0390020022828BF022010B4E0
:10D7A000084C094B207000EB8002C0EBC202074915
:10D7B0005DF8044B013003EB4203C0B20B601AF07A
:10D7C000AFBE00BF6C6B0020A2700020CC5B0020BD
:10D7D00008B513F06DFAFCF743FDBDE8084013F0FF
:10D7E0004FBA00BF38B5484B5A899989914224BF36
:10D7F00000225A81198ADA89914224BF0022DA81F3
:10D80000DA78CAB1072A41496AD091F85700404DE9
:10D81000012400210A282C709C70D9715DD00C283D
:10D8200007D0002A6CD0DFED3B7A072A0ED00A28F9
:10D8300062D0DFED397A09E0344A92F857000A28BD
:10D8400056D00C285BD1D979DFED347A344C9FED7A
:10D85000350AA278002918BFF0EE407A062A04D8CB
:10D86000314901EB820191ED0F0A217979B1013A39
:10D87000032A0BD8F7EE007A87EE800A30F05CFFBF
:10D880002388984228BF1846208038BD38BD9B7831
:10D890001F4A07EE103A1178B8EEC77A67EE277A7A
:10D8A00007EE101AB8EEC77A27EE277AB4EEC70A49
:10D8B000F1EE10FAEADD80EE277AFDEEC77A17EE78
:10D8C000903A102BA8BF1023012BB8BF0123DBB265
:10D8D0008B4238BF0B46137038BDDFED147AA4E7D6
:10D8E00091F857000A2803D00C28ACD0D9799AE7D0
:10D8F000D979DFED0E7AA9E7DFED0D7AA6E7D979C0
:10D90000DFED047AA2E700BFD061002098AA0020D2
:10D91000308600206F1203396F12833A0AD7A33979
:10D92000A05E00206F1203381C0B04085304E93872
:10D930000F506E3A38B50D4C0D4DAC4206D26168B1
:10D9400020461434FCF718FCAC42F8D3FDF750FA2B
:10D95000084A094B094C1460002209491A705A7090
:10D9600008480860BDE8384017F084B8880100080E
:10D970004C060008CC5B00206C6B0020A2700020DD
:10D98000D85C00206A6F002008B5FFF7D3FF13F0C2
:10D990008FF9FCF765FCBDE8084013F071B900BFD2
:10D9A000F0B50C2934D8DFE801F0893333335E3326
:10D9B0003333343333330700048C9689B2F802E0F2
:10D9C0001788734D24F480542404240C0484038C9D
:10D9D0008488818B23F4005321F4E6411B0409045D
:10D9E0001B0C46EA0E06090C43EA063341EA0721FE
:10D9F000A8429BB2A4B289B200F09E8005F5806572
:10DA0000A84200F099809268848081830264038434
:10DA1000F0BD048C9589B2F802C0B2F800E05C4F0A
:10DA200024F480742404240C0484038C8688818B61
:10DA300023F400731B0421F073011B0C45EA0C0452
:10DA4000090443EA0423090CB8429BB2B6B241EA86
:10DA50000E015CD04F4CA04259D0926886808183E1
:10DA6000C2630384F0BD048C9589B2F802C0B2F899
:10DA700000E0474E24F010042404240C0484038C9A
:10DA80008788018B23F0200321F4E6411B0409045D
:10DA90001B0C45EA0C04090C43EA041341EA0E216D
:10DAA000B0429BB2BFB289B25DD03A4CA0425AD0CC
:10DAB00092688780018382630384F0BD048C978918
:10DAC000B2F802E01688324D24F001042404240C3C
:10DAD0000484038C8488018B23F002031B0421F04F
:10DAE00073011B0C47EA0E0709043B43090CA842CB
:10DAF0009BB2A4B241EA060125D005F58065A84293
:10DB000021D092688480018342630384F0BDD5896B
:10DB1000148A578A23F4006343EA05254FF6FF333E
:10DB20002B40958826F440563C4343EA052346EAB9
:10DB300004169BB2B6B290E7158A24F4804444EAF6
:10DB40008514A4B25FE7D689158A578A23F00803A3
:10DB5000334324F4407496883D4323F004032C435C
:10DB60003343A4B2CDE7D489158A568A23F08003C3
:10DB700043EA04134FF6BF741C40938827F44067B0
:10DB8000354344EA031347EA85079BB2BFB28FE7E8
:10DB900000000140000401402DE9F04FA0220021C7
:10DBA00083B08A488A4CDFF84C928A4D8A4E8B4F5C
:10DBB000DFF8448232F0CDFE89488A49DFF83CE242
:10DBC000DFF83CC200221359834200F0D580B3F144
:10DBD000804F00F0E580AB4200F0E480B34200F0FB
:10DBE000E380BB4200F0E280734500F0E1806345D2
:10DBF00000F0E080434500F0DF80DFF808A25345E5
:10DC000000F0DC800AF5806A534500F0D9800AF5FF
:10DC1000806A534500F0D680AAF5983A534500F043
:10DC2000D3800AF5806A53457BD00AF5806A534554
:10DC300008BF0D2376D01832C02AC4D1644C6A4E76
:10DC40006A4F6B4D04F1C00802E01834A04565D05E
:10DC5000A379002BF9D023794FEA131909F1FF3981
:10DC6000B9F1020F03F00F03EFD836F8190040FAAC
:10DC700003F2D207E9D54FF0010A0AFA03F3013B98
:10DC8000184030F057FA17F80930184415EBC00265
:10DC9000DBD055F83000DFF870E1217A00F13F4326
:10DCA00003F57E039B0A1EF8033003F01F0E5B0989
:10DCB000032B0AFA0EFA61D0042B68D0022B52D043
:10DCC00093880093B3FA83F3C3F11F039BB2DA087E
:10DCD00000EB820203F00703D2F820E09B004FF034
:10DCE0000F0C0CFA03FC2EEA0C0EC2F820E0D2F85E
:10DCF00020E001FA03F343EA0E03136269460023AE
:10DD0000022218348DF804208DF805308DF8063085
:10DD10008DF807302AF0C8FEA04599D103B0BDE8C0
:10DD2000F08F0C2309EBC3034FF0010A93F85C302A
:10DD300003F01F0B5B09032B0AFA0BFA09D0042B23
:10DD40000CD0022B7FF477AF4B6C4AEA03034B6491
:10DD500071E70B6C4AEA03030B646CE70B6B4AEA4E
:10DD600003030B6367E7DFF87CE0DEF844304AEA40
:10DD70000303CEF84430A3E70023D3E7DFF864E0E1
:10DD8000DEF840304AEA0303CEF8403098E7DFF887
:10DD900054E0DEF830304AEA0303CEF830308FE743
:10DDA0000123BFE70223BDE70323BBE70423B9E751
:10DDB0000523B7E70623B5E70723B3E70823B1E751
:10DDC0000923AFE70A23ADE70B23ABE7BC640020D0
:10DDD000EC3204080004004000080040000C004041
:10DDE00000000140003802408842040884420408D0
:10DDF00080B200201C0B0408000401400010004009
:10DE000000140040004001407C42040801490248DF
:10DE1000FEF7D0BB346500200004014001490248F0
:10DE2000FEF7C8BB346500200004014001490248E8
:10DE3000FEF7C0BB0C650020000C00400149024801
:10DE4000FEF7B8BBE46400200004004002494FF034
:10DE50008040FEF7AFBB00BFBC640020F0B5046893
:10DE6000434DA30AAB4269D05BD9424DAB4251D07E
:10DE70003E35AB4266D14FF0980E03264779B0008D
:10DE80004FEA970C00295FD063460227A5899F407F
:10DE900083190CEB43032F4303F1040C364DBFB23F
:10DEA00045F8231045F82C20A781EFF3118150226B
:10DEB00082F31288821905EBC202136973B31362ED
:10DEC0000433821905EBC202576917B11F60536909
:10DED0000433821905EBC202976917B11F60936979
:10DEE0000433821905EBC202D76917B11F60D369E9
:10DEF00004330027CAB21F6082F31188304405EB57
:10DF0000C000036AA3B9A38923F001031B041B0CFF
:10DF1000A381F0BD4FF0700E0226AFE705EB0E03B4
:10DF2000CFE7B3F5801F0ED14FF0200E0026A5E7F6
:10DF3000A3899BB243F00103A381F0BD4FF0480ECB
:10DF400001269BE7F0BDF0BD0223BF0803FA07F7E7
:10DF5000A389094D9BB223EA070387190CEB470CF1
:10DF6000A3810CF1040345F82C1045F823209CE70D
:10DF70000100100003001000BC64002010B503680D
:10DF800083480139834282B089B200F0CB80A0F58A
:10DF90008060834200F0C68000F58040834200F03C
:10DFA000B88000F58060834200F0B38000F58060A7
:10DFB000834200F0AE80774C188824686408B4FB74
:10DFC000F2F4013CA4B282B2B3F1804F0AD072489D
:10DFD000834207D000F58060834203D000F5806063
:10DFE000834202D122F0700292B26C48834200F068
:10DFF000A28000F58060834200F0A78022F4407286
:10E0000000F56C4092B283421A80D9621C854FD0D1
:10E010005F4A93424CD001229A821A8892B242F00F
:10E0200001021A80B3F1804F00F099805A4A93425E
:10E0300000F0978002F58062934200F0948002F530
:10E040008062934200F0918002F58062934200F07A
:10E050008E8002F58062934200F08B8002F5704260
:10E06000934200F0888002F57052934200F0858060
:10E0700002F58062934200F0828002F58062934252
:10E080007FD0A2F5983293427DD002F58062934210
:10E090007BD002F58062934208BF0D2215D002A802
:10E0A0004FF0012340F8043D2AF04CFF02B010BDB0
:10E0B0000122002119869A821A88394892B242F0C8
:10E0C000010283421A80ADD10A46364B03EBC203EC
:10E0D00001A893F85D408DF80440012300228DF8DB
:10E0E00005308DF807308DF806202AF02BFF1B2C09
:10E0F00008D02E2CDAD12C4B019301A82AF022FF54
:10E1000002B010BD294B019301A82AF01BFF02B0F9
:10E1100010BD204C18882468B4FBF2F4013CA4B272
:10E1200082B251E71B4C18882468B4FBF2F4013C1E
:10E13000A4B282B256E701201A80D9621C85988267
:10E140001A8892B202431A8070E701201A80D962BD
:10E150001C8598821A8892B202431A8062E70122D3
:10E16000B3E70222B1E70322AFE70422ADE70522BD
:10E17000ABE70622A9E70722A7E70822A5E70922BD
:10E18000A3E70A22A1E70B229FE70C229DE700BF2D
:10E1900000040140DC5D002000040040001000404D
:10E1A000000001401C0B04082C01000119010001B2
:10E1B0002C4B98423DD0B0F1804F3CD0A3F57C432E
:10E1C00098423AD003F58063984238D003F58063D3
:10E1D000984236D003F58063984234D003F58063CB
:10E1E000984232D003F57043984230D003F5705313
:10E1F00098422ED003F5806398422CD003F58063BB
:10E2000098422AD0A3F59833984228D003F580632A
:10E21000984207D003F58063984208BF0D2202D0D0
:10E22000002070470C22104B03EBC20393F85C00F4
:10E2300070470022F7E70122F5E70222F3E7032205
:10E24000F1E70422EFE70522EDE70622EBE70722DC
:10E25000E9E70822E7E70922E5E70A22E3E70B22DC
:10E26000E1E700BF000001401C0B04082DE98048D5
:10E27000013085B0C3B203938A4D8B4F8B4C8C4ECB
:10E280000A230293DFF82C9222F07EFD4FF4FA7AF3
:10E290004FF0100C4FF47A70D9F80430C3F3080330
:10E2A000002B40F0C180EFF31183002B40F0BC80C5
:10E2B0002968A26800BF2B689942F9D1D7F800E01D
:10E2C00000FB0EF39B1AB3FBFEF300FB01314FF092
:10E2D000010E0191D9F80430C3F30803002B40F07C
:10E2E0008780EFF31183002B40F082802B68A168B8
:10E2F00000BF2A689342F9D1D7F800B000FB0BF2B7
:10E30000521AB2FBFBF200FB0323019A9B1AB3F5EE
:10E310007A7FDFD3BAF1010ABED1039B002B40F014
:10E32000BD804FF47A7ADFF88C9150464FF0100C94
:10E33000D9F80430C3F30803002B40F09280EFF3C8
:10E340001183002B40F08D802968A26800BF2B68E4
:10E350009942F9D1D7F800E000FB0EF39B1AB3FB0A
:10E36000FEF300FB01314FF0010E0191D9F80430AA
:10E37000C3F3080303BBEFF31183EBB92B68A16868
:10E3800000BF2A689342F9D1D7F800B000FB0BF226
:10E39000521AB2FBFBF200FB0323019A9B1AB3F55E
:10E3A0007A7FE3D3BAF1010AC2D1029B013B029307
:10E3B0007FF468AFFDF78AF9EFF311888CF31288C8
:10E3C000A1682368DB0344BFC6F800E0A1682B689E
:10E3D00032685FFA88F888F31188D7F800801A4409
:10E3E00000FB08F35B1AB3FBF8F300FB0233D4E73E
:10E3F000EFF311888CF31288A1682368DB0344BF14
:10E40000C6F800E0A1682B6832685FFA88F888F3E4
:10E410001188D7F800801A4400FB08F35B1AB3FB9D
:10E42000F8F300FB023370E7EFF311828CF31288EC
:10E43000D4F808E02368D90303D501233360D4F866
:10E4400008E02B683168D2B282F311883A68194427
:10E4500000FB02F3A3EB0E03B3FBF2F300FB01316D
:10E4600035E7EFF311828CF31288D4F808E02368C3
:10E47000D90303D501233360D4F808E02B68316851
:10E48000D2B282F311883A68194400FB02F3A3EB7D
:10E490000E03B3FBF2F300FB013164E718462EF0E4
:10E4A0001DFC3EE760AA002064AA002010E000E006
:10E4B0005CAA002000ED00E02DE9F047AC4FAD4E26
:10E4C00012F0F6FBBE421ED2DFF83483DFF834933D
:10E4D0004446258862197DB14A450DD2052D0BD9D8
:10E4E00033886188C3F30B03994200F0EE80144631
:10E4F00025886219002DEFD1716830461436FBF77C
:10E500003BFEBE42E4D39C4A1378A3F117010229D3
:10E510000FD99A4911F83300002840F01B81D80028
:10E520000144497829B1964911F833300BB91823C1
:10E530001370944C6378022B84BF0023637023789C
:10E54000022B84BF002323708F4B9A78042A00F09B
:10E55000F88032B91A88B2F5F07F84BF4FF4F072B8
:10E560001A808A4D8A4A2B681A40002A00F0FB80E4
:10E57000D80700F1E180590400F1D9801A0700F1B1
:10E58000D1809B0400F1C780824D2B685A8C998CF6
:10E59000914224BF00225A84FFF724F921F0B0FFF2
:10E5A000002800F0B4804FF40070FBF71BFE4FF41E
:10E5B0000010FBF717FE4FF00070FBF713FE4FF053
:10E5C0008060FBF70FFE6378022B06D8724A73490E
:10E5D00003EB430302EB83030B602378022B07D882
:10E5E00003EB83016E4AC3EBC10302EB43032B60D1
:10E5F00020F0B4FA002130226A4832F0AAF92868E3
:10E6000028F0C0FC684B2D6803F1500102E0043390
:10E6100099427AD01A78002AF9D19C78D878844225
:10E62000F5D26249624B0A7028461D6025F074FEDF
:10E63000604B614A1E7961496148624B1160C8258F
:10E64000642212FB0652604C406B31F8061C5A6083
:10E65000002221809A60DA601A615A619A61DA6157
:10E6600083F8202083F8212008B112F05FF9574B7E
:10E670009FED575A1B88574A9FED576A5579574C5B
:10E6800057495848086006EE903AF8EEE66A138853
:10E69000C5EE265A07EE103A53881279C4ED005A97
:10E6A00007EE903AB8EEC77A4F4BF8EEE77A1D7254
:10E6B0005A7227EE067A67EE867ABDE8F04783ED58
:10E6C000017AC3ED007A12F0DBBA63799B077FF41D
:10E6D0000EAF716894F804A03046FBF74DFD338807
:10E6E000BAEB133F04D01436BE42FFF4F1AE0AE792
:10E6F00073887068AA1FC3F30B039A4204F10601E2
:10E70000A8BF1A462FF010FEEDE7012289E737482F
:10E7100018F0BAFB47E73648FBF764FD4020FBF7EB
:10E7200061FD31E73348FBF75DFD2B6829E732488F
:10E73000FBF758FD2B6821E73048FBF753FD2B68AA
:10E7400019E79A8AB2F57A7FBFF40BAF4FF47A7269
:10E750009A8206E7D8000C186468002C7FF4E0AEBB
:10E7600017241470DCE643F008032B6000E700BFB9
:10E770004C060008880100085C460020643A040842
:10E78000803704086C6B0020A05E0020D071002050
:10E7900009600002CC5B00206A6F0020D85C00207A
:10E7A000A27000202C290020604600201A020020C0
:10E7B00060290020BC5300201CA900201A40002022
:10E7C00000880020845B0020A63F002054590020D0
:10E7D000C0C9FB48A425002017B7D13858590020DC
:10E7E000905100203661023D6C510020886B002062
:10E7F00009400002016000020920000208600002D6
:10E80000024000080080000808B512F051FAFBF73A
:10E8100027FD12F035FAFFF74FFE0120BDE8084052
:10E8200019F07EBE2DE9F04F013085B0C3B20393DD
:10E830000B4602918B4C8C4E002B00F099808B4D37
:10E840008B4FDFF8309222F09FFA4FF4FA7A4FF0B4
:10E85000100C4FF47A70D9F80430C3F30803002B7E
:10E8600040F0DE80EFF31183002B40F0D98029685F
:10E87000A26800BF2B689942F9D1D7F800E000FBED
:10E880000EF39B1AB3FBFEF300FB01314FF0010EB8
:10E890000191D9F80430C3F30803002B40F08780BE
:10E8A000EFF31183002B40F082802B68A16800BF3A
:10E8B0002A689342F9D1D7F800B000FB0BF2521A44
:10E8C000B2FBFBF200FB0323019A9B1AB3F57A7F9C
:10E8D000DFD3BAF1010ABED1039B002B40F0BD800B
:10E8E0004FF47A7ADFF88C9150464FF0100CD9F83B
:10E8F0000430C3F30803002B75D1EFF31183002B11
:10E9000071D12968A26800BF2B689942F9D1D7F864
:10E9100000E000FB0EF39B1AB3FBFEF300FB01319A
:10E920004FF0010E0191D9F80430C3F3080313BB73
:10E93000EFF31183FBB92B68A16800BF2A689342EB
:10E94000F9D1D7F800B000FB0BF2521AB2FBFBF280
:10E9500000FB0323019A9B1AB3F57A7FE3D3BAF144
:10E96000010AC4D1029B013B0293002B7FF467AFE5
:10E9700005B0BDE8F08FEFF311888CF31288A16821
:10E980002368DB0344BFC6F800E0A1682B68326847
:10E990005FFA88F888F31188D7F800801A4400FBE2
:10E9A00008F35B1AB3FBF8F300FB0233D2E7EFF393
:10E9B00011888CF31288A1682368DB0344BFC6F872
:10E9C00000E0A1682B6832685FFA88F888F3118844
:10E9D000D7F800801A4400FB08F35B1AB3FBF8F386
:10E9E00000FB023370E7EFF311828CF31288D4F846
:10E9F00008E02368D90303D501233360D4F808E085
:10EA00002B683168D2B282F311883A68194400FB4E
:10EA100002F3A3EB0E03B3FBF2F300FB01317FE73C
:10EA2000EFF311828CF31288D4F808E02368D9033D
:10EA300003D501233360D4F808E02B683168D2B2E3
:10EA400082F311883A68194400FB02F3A3EB0E032A
:10EA5000B3FBF2F300FB013118E718462EF03EF944
:10EA60003EE700BF10E000E05CAA002060AA0020A2
:10EA700064AA002000ED00E0204B5B68C3F30803AC
:10EA800030B4BBB9EFF31183A3B91D4B1D4C18680B
:10EA9000A16800BF1A689042F9D11B4B1C684FF463
:10EAA0007A7202FB04F3591AB1FBF4F130BC02FB99
:10EAB00000107047EFF31182102383F3128811497D
:10EAC0008C680B6813F4803F104B02D00120186053
:10EAD0008C680B49D2B20D68186882F311880A4B12
:10EAE00019684FF47A72284402FB01F31B1B30BCF7
:10EAF000B3FBF1F302FB0030704700BF00ED00E014
:10EB000060AA002010E000E064AA00205CAA0020B7
:10EB10002DE9F84F8046FFF7AFFF254E2549DFF876
:10EB2000A0E0254A254D844610274FF47A74012031
:10EB3000DEF80430C3F30803D3B9EFF31183BBB994
:10EB40000B68D2F808A000BFD1F800904B45F7D170
:10EB5000D6F800B004FB0BF9A9EB0A09B9FBFBF9E5
:10EB600004FB0393A3EB0C034345E1D3BDE8F88F0B
:10EB7000EFF3118A87F31288D2F808B01368DB0329
:10EB800044BF2860D2F808B00B68D5F800905FFA4F
:10EB90008AFA8AF31188D6F800A0994404FB0AF394
:10EBA000A3EB0B03B3FBFAF304FB0933DAE700BF73
:10EBB00064AA002060AA002010E000E05CAA002007
:10EBC00000ED00E02DE9F04FDFF830C1474A484939
:10EBD000484E494D8046102718F1FF38C0F0848018
:10EBE000DCF80430C3F30803002B5CD1EFF311838E
:10EBF000002B58D10B68946800BF08688342F9D194
:10EC0000D6F800904FF47A7000FB09FEAEEB040ECC
:10EC1000BEFBF9FE00FB03EEDCF80430C3F308038F
:10EC20004FF47A740120FBB9EFF31183E3B90B6859
:10EC3000D2F808A000BFD1F800904B45F7D1D6F824
:10EC400000B004FB0BF9A9EB0A09B9FBFBF904FBC3
:10EC50000393A3EB0E03B3F57A7FBDD2DCF8043047
:10EC6000C3F30803002BDFD0EFF3118A87F3128878
:10EC7000D2F808B01368DB0344BF2860D2F808B0AC
:10EC80000B68D5F800905FFA8AFA8AF31188D6F8F3
:10EC900000A0994404FB0AF3A3EB0B03B3FBFAF3C4
:10ECA00004FB0933D5E7EFF3118487F31288D2F818
:10ECB00008901368D80303D501232B60D2F808907D
:10ECC0000B682868E4B284F31188D6F800A04FF4EA
:10ECD0007A7400EB030E04FB0AF3A3EB0903B3FB06
:10ECE000FAF304FB0E3E97E7BDE8F08F10E000E07A
:10ECF00060AA002064AA00205CAA002000ED00E0C9
:10ED000030B4EFF31183102282F312880649074CC6
:10ED10000A680748013200250A602560DBB20268F4
:10ED200083F3118830BC704760AA00205CAA0020E1
:10ED300010E000E00F4B1B88014643B90E4B0F4A11
:10ED40001B7810680BB981F00101FAF7B9BE0C4BC2
:10ED50005A691AB118B91A68106058747047094A8C
:10ED600018681188084A92FBF1F201210260597477
:10ED7000704700BF10B4002012B4002014B400206B
:10ED800018B4002030B4002020A1070038B5254B6E
:10ED90005C69236B73B1636D626BCAB1998A1A881F
:10EDA000C90592B201D5D20700D438BD4FF6F7722B
:10EDB0001A8038BD636D99891A88890692B2EBD59D
:10EDC0009206E9D5E26ACAB1988880B29047E2E734
:10EDD00099891A880D0692B2E0D51006DED5A26A8E
:10EDE000616A8A4219D0A1692569885C98800132DC
:10EDF000B2FBF5F105FB1122A262CFE79B88E26925
:10EE00006169DBB28B54E269E068636D0132B2FB89
:10EE1000F0F100FB1122E261BEE7DA6822F0800225
:10EE2000DA60BBE7C439002038B5254B9C68236BFA
:10EE300073B1636D626BCAB1998A1A88C90592B2BF
:10EE400001D5D20700D438BD4FF6F7721A8038BD0D
:10EE5000636D99891A88890692B2EBD59206E9D535
:10EE6000E26ACAB1988880B29047E2E799891A8825
:10EE70000D0692B2E0D51006DED5A26A616A8A421A
:10EE800019D0A1692569885C98800132B2FBF5F13F
:10EE900005FB1122A262CFE79B88E2696169DBB2C0
:10EEA0008B54E269E068636D0132B2FBF0F100FB64
:10EEB0001122E261BEE7DA6822F08002DA60BBE785
:10EEC000C43900202DE9F04F9DB0B0F908500D81F4
:10EED000EDB2442D00AF0C46904600F0CC820646C1
:10EEE00043D9812D00F0048200F29980542D00F066
:10EEF000CE8040F2E9816E2D00F08B82802D40F0B3
:10EF00001981BF4B93F800A00AF1020A1AF0FF0A18
:10EF100000F09980BB4BDFF82483BB4EDFF820B3B1
:10EF20009A4403F101090A2516E0322D00F0D4823B
:10EF3000A5F13C00C0B2132840F2D482002322681D
:10EF4000511C216015702268D14502F10101216038
:10EF5000137078D019F8015B0A2DE6D1BBF80030A8
:10EF6000FF2BA8BFFF23DBB2E9E7052D00F071827C
:10EF700020D8022D00F0838040F29381032D00F011
:10EF80003E82042D40F0D6802A46A0492046FBF759
:10EF900083FB00212046FBF7C7FB22680221531C9C
:10EFA0000125236028462B46743711706381BD46C6
:10EFB000BDE8F08F242D60D040F20481282D00F0B0
:10EFC000E081382D40F0B6800A68914B0125511C34
:10EFD0002160157022680521501920601170226887
:10EFE0000A215019206011702268002150192060F8
:10EFF00011702268197850192060117022685978B0
:10F0000050192060117022689978531923602B469B
:10F010001170284674376381BD46BDE8F08FA02D7E
:10F0200019D040F21381B82D00F0E781FE2D40F099
:10F030008180784D05F1080635F8021B2046FBF764
:10F0400073FBB542F8D101252B46284674376381FE
:10F05000BD46BDE8F08F704B08461968FBF74CFBC6
:10F060006E4B20461968FBF747FB6D4B196820462D
:10F070000125FBF741FB2B46E7E76A4BF6E7042245
:10F08000694920460125FBF707FB2B46C1E70B68C2
:10F09000664ADFF8B081581C11212060197023687E
:10F0A0001278591C21601A70236898F85B20591C4B
:10F0B00021601A70236898F85A20591C21601A7030
:10F0C000B8F856102046FBF72FFB00212046FBF72F
:10F0D0002BFBB8F858102046FBF726FBA8F10205D9
:10F0E00008F1480635F8021F2046FBF71DFBB54224
:10F0F000F8D122684E4B0C21501C20605D18117015
:10F10000226813F8011F501C9D4220601170F7D136
:10F1100023680222591C21601A70B8F85C1020463E
:10F12000FBF702FB0125B8F85E102046FBF7FCFA5E
:10F130002B466EE721462846FDF794FA0346002841
:10F1400081D1742D00F0C680772D0DD132687168A1
:10F1500091421EBF531C33601178364A08BF1946CE
:10F1600020462CF043FD6EE7F52D01F0E383762D6C
:10F1700000F08981472D00F074823268392D1146E4
:10F1800000F05B8300F20882212D01F0B383292D6A
:10F1900040F07083531C336013780A2B01F086848F
:10F1A000502B41F02E833046FBF764FADFF898804D
:10F1B000A8F800003046FBF75DFA0125A8F8020028
:10F1C0002B4626E7202DB5D10B681B4D591C6A78BC
:10F1D00021601A7023682A78591C21601A702368EC
:10F1E000AA78591C21601A7029892046FBF79CFADD
:10F1F00023686A79591C21601A702268A979CEE6C1
:10F20000596C0020E40B0408942B0020726B002042
:10F210008D7000207C6C0020107AFF1F147AFF1F75
:10F22000187AFF1FD0710020B84204087C6B0020C0
:10F23000ADA9002055B103086088002067666666A6
:10F24000BC2B002064A900207C2B0020822D7FF4A1
:10F2500071AF0B68BB4ABC4D1178BC4A581C20608A
:10F26000197011892046FBF75FFAB94B22681B8899
:10F27000FF2B02F10101A8BFFF2321601370A968D1
:10F2800081F3100189B22046FBF74EFA296801F399
:10F290000F0189B22046FBF747FAAE4B2268197876
:10F2A0007DE6012D7FF446AF0B680022591C2160DA
:10F2B0001A7023685A1C22601D7022682421531C76
:10F2C00023602B461170A4E6522D7FF433AF2268E1
:10F2D000002164E63268716891421EBF531C33609E
:10F2E00011789D4A08BF194620462CF07FFCAAE6FB
:10F2F0009A4B1E78033616F0FF063FF4A4AE984BE7
:10F30000DFF88C821E4403F1010A4FF00A0920E065
:10F31000B9F1500F00F0DE80B9F1320F00F0F78044
:10F32000A9F13C00C0B2132840F2F4800025294620
:10F3300023685A1C2260204683F80090FBF7F4F9FA
:10F3400029462046FBF7F0F9B2453FF47CAE1AF8A7
:10F35000019BB9F10A0FDBD1824B9D68196805EB5F
:10F3600085054FF6FF736D009D42A8BF1D4699426B
:10F37000A8BF194625EAE57521EAE171ADB289B267
:10F38000D6E70B68DFF80C92774E591C02222160F9
:10F390001A7023684FF006085A1C226083F8008018
:10F3A00023680A22591C21601A70236801255A1902
:10F3B00022601D70B9F800102046FBF7B5F9B9F8C6
:10F3C00002102046FBF7B0F923685A19226083F82F
:10F3D000008023685022591921601A702368002286
:10F3E000591921601A7031882046FBF79DF9718800
:10F3F0002046FBF799F92B460BE65C4B36E60B688B
:10F400005A1C0A601D700B680222591C21601A7078
:10F410005DE74F4B0A681B884B4DFF2BA8BFFF23AE
:10F42000511C21601370A96881F3100189B2204634
:10F43000FBF77AF94E4B20461988FBF775F92968D6
:10F4400001F30F0189B220460125FBF76DF92B4628
:10F45000DFE50B2247492046FBF71EF90822464903
:10F460002046FBF719F90125072244492046FBF7FE
:10F4700013F92B46CDE5002A3FF4E5AD404B136070
:10F4800001252B46C5E53268511C31601278002AEF
:10F4900001F01383102A07BF3A4B93E822001D4660
:10F4A00029462368581C20601A702046FBF724F96F
:10F4B00029462046FBF720F9334B20461968FBF715
:10F4C0001BF920460021FBF72FF900212046FBF70E
:10F4D0002BF9FCE62D4B40E73388FF2BA8BFFF2319
:10F4E000DBB22CE523F088FC00283FF427AD03783D
:10F4F0000A2B25D8B0F9023088FB0312DB17C3EBC7
:10F50000A2039BB2FF2BA8BFFF23DBB217E598E84D
:10F51000220024E723F070FC00283FF407AF0378B3
:10F520000A2B3FF603AFB0F90430B0F9061003EB35
:10F53000830383F3500521EAE171ADB289B2F7E6A6
:10F540000023E2E75A6D0020F08700206088002049
:10F55000446D0020E0A900208DBA0308596C0020FA
:10F56000F40B0408482B00207C2B0020B85100200D
:10F57000D2A90020C0420408CC420408D8420408A2
:10F5800095C500086429002048590020802B0020E0
:10F590008C2B0020BC590020552D00F02781572DC1
:10F5A00040F06881531C336012F8378B07F12F014C
:10F5B0000133336013F8010C01F8010F9A42F7D1BF
:10F5C000DFF8A4A29AF80050002DFDD1DFF89CB21C
:10F5D0000126DBF800008AF80060FAF751FA9F4B29
:10F5E00028461E702DF0EAFA28462DF0E7FA092089
:10F5F0002DF0E4FA40462DF0E1FA07F130084546D7
:10F6000007F16609A5EB0806F6B20A202DF0D6FA36
:10F6100030462DF0D3FA15F8016B0B202DF0CEFA01
:10F6200030462DF0CBFA0020F9F7FAFD4D45E9D12F
:10F6300008202DF0C3FAA0202DF0C0FAA0202DF054
:10F64000BDFA00202DF0BAFA10F02000F6D10646DF
:10F650000125DBF80000FAF719FA8AF800602B465A
:10F66000D7E4726835687B623046551BFAF7EAFFCB
:10F67000052D38627B6A01F201828026B34601259E
:10F6800094E80600521A103AB242B8BF1FFA82FB41
:10F69000734A396A92683A61521A9345396A7B62B1
:10F6A0002046FA6088BF1FFA82FBFBF725F87B6AC9
:10F6B000002B01F0C281002D41F099812368C7F829
:10F6C00000D05D71C0B00533C7F804D0FB61BBF159
:10F6D000000F01F0C1823B6A3A69934281F068836E
:10F6E0003E6A7D62AA46A846BC608025FB68A3EB03
:10F6F00008085B4BB8F5807F9B6828BF4FF4807883
:10F7000006EB08029A4288BFA3EB0608FBF7B6FC9B
:10F710007C68424621463046FBF730FDF969B86106
:10F7200004EB000C0B787B6164452ED2DFF840912E
:10F730000CF1FF3C04F1FF3E1EF8013F09EB830290
:10F7400019F823405688ECB100234FF4004204F12D
:10F75000FF3816424FEA520202D008782843087058
:10F760006D0806D10AF1010A4D701FFA8AFA0131BB
:10F770008025D34503D8F44532D8984530DC013391
:10F780009C42E6D1F445D7D1F9617B6ABA6913444A
:10F790009BB2D3457B6206D97B6A3A6A9846D618F3
:10F7A0003B699E42A2D3BC68802D1CBF0AF10103B5
:10F7B0001FFA83FA0AF1020189B22046FAF7B4FF70
:10F7C0002368796A01255A19226020461D70FAF7CC
:10F7D000ABFF2368534423602B46D7F800D018E4CE
:10F7E000FB69BC681A463B7D1370DDE7531C336030
:10F7F00092F80080B8F1FF0F01F0C681B8F1FE0F5A
:10F8000001F0A4813046FAF735FF96E80C009B1A08
:10F81000002B07DD531C336013781BB9B8F10B0FB5
:10F8200041F2A781B8F1240F00F29D820D4B012512
:10F8300023F818002B46FFF7ECBB531C33601378FA
:10F840000A2B01F03F813046FAF720FF3046FAF7E5
:10F850001DFF3046FAF71AFFFFF7F5BBAE4C00204C
:10F86000DC03002064A90020A54C0020606B002070
:10F87000040C040870680B3D831AEF2D00F27382AC
:10F880000FF2040E5EF825F00705010867FD000879
:10F8900067FD000867FD000867FD000867FD0008B8
:10F8A00067FD000867FD000867FD000867FD0008A8
:10F8B00067FD000867FD000867FD000867FD000898
:10F8C00067FD000867FD000867FD000867FD000888
:10F8D00067FD000867FD000867FD000867FD000878
:10F8E00067FD000867FD00087508010867FD00084E
:10F8F0005308010867FD00085B06010867FD000862
:10F9000067FD000867FD00083306010867FD000871
:10F91000D905010867FD00087505010867FD0008A5
:10F920004F05010867FD00083D05010867FD000857
:10F930005507010867FD0008BB06010867FD0008C0
:10F9400067FD000867FD000867FD000847F0000834
:10F9500067FD00089F06010867FD000867FD0008B5
:10F960008506010867FD0008B907010867FD000862
:10F9700067FD000867FD000867FD0008AD07010886
:10F9800067FD000867FD000867FD0008130801080F
:10F9900067FD0008B904010867FD000867FD00085D
:10F9A0007704010867FD000867FD000867FD00088F
:10F9B00067FD000867FD000867FD000867FD000897
:10F9C0002F03010867FD00080304010867FD000814
:10F9D000BD02010867FD0008ED01010867FD000890
:10F9E000C5010108A701010867FD000867FD0008BF
:10F9F00067FD000867FD000867FD000867FD000857
:10FA000067FD000867FD000867FD000867FD000846
:10FA100067FD000867FD000867FD000867FD000836
:10FA200067FD000867FD000867FD000867FD000826
:10FA300067FD000867FD000867FD000867FD000816
:10FA400067FD000867FD000867FD000867FD000806
:10FA500067FD000867FD000867FD000867FD0008F6
:10FA600067FD000867FD000867FD000867FD0008E6
:10FA700067FD000867FD000867FD000867FD0008D6
:10FA800067FD000867FD000867FD000867FD0008C6
:10FA900067FD000867FD000867FD000867FD0008B6
:10FAA00067FD000867FD000867FD000867FD0008A6
:10FAB00067FD000867FD000867FD000867FD000896
:10FAC00067FD000867FD000867FD000867FD000886
:10FAD00067FD000867FD000867FD000867FD000876
:10FAE00067FD000867FD000867FD000867FD000866
:10FAF00067FD000867FD000867FD000867FD000856
:10FB000067FD000867FD000867FD000867FD000845
:10FB100067FD000867FD000867FD000867FD000835
:10FB200067FD000867FD000867FD000867FD000825
:10FB300067FD000867FD00087D01010867FD0008FA
:10FB40006101010867FD000867FD000867FD000806
:10FB500067FD000867FD000867FD000867FD0008F5
:10FB600067FD000867FD000867FD000867FD0008E5
:10FB700067FD000867FD000867FD00080301010834
:10FB8000B10001087900010867FD0008D7FF0008EF
:10FB9000BDFF000851FF000867FD000837FF00089F
:10FBA000CBFE0008A3FE000891FE000835FE000809
:10FBB00067FD000805FE000867FD000867FD0008F6
:10FBC000DBFD0008ADFD000899FD000871FD00088F
:10FBD00049FD00081FFD0008F3FC0008DBFC0008DD
:10FBE00067FD000867FD000867FD000867FD000865
:10FBF00067FD000867FD000867FD000867FD000855
:10FC000067FD000867FD000867FD000867FD000844
:10FC100067FD000867FD0008BBFC000867FD0008E1
:10FC200067FD000863FC000867FD000867FD000829
:10FC300067FD000867FD000867FD000867FD000814
:10FC400067FD000849FC0008C84B1B78DB0700F182
:10FC50008A800125FDF7BCFDFEF72EFC2B46FFF741
:10FC6000D8B9531C336013780F2B7CD8911C3160AA
:10FC7000C3EBC303BE495078C854D01C30600B445A
:10FC800091785970111D3160D1789970511D316092
:10FC90001179D970911D316051791971D11D31607F
:10FCA0009179597102F108013160D2799A71012577
:10FCB00026F0F0FE2B46FFF7ACB93046FAF7DAFC37
:10FCC000DFF8BC82A8F80E003046FAF7D3FC012515
:10FCD000A8F80C002B46FFF79CB93046FAF7CAFC8F
:10FCE000A44A00EB80004300012513802B46FFF758
:10FCF00090B91146531C33609F4B11F8020B1870DA
:10FD0000316051785970D11C316091789970111D12
:10FD10003160D278DA7001252B46FFF77AB9304688
:10FD2000FAF7A8FCDFF88482A8F810003046FAF74A
:10FD3000A1FCA8F812003046FAF79CFC0125A8F8AF
:10FD400014002B46FFF765B91346511C316013F8B8
:10FD5000020B3360D31C5178336092781DF0CAFDDA
:10FD600000287FF470A94FF0FF352B46FFF751B9FB
:10FD70001346511C3160814913F8020B087033603F
:10FD80007F4953788B70D31C33607A4B92789A708A
:10FD900001252B46FFF73DB97A4B7B4918684E2267
:10FDA00001252EF0C1FA2B46FFF733B91146531C3B
:10FDB0003360764B11F8020B18703160517859702E
:10FDC000D11C316092789A703046FAF753FC704B30
:10FDD0000125D8802B46FFF71CB93046FAF74AFCBC
:10FDE000DFF8AC81A8F800003046FAF743FCA8F829
:10FDF00002003046FAF73EFC0125A8F804002B4625
:10FE0000FFF707B9DFF8A89199F80030002B3FF40D
:10FE10001AA9DFF8A08100253046FAF72BFC16F06E
:10FE2000B7FA99F80030A8EC010A01359D42F3DBDE
:10FE3000FFF709B90D2B96D1531C33601578072DA8
:10FE400091D8DFF8749130464FF00C08FAF712FCA5
:10FE500008FB05F809EB0805A8803046FAF70AFC0C
:10FE6000E8803046FAF706FC336828811A46591CA8
:10FE7000316012F8021BA97232605B78EB72304677
:10FE8000FAF7E0FB012549F808002B46FFF7C1B857
:10FE90003046FAF7EFFB3F4B012518802B46FFF762
:10FEA000B8B8531C33601078060600F185872F4BD5
:10FEB0001B78DD073FF5C7A8032828BF00200125D0
:10FEC000FDF76AFC2B46FFF7A4B8531C336030469D
:10FED00092F800A0FAF7B6FB81463046FAF7B2FB7B
:10FEE00005463046FAF7AEFB80463046FAF7C2FBCD
:10FEF0003046FAF7BFFB3046FAF7C8FBBAF1000FFD
:10FF000000F03A87BAF1100F7FF49DA8224BC3F896
:10FF100000905D60B8F1000F02D0204BC3F8008064
:10FF20001F49204B0222081F01251A7024F092F964
:10FF30002B46FFF76EB80D4B1B78D8073FF583A80B
:10FF40000125FDF721FDFEF7B7FA2B46FFF761B853
:10FF5000064B1B78DA073FF576A8134A137801257C
:10FF600043F0040313702B46FFF753B8288A002090
:10FF7000E8800020CC460020B44A0020D061002058
:10FF800014400020CC5B0020F427040820590020F6
:10FF9000A0530020B04A00206429002048590020C6
:10FFA000682900209E49002078880020A05E00205B
:10FFB000596C0020F452002018870020B14B1B78A8
:10FFC000D9073FF540A8B04B4FF4C87201251A80FD
:10FFD0002B46FFF71EB8092B7FF7C5AEDFF8D4829A
:10FFE0001346511CD8F80050316013F8021B2970D9
:10FFF00033605378AB70D31C33609378642B02F179
:020000040801F1
:100000000401A8BF64236B713160D378642B02F1C3
:100010000501A8BF6423AB7131601379EB71931DA7
:1000200033605379642B02F10701A8BF64232B725C
:1000300031609379EB7002F108033360D3792B714F
:100040003046FAF717FB726833686881D11A0029C5
:100050000CDD591CD8F800003160521A002A1978BA
:10006000417203DD9A1C32605B78437001251EF0FB
:1000700075FD2B46FEF7CDBF844B1868D31C014697
:1000800021329D1E356013F8035C0D705D1E3560D6
:1000900013F8025C4D70336013F8015C8D7003330C
:1000A0009A4201F10301ECD127F0E0F8FEF7CBBF53
:1000B000531C336013787649002B00F074860B785C
:1000C00043F00203901C0B70724D306053782B7517
:1000D0003046FAF7B7FA28603046FAF7B3FA6860A4
:1000E0003046FAF7C7FA28813046FAF7C3FA6A4A67
:1000F000E8811378012543F0020313702B46FEF7C5
:1001000088BFC3F34705122D3FF62DAEC5B107F1E9
:10011000700307F12E0A03EB4508D146A8F1420807
:100120003046FAF7A7FA29F8020FC845F8D15B4B19
:100130003AF8022F23F8022FD145F9D1112D09D811
:10014000574A6B00023B13440021223223F8021F5E
:100150009A42FBD1534A01231D461370FEF759BF43
:10016000DFF8548100233046C8F80030FAF76AFA05
:100170000125C8F800002B46FEF74BBF1346511C63
:10018000316013F8025B3360D31C50783360917890
:10019000002D00F0EB85012D7EF455AF0AF094FBA5
:1001A0002B46FEF736BF374B1B7813F001017FF467
:1001B000DAAD531C3360107801250AF0C7FA2B46DC
:1001C000FEF727BF1346511C3160374913F8020B65
:1001D000C8703360354953784B71D31C3360344B4E
:1001E0009278DA7001252B46FEF713BF3046FAF7F6
:1001F00041FA3046FAF73EFA3046FAF73BFA304613
:10020000FAF744FA3368214D1946581C2A683060C1
:1002100011F8020B82F82C003160597882F8361000
:10022000D91C31609B7882F837303046FAF72EFAC5
:100230003046FAF72BFA3046FAF728FA3046D5F866
:100240000080FAF717FAA8F83A003046D5F800808F
:10025000FAF710FA96E80C00991A0129A8F8380064
:100260000ADD511C2B683160127883F82E2030464D
:10027000FAF70CFA96E80C009B1A032B00F3A884FB
:10028000286811E7288A0020F85C0020CC5B002059
:10029000788800207C8800209C490020DE3D0020DA
:1002A000E03D0020043E002014400020EC890020A6
:1002B000CC460020D85C0020B8510020531C33608D
:1002C000B94DDFF80C83137888F805303046D5F83F
:1002D0000090FAF7CFF9A9F820003046D5F8009041
:1002E000FAF7C8F996E80C00991A0729A9F81E0030
:1002F00000F32085991A032900F30E859B1A002B21
:1003000005DD511C2B683160127883F82620FDF73B
:1003100069FA1FF0E9FCA54B1B68002B00F0A184D3
:100320002868012526F04AFC2B46FEF772BE3046AF
:10033000FAF7A0F9054624F09BF8FF283EF483AEB7
:100340003F2D00F2D28407F17008002308F8403DE9
:100350004FEAD509414607F12F0087F82F3009F100
:10036000010924F065F897F82F305FFA89F905F054
:1003700007054B4505F1010503D197F83030AB4235
:1003800003D02946484624F05FF833687268D21AD1
:10039000012A7EF758AE5A1C07F170003260002225
:1003A0001D7800F8412D24F037F897F82F30AB4234
:1003B0000AD07F4B1B683BB19A79AA4204D31B68D1
:1003C0001B690BB12846984733685A1C3260404677
:1003D00000221D7887F8302024F012F897F830308A
:1003E000AB423EF430AE724B1B68002B3EF42BAE9A
:1003F0001B685B69002B3EF426AE28469847FEF743
:1004000022BE1346511C3160DFF8C48113F8021B71
:1004100088F802103360674953780B70D31C33603F
:10042000654D93782B71131D3360D378092BA8BFCA
:1004300009233046AB70FAF71DF996E80C00991ABB
:100440000129288005DD3046FAF714F996E80C00FA
:10045000E881934240F01084FDF7C4F93368726874
:100460009A423EF4F0AD5A1C32601B78EB700125C5
:100470002B46FEF7CEBD514B1B78012B3EF6E3AD6C
:100480001146531C3360DFF84C8111F8023B88F8A9
:1004900002303160D31C92F801E03360C31A012BA3
:1004A000917840F3CD833046FAF7E4F80125A8F8B7
:1004B00000002B46FEF7ADBD531C336092F8008060
:1004C000B8F1110F3FF64FAC931C33603C4D53789D
:1004D00005F818303046FAF7CDF840F6CA039842CE
:1004E000A8BF184640F2EE23984205EB4801B8BF7A
:1004F00018460125A0F2EE222B46192092FBF0F2BD
:100500004A70FEF786BD2F4A102B4FF0000128BF1E
:100510001023116051609160D1601174002B3EF482
:1005200092AD3168013A0B440131316011F8010C90
:1005300002F8010F9942F7D1FEF785BD531C3360D5
:10054000214B12785A7501252B46FEF762BD511CCE
:10055000316015781F2D3FF606AC052B7FF403ACF8
:100560003046FAF76FF8194B43F8250014F082FA79
:10057000FEF769BD154D05F140083046FAF77AF8E7
:100580003368A5F88000591C1A46316012F8021B26
:1005900085F8821032605B7885F883300435A84591
:1005A000EBD1FEF750BD00BFCC5B002054460020CD
:1005B000C85B002030860020A05E0020BB710020B8
:1005C000C4400020B45B002064630020505A002027
:1005D000D0610020CCA90020531CBB4D33601378A0
:1005E0002B723046FAF746F8A8833046FAF742F8FD
:1005F00028833046FAF73EF8336868835A1C326025
:100600001B78EB7473689A1A032A00F34F833268DD
:10061000991A052900F33A839B1A002B7EF713AD34
:10062000531C3360137885F8213001252B46FEF7E3
:10063000F0BC531C3360A54915780D70C31A002B0C
:100640007EF701AD931C33605378003318BF01234C
:1006500001254B702B46FEF7DCBC3046FAF70AF852
:10066000DFF87C82C8F800003046FAF703F8C8F8D3
:1006700004003046F9F7FEFF0125C8F808002B46B4
:10068000FEF7C7BC924B03F10801501C3060127892
:1006900003F8012F99423EF4D6AC3268F5E71346D1
:1006A000511C31608B4913F8020B8870336053780A
:1006B0004B7001252B46FEF7ACBC0722B3FBF2F2D0
:1006C000C2EBC2055B1B7FF44EABD2B202F1FF3925
:1006D0005FFA89F9002A3EF4B6ACDFF8FCA109F113
:1006E00001091D464B1C336091F900107A4B4FF005
:1006F000000805E008F10108B8F1060F3FF433AB3C
:1007000093F902208A4203F10803F3D10AEBC80BE4
:1007100030468BF80210F9F7ADFF33682AF838003D
:100720001A46591C316012F8021B8BF80310326014
:100730005A788BF80420DA1C32609A788BF80620FD
:10074000191D31600135DB788BF80530A945C9D119
:10075000FEF779BC531C336013780E2B3FF603ABC6
:10076000911C31605578032D3FF6FDAA5B480621A8
:1007700001FB03F1431802F1030E5D71C6F800E0BE
:1007800095784554111D3160D1785970511D3160F3
:1007900011799970911D31605179D970D11D3160F5
:1007A00092791A7101252B46FEF733BC0125FAF721
:1007B000C7FC2B46FEF72DBC531C3360434B12780D
:1007C000DFF82C811A700023C8F800303046F9F7A2
:1007D00039FF3368D8F800203B49414D10435A1C7B
:1007E000C8F8000032601B780B723046F9F742FF00
:1007F00028603046F9F73EFF68603046F9F73AFF67
:10080000A8603046F9F736FF3046F9F733FFFEF7B8
:100810001ABC1346511C334D316013F8021B297169
:10082000336053786B713046F9F724FF33682880C2
:100830005A1C32601B78AB713046F9F71BFF3368E6
:1008400068805A1C32601B78EB7101252B46FEF73D
:10085000E0BBDFF89C800023C8F800303046F9F791
:10086000F1FED8F8003001250343C8F800302B46CC
:10087000FEF7CFBB531C33601578132D3FF673AAD8
:10088000931C336050787A622BF0EAF900283FF429
:100890006AAA7A6A144B017803F82510D11C3160DA
:1008A00003EB850391785970111D3160D0789870F1
:1008B000501D30600D491279DA70086801251EF06C
:1008C000DBF82B46FEF7A5BB646300205C460020E6
:1008D00063630020FC5C0020886B0020C451002072
:1008E000643A0020BC53002060460020CC5B00200E
:1008F000D07100201346511C3160C34D13F8021B08
:100900006970336053782B70D31C33609378AB706D
:100910003046F9F7AFFE33682881591C1A4631601A
:1009200012F8021B697132605B78AB7101252B46AE
:10093000FEF76FBB336872689A4240F0D480B34BC5
:10094000FF221A704FF0000AB14D0DF095FE51468E
:100950002022B04885F800A02FF0FBFF87F830A0D8
:1009600097F83030072B00F23181DFF8CC92A94E96
:10097000524697F8303003EB430309EBC3035B7C2B
:10098000E3B197F8303003EB430309EBC3032021B5
:100990005B699BB197F8303003EB430309EBC3036A
:1009A000586946F82200F8F7B3FF2B7856F8230071
:1009B000F9F76CF82A780132D2B22A7097F8303001
:1009C0000133DBB287F8303097F83030072BD0D9BD
:1009D0002368591C21601A70B8F1000F3EF433AB44
:1009E0008D4BC8F8003001252B46FEF712BB8B4B10
:1009F0003A6A9B68D4F800905A4493424BD23A6AC0
:100A0000A3EB0208FAF73AFB42464946386AFAF77E
:100A1000B5FB236803442360002D3EF414ABB042C1
:100A2000BEF611AB002100E0236801305A1CB04231
:100A300022601970F8D1FEF706BB002DD7D15946B8
:100A40002046F9F771FE23685A1C22601D70734B13
:100A500026689D683B6A0BEB03029542C0F0C68096
:100A6000FAF70CFB5A463146386AFAF787FB2368D7
:100A70000125034423602B46FEF7CBBA3046F9F735
:100A8000F9FD326871687B6A9142834654D106460B
:100A90001D46FEF7F5BDFAF7F1FA5A464946386A9F
:100AA000FAF76CFB236803442360B8E73046F9F794
:100AB000E1FDDFF88881FEF77BBB594B93E822000C
:100AC000FEF7EFBC931C3360564B51781970D11C64
:100AD000316091785970111D3160D2789A7001257A
:100AE0002B46FEF796BA5A1C19463260474811F851
:100AF000022B027031605B784370042A03D9FF2A0D
:100B00007EF4E5AB1EE748490978994205D8022AE8
:100B10007EF4DDABFF2B7EF4DAAB236801255A1996
:100B200022601D70B8F1000F3EF48DAA3F4BC8F84B
:100B300000302B46FEF76DBA511C316012781D460D
:100B4000131C064618BF0123FEF79ABD931C3360A1
:100B50005578022D3FF607A93046F9F78BFD344B47
:100B600003EB45034FF0FF35A3F85C002B46FEF77F
:100B700050BA2F4B0030984418BF0120012588F847
:100B80004A002B46FEF745BA931C3360294B517837
:100B90001970D31C3360DFF89880937888F85B3045
:100BA000131D3360D37888F85A303046F9F762FD68
:100BB000A8F856003046F9F75DFD3046F9F75AFDC2
:100BC0000125A8F858002B46FEF723BA5246FFE647
:100BD0003046D5F80080F9F74DFDA8F832003046D0
:100BE0002E68F9F747FDB086FFF74ABB3B6AED1A5E
:100BF000FAF744FA2A463146386AFAF7BFFA236808
:100C000003442360FEF71FBA60880020B42500204B
:100C1000C67F0020783F0020D5630308DC03002056
:100C2000E04900208D700020596C0020A1C500080B
:100C300064A900207C6B0020E05D0020BC590020EE
:100C4000634B1A88012512FB0EF22B4692FBF1F240
:100C5000A8F80020FEF7DDB9DA46C7F824B0FEF7A1
:100C6000A9BD5C485C495D4A5D4B036001250B6092
:100C700013602B46FEF7CDB9531C33601378003355
:100C800018BF012388F80730FFF7E6BB531C336019
:100C90001378EB723046F9F7D5FC3368E8605A1CDC
:100CA00032601B782B7496E80C00B5E43046F9F7F7
:100CB000E1FCA8843046F9F7DDFC96E80C00991AAF
:100CC0000329E8847FF7A4AC1346511C316013F864
:100CD000021BA9773360537885F820303046F9F746
:100CE000C9FC96E80C00688492E407F1300840469D
:100CF00023F07AFB3B8EAB423FF447AB394B1B688A
:100D0000002B3FF442AB1B689B69002B3FF43DABCB
:100D100028469847FFF739BB3046F9F7ABFCA8F8EF
:100D20000E003046F9F7A6FC96E80C00A8F8100073
:100D3000FFF7E4BA3046F9F79DFCA8F80A00304600
:100D4000F9F798FCA8F80C003046D5F80090F9F7B0
:100D500091FCA9F822003046D5F80090F9F78AFCFA
:100D600096E80C00A9F82400FFF7C4BA012526F084
:100D7000EDF82B46FEF74DB91B4B1020C3F8009041
:100D80005D6017F0E5FB194A137843F00103137017
:100D9000B8F1000F3EF457A9154B0125C3F80080A8
:100DA0002B46FEF736B90B7803F0FD03FFF78AB93F
:100DB0007D62AA46FEF7FEBC00F07F00032828BF34
:100DC0000020012509F09CFD2B46FEF722B900BF4B
:100DD000D2440020D88100202C8200202C860020C4
:100DE00059870008C85B0020E0490020788800206F
:100DF000485900202DE9F04F2DED028B95B080462B
:100E000027F0DAF88E4B1D7825B115B0BDEC028BBA
:100E1000BDE8F08F8B4B1B685905F6D58A4BDFF880
:100E200080B21B686BB1894ADBF800101368CB1ADB
:100E30007C2B06D98648116003780133037026F0B5
:100E40005FFD844B1B78002B6DD0834C834AD4F814
:100E50001031A8EB0303934201F2278394F8189111
:100E6000B9F1000F32D17E4F3868F8F7BBF9C0B244
:100E700001280FD902287B4E42F013803378002BD3
:100E800042F00881D4F81C31A8EB0303B3F57A6F64
:100E900082F0CE82D4F82031002B44D094F818315F
:100EA000BBB9714B1B689B7801211E3B00228B4212
:100EB00084F8181184F82C2142F26C8238680221DF
:100EC000043022F0E3FA94F8243110E0D4F8203111
:100ED0004BB3D4F8283140F6B732A8EB0303934262
:100EE00021D994F82431002B01F0D9865C4F013BC5
:100EF000DBB284F82431002B01F00A84D4F820619D
:100F000094F82C2116F8011B94F82D313868C4F898
:100F100020610A44013384F82C2184F82D31F8F73C
:100F200065F9C4F82881514BDBF800601B7843B1A8
:100F30004F4F386828B14F4B1B78013B012B41F2D2
:100F4000F6834D4B1B786BB14C4F3B6853B1DBF8CC
:100F50000030414C03931A46D4F84431D31A632B22
:100F600001F29381464F3B78022B01F078863D4E8B
:100F700096F87430032B01F0B683424B1B7873B1A3
:100F8000414D2B685BB1344CFDF776FDD4F8503100
:100F9000039044F61F62C31A934200F231813B4B27
:100FA0001B78002B7ED13A4B1B7843B12A4CD4F8E6
:100FB000A03203F5C333A033984581F03782354B17
:100FC0001B78002B3FF421AF234E334C334D06F2F8
:100FD000C1272068F8F706F900283FF416AF20680B
:100FE000F8F7F8F82B7880465A1E33B120682A703B
:100FF000F8F7F8F80028F2D107E703223946781EFF
:101000002FF08DFC96F8C03296F8C12286F8C38284
:1010100083F47F4383F0FF039B1A1FFA88F89BB287
:10102000B8EB132FD5D196F8C222DBB29A42D0D1B9
:10103000781E21F05BFF2B7818442870C9E700BFA9
:10104000A44C0020F4610020E88700205088002094
:101050004C88002026890020B82500203F0D030081
:10106000206F00202C000020246F00202889002001
:10107000FC6C00203089002038890020186F002087
:101080006E3F00204089002044890020B089002064
:10109000C18900204A8900205089002054890020FD
:1010A00060AA0020484C2278A2B1484B9B7A53B1E9
:1010B000FDF7E2FC464B1B68C31AA3F57A73B3F540
:1010C000FA6F07D82278434B43491868F8F756F867
:1010D00000232370414CD4F8983203F5C333A03376
:1010E0009845FFF460AF3E4DC4F898822B78002BF2
:1010F00041F010873B4D2B78002B41F06B8694F824
:101100009C2239498D5CEA0702F10780AF0701F1A3
:10111000C787680701F188872A0748D5334B344EC3
:101120000D9314AA1146A3F13D0241F8202D002091
:10113000A3F140020D4603F8400C05910223112152
:101140005170937028463168F9F7B0FA28467168F3
:10115000F9F7ACFAF389274903EBC3039B00053386
:1011600081FB0321DB17C3EBA101284689B2F9F704
:10117000B5FA338A03EB8303590089B22846F9F79D
:10118000ADFA1D4B059D1B789B0743BF318901F5C7
:101190007A7189B24FF47A712846F9F79FFA0C9B5D
:1011A000327D591C0C9128461A7026F095FE134A80
:1011B00094F89C321178013393FBF1F201FB123366
:1011C00084F89C32EFE600BF188900206463002099
:1011D000DC3E0020B4890020D8880020B8250020FB
:1011E000B8890020B9890020BC890020D888002057
:1011F0007C8800206766666678880020C0890020A9
:1012000094F85631002B41F0CB85D34B1A6802F08D
:101210000803002B48F603414AF60B404BF60F43F8
:1012200049F6074604BF03460E4612F0040F4FF07E
:10123000190118BF1E46970684F8561103D546F4C7
:10124000804646F02006C54B5F79C6F30909002F9A
:1012500042F013819B79002B42F01E821F466420CE
:101260004FF0FF3A4FF0000E0C960D96ADF83E7021
:10127000ADF83CE0CDF842E0CDF846E0CDF84AE0EC
:10128000CDF83890ADF840A08DF84E000CAE0FCEE2
:10129000B34F84F805E00FC796E80F0007C727F89B
:1012A000023B39464FF0010E1B0CFE261F20C822C0
:1012B00001F81E39A670A27184F807E0E07094F876
:1012C0006601207180F0F10383EA0313DAB2130997
:1012D00083F0E70343EA022383EAC2031BB283EAF3
:1012E0000312D2B2C3F3072383EA121343EA0223A1
:1012F00083EAC2031BB283F0C80282EA0212D2B2AE
:10130000C3F3072383EA121343EA022383EAC203E7
:101310001BB283EA0E0686EA0616F6B2C3F307226C
:1013200082EA161242EA062200EB0E0382EAC606A1
:1013300007EB0E0084F86631268011F8013B7340FC
:1013400083EA0313DBB21A0982EA162242EA032275
:1013500082EAC3031BB29EB281422680EDD183F0A4
:101360007C0383EA0313DBB24FEA131E8EEA162EC8
:101370008EEA032E8EEAC30E0FFA8EFE1FFA8EFC43
:10138000784FA4F800C05FFA8EFE4FEA1C2C84F858
:1013900028C084F827E007F5C77904F1220A3868E5
:1013A0007968BA68FB684E460FC610375745B14694
:1013B000F5D1386830606C4E3B7989F8043006F11D
:1013C000270784F8B5E184F8B6C116F8011F28682C
:1013D000F7F70CFFB742F8D194F85731002B41F0E2
:1013E000E4846249DBF8002009780A2084F8570178
:1013F000002901F000865E4E01293088079042F2F4
:10140000518170880690022902F04F80B0880590C3
:10141000032902F05E81F0880490042902F05481CF
:101420000529308902F04C810629B6F80A9002F0AD
:1014300044810729B6F80CC000D0F38994F86611EE
:101440000C920F4687F0300282EA0212D2B21609DD
:101450004849089786F07A0646EA022609882771E5
:1014600086EAC202444EC1EB012186FB017A079E47
:101470004FF0000E66F30F0E069E12B266F31F4E7B
:101480008A44059ECDF834E0C917C1EB6A2A0027CB
:1014900082EA0211C9B266F30F07C2F307220026DF
:1014A00082EA111260F30F06002007926CF30F001E
:1014B000049A8DF845A063F31F40079B109062F3D8
:1014C0001F4769F31F464FF000090E970F968DF8DE
:1014D000449043EA01220DF1300E82EAC106BEE8D3
:1014E0000F0036B286F0C80C8CEA0C1C1C4F84F836
:1014F00005905FFA8CFCC6F307260FC786EA1C1618
:1015000046EA0C239EE8030083EACC031BB283F077
:10151000230247F8040B82EA0212D2B2C3F3072374
:10152000089E83EA1213384643EA022383EAC20282
:1015300006F1010E20F814194FF0230C1621FE2697
:10154000C82384F866E102372280E17084F807C07E
:10155000A670A371114611E07488002060880020F5
:10156000C0250020BA25002047270020946F0020C6
:10157000F4A70020D2A900200308208010F8013B26
:101580004B4083EA0313DBB21A0982EA112242EAD2
:10159000032282EAC3031BB299B2B8422180EDD183
:1015A00083F0F40383EA0313DBB24FEA131E8EEADF
:1015B000112E8EEA032E8EEAC30E0FFA8EFE1FFA4C
:1015C0008EF7C84E27804FEA172C5FFA8EFE84F8FC
:1015D0001EE084F81FC07168B2683068F36806F5D1
:1015E000C7770FC730697169B26904F28F1607C7F0
:1015F00004F2AD1784F8ADC184F8ACE116F8011F10
:101600002868F7F7F3FDB742F8D194F85A31002B68
:1016100041F0DB83B44B06931B681922980684F8CB
:101620005A2140F1EA82B14BB14E1B78990741F142
:101630002187337D042B8CBF03270227FDF71CFA7B
:10164000338A32890C9003EB83035B00ADF84A3098
:101650004FF47A7033688DF84C700E93F18996F8D8
:1016600014E073688DF84DE000FB02F24FF0000CBF
:101670000CAF4FF0FF30CDF834C010920F93ADF89F
:1016800048101190BE46BEE80F000597994F0FC74E
:101690009EE80F0007C73A46182122F81C39E1716D
:1016A00094F8661184F805C081F0780383EA031387
:1016B000D8B2030983F0F60343EA002383EAC003A8
:1016C0001BB283EA0310C0B2C3F3072383EA1013EB
:1016D00043EA002383EAC0031BB283F0C80080EA18
:1016E000001E5FFA8EFEC3F3072080EA1E1040EA58
:1016F0000E2080EACE0000B280F0180383EA0313C4
:10170000DBB2C0F3072080EA131040EA032080EA2E
:10171000C30301F1010EFE204FF01E0C4FF0C8096B
:10172000A0700237217184F866E1238084F803C039
:1017300084F80690184612F8011B414081EA011115
:10174000C9B20B0983EA102343EA012383EAC101EA
:1017500009B288B2BA422080EDD181F0180181EA45
:101760000111C9B20A0982EA102383EA012383EA3C
:10177000C1031BB29AB25B490491DBB24FEA122C4F
:101780002280079384F827C084F826300F4601F59D
:10179000C77A04F1220938687968BA68FB68D646C6
:1017A000AEE80F0010374F45F246F4D13868CEF856
:1017B0000000DFF84C919DF81C3084F8B43109F139
:1017C000260784F8B5C1CA461AF8011F2868F7F73A
:1017D0000DFD5745F8D1FDF74FF9069B71681B6861
:1017E0003289069113F0140F4FF47A71D6F800E0A5
:1017F00001FB02F141F00B860E4694F866A10C90B5
:101800008AF06A003C4B3D4FB3F90420CDF834E038
:1018100080EA0010C0B2030983F0D50343EA002335
:1018200083EAC0031BB283EA0310C0B2C3F30723E9
:1018300083EA101343EA002383EAC0031BB287FB49
:101840000207D2174FF0000CC2EBA7020698DDF892
:1018500014E0109683F0C8070E900F91ADF84A205F
:10186000ADF844C0ADF846C0ADF848C087EA0717E8
:10187000FFB2C3F30726BEE80F0086EA171646EA52
:10188000072686EAC7071B4E84F804A03FB20FC69E
:1018900087F021039EE8070083EA0313DBB2C7F356
:1018A000072787EA13170AF1010E47EA032786E89C
:1018B000070087EAC30384F866E14FF0210A4FF07E
:1018C000FE0E1C27C8220C3684F805C084F807A039
:1018D00084F802E0A6F11C01E7701846A27123808B
:1018E00010E000BFBA25002074880020788800200E
:1018F0007C880020C0250020588800206766666626
:101900004727002011F8012B424082EA0212D2B28E
:10191000130983EA102343EA022383EAC20212B2C4
:1019200090B2B1422080EDD182F0680282EA0212C8
:10193000D2B24FEA121A8AEA102383EA022A8AEA0A
:10194000C20A0FFA8AFA1FFA8AF3D74E23804FEAA7
:10195000132C5FFA8AFA04F1220384F825C084F874
:1019600024A006F5C77E0693F36830687168B268F4
:1019700077460FC7069B10369E42BE46F4D1338889
:10198000CA4E3B804F4684F8B2A184F8B3C117F821
:10199000011F2868F7F72AFCBE42F8D194F866E1E7
:1019A000C34AC44E84F804E08EF0EB0383EA0313C9
:1019B000D9B20B0983F0C50343EA012383EAC103CB
:1019C0001BB283EA0310C0B2C3F3072181EA1011EE
:1019D00041EA002181EAC0010CCA09B281F0C807BE
:1019E00087EA0717FFB24FF0000C0C92C1F30721F2
:1019F000059A0D93CDF838C081EA171343EA0723FF
:101A000007CA83EAC7031BB283F0310786E80700E1
:101A100087EA0717FFB2C3F3072383EA171343EAE2
:101A2000072383EAC703277A607AA17AE27A267BC2
:101A300084F805C01BB25F4087EA0717FFB2C3F303
:101A4000072383EA171343EA072383EAC7031BB27A
:101A5000584080EA0010C0B2C3F3072383EA101392
:101A600043EA002383EAC0031BB2594081EA011014
:101A7000C0B2C3F3072181EA101141EA002181EAD3
:101A8000C00109B24A4082EA0212D2B2C1F307236E
:101A900083EA121343EA022383EAC2031BB25E40C5
:101AA00086EA0616F6B2C3F3072383EA161343EA5F
:101AB0000623607BA17BE27B277C94F811C083EA3C
:101AC000C6031BB2584080EA0010C0B2C3F307231C
:101AD00083EA101343EA002383EAC0031BB2594090
:101AE00081EA0111C9B2C3F3072383EA111343EA60
:101AF000012383EAC1031BB25A4082EA0212D2B226
:101B0000C3F3072383EA121343EA022383EAC203DF
:101B10001BB25F4087EA0717FFB2C3F3072383EACC
:101B2000171343EA072383EAC7031BB28CEA030CAB
:101B30008CEA0C1C5FFA8CFCC3F3072383EA1C13AA
:101B400043EA0C2383EACC03A17CE27C5A4F1BB20C
:101B5000594081EA0111C9B2C3F3072383EA111383
:101B600043EA012383EAC1031BB25A4082EA02120C
:101B7000D2B2C3F3072383EA121343EA022383EAB0
:101B8000C2031BB283F0270686EA0612D2B2C3F361
:101B9000072686EA121646EA022686EAC20636B208
:101BA0000EF10103B2B231204FF0FE0C0C2184F88B
:101BB0006631C8234FEA122E5FFA86FA2280E0715E
:101BC00084F802C0E170A371049E84F814A084F824
:101BD00015E07168B268F3683068B6F810C00FC7D6
:101BE00027F803CB84F8A3E184F8A2A119F8011F18
:101BF0002868F7F7FBFA4F45F8D194F85E71002F8B
:101C000041F0DE802D4B94F866E1B3F90010B3F992
:101C10000220B3F904309FED2A6A677107EE103A8B
:101C2000DBF800300C938EF06A0383EA031306EEB0
:101C3000901AD9B20B0983F0D50343EA012383EA52
:101C4000C1031BB283EA03115242C9B207EE902AC4
:101C5000C3F3072383EA111343EA0123F8EEE77A7B
:101C6000F8EEE66AB8EEC77A83EAC1031BB267EE04
:101C7000867A66EE866A27EE067A002083F0C80C24
:101C8000CDED0E7ACDED0D6A8DED0F7A109011909D
:101C900012908CEA0C160DF13009F6B2C3F3072C42
:101CA000B9E80F000EE000BFBA2500206B27002026
:101CB000E0490020C0250020482700205888002047
:101CC00088C3E43A8CEA161C4CEA062C8CEAC60C53
:101CD000D04E0FFA8CFC0FC68CF01E0799E8070057
:101CE00087EA0717FFB2CCF3072383EA171343EA07
:101CF000072386E8070083EAC707C8214FF00509D4
:101D00004FF01E0CFE231C200EF10102A17184F87D
:101D10005E9184F807C0A370E070A6F1100184F80A
:101D200004E00C36278084F8662111F8013B7B40E3
:101D300083EA0313DBB21A0982EA172242EA03227A
:101D400082EAC3031BB29FB2B1422780EDD183F078
:101D5000270383EA0313DBB24FEA131E8EEA172E22
:101D60008EEA032E8EEAC30E0FFA8EFE1FFA8EFC49
:101D7000A94FA4F800C05FFA8EFE4FEA1C2C84F82D
:101D800025C084F824E007F5C77904F1220A3868F1
:101D90007968BA68FB684E460FC610375745B1469A
:101DA000F5D19E4E3B88A9F8003006F1240784F84F
:101DB000B2E184F8B3C116F8011F2868F7F716FAE4
:101DC000B742F8D194F85F91B9F1000F40F0F28773
:101DD000934B1B68052284F85F219A0641F1158117
:101DE000904ADFED917AD18907EE101AB8EEC77AE2
:101DF00013F0140F27EE277A01F071838B4BDFED80
:101E00008A6AD3ED007AF8EEE77A67EEA67A94F85C
:101E100066C1874B874AB3F90410B2F90620864E93
:101E200086488DED0D7A8CF0220383EA0313DFB22E
:101E30003B0983F0590343EA072383EAC703B2F55A
:101E4000FA6F1BB2A8BF4FF4FA6283EA0317FFB21E
:101E5000B2F57A7FC3F3072383EA1713B8BF4FF4B1
:101E60007A724FF0640E43EA0723A2F57A720EFBF2
:101E700002F283EAC70786FB02E680FB01E03FB27D
:101E8000C917D217C2EBA612C1EBA0034FF0000A8C
:101E90000CA987F0C806CDED0E7AADF84220ADF85A
:101EA0004030CDF830A0CDF83CA08E4686EA06162C
:101EB000F6B20591C7F30727BEE80F0087EA1617A9
:101EC00047EA062787EAC606524FDEF800E084F8A4
:101ED00004C00FC736B286F04A0383EA0313DBB2AD
:101EE000C6F3072181EA13113A4641EA03210CF1B6
:101EF000010C81EAC303142042F810E9FE264FF0DA
:101F00004A0E002184F866C14FF0C80CE0702380AF
:101F1000043784F807E0A670617184F806C018469B
:101F200012F8011B414081EA0111C9B20B0983EA91
:101F3000102343EA012383EAC10109B288B2BA42FD
:101F40002080EDD181F0140181EA0111C9B24FEA7C
:101F5000111E8EEA102E8EEA012E8EEAC10E2E4B35
:101F60000FFA8EFE1FFA8EF61F464FEA162C5FFA06
:101F70008EFE84F81CE084F81DC0386859689A68A1
:101F8000DB68B7F818A0049726803E4607F5C777A8
:101F90000FC73069716903C704F28F16A7F800A054
:101FA000374684F8ABC184F8AAE104F2AB1A17F8FB
:101FB000011F2868F7F71AF9BA45F8D1204B214AD2
:101FC0001B781278013B12F00100DBB214BFC02174
:101FD0004021172B03D81C4A134493F830901B4B15
:101FE0001A8897071ABF002341F01001012312F449
:101FF000027F18BF022312F0100F18BF062312F041
:10200000200F18BF1023002841F008824FF0030C66
:102010001EE000BFC0250020BA2500204727002071
:10202000748800207C8800200AD7233C5488002034
:1020300058880020F4A70020D34D621067666666BA
:102040005C460020288A0020081004087C5B0020E1
:1020500094F866E10C938EF0460383EA0313DAB238
:10206000130983F0920343EA022383EAC2031BB2FB
:1020700083EA0310C0B2C3F3072282EA101242EAD5
:10208000002282EAC00212B282F0C80787EA07176C
:10209000FFB2C2F3072282EA171200238DF837C07D
:1020A000032042EA072C059A8DF834908DF83530DC
:1020B0008DF836108DF8380007CA8CEAC70C0FFA75
:1020C0008CFCD04FE3718CEA0C1903C75FFA89F9D5
:1020D000CCF3072C8CEA191C4CEA092181EAC909C6
:1020E00094F808C03A700FFA89F98CEA090C8CEA66
:1020F0000C1C5FFA8CFCC9F3072282EA1C1242EA2C
:102100000C22607AA17A94F80B90637182EACC0277
:1021100012B2504080EA001C5FFA8CFCC2F3072028
:1021200080EA1C1040EA0C2080EACC0000B241405A
:1021300081EA0111C9B2C0F3072282EA111242EA10
:10214000012282EAC10212B289EA020989EA091966
:102150005FFA89F9C2F3072282EA191242EA0922D8
:1021600094F80CC0607BA17B84F804E082EAC90289
:1021700012B28CEA020C8CEA0C1C5FFA8CFCC2F3E3
:10218000072282EA1C1242EA0C2282EACC0212B234
:10219000504080EA0010C0B2C2F3072282EA101257
:1021A00042EA002282EAC00212B2514081EA0111E1
:1021B000C9B2C2F3072282EA111242EA012282EA7C
:1021C000C102E17B94F8109013B281EA030282EA23
:1021D0000212D2B2C3F3072383EA121343EA0223A3
:1021E00083EAC2031BB289EA030282EA0212D2B274
:1021F000C3F3072383EA121343EA022383EAC203E9
:102200001BB283F0320282EA0212D2B2C3F3072376
:1022100083EA121343EA022383EAC2031BB29AB28F
:102220004FF0FE0C5FFA83FB0920C8210EF1010E6E
:1022300084F802C04FEA122CE070A17184F866E1C4
:10224000228084F812C084F811B0049B1868596881
:102250009A68B3F80CA007F5C07EAEE8070007F552
:10226000C8778EF80290AEF800A084F8A0C184F878
:102270009FB116F8011F2868F6F7B8FFB742F8D1EA
:10228000039BC4F85031FEF78ABEDFF898A15E4E7A
:10229000DFF89491412021F0A7F8BAF9023086FBCB
:1022A0000320DB17C3EBA00080B221F081F8BAF95C
:1022B000003086FB0320DB17C3EBA00080B221F0C7
:1022C00077F8BAF9043086FB0320DB17C3EBA000D4
:1022D00080B221F06DF899F800103868F6F786FFA3
:1022E00094F848A11AF0010600F0F784474B0693D2
:1022F0001B689A0673D5464B464E1B789B0741F1E7
:102300005180337D042B8CBF4FF0030A4FF0020A3B
:10231000472021F069F8306821F016F8706821F044
:1023200013F83D4AF3893868A2FB0323C3F347132C
:1023300019460493F6F75AFF069B99F800101A689D
:10234000049B12F0140F83EA010389F8003040F077
:1023500067863389642000FB03F020F0F5FF367DAB
:1023600038684AEA8606F6B23146F6F73FFF99F832
:10237000003038685E40314689F80060F6F736FF75
:1023800094F848A1BAF1000F29D1244E4F2021F032
:102390002BF8306820F0D8FF706820F0D5FF504649
:1023A00020F0D2FF01213868F6F720FF184A99F88B
:1023B00000301678386806F00106314683F00103D4
:1023C00089F80030F6F712FF99F8003038685E405F
:1023D000314689F80060F6F709FF94F848A1039B9D
:1023E0000F4AC4F844310AF10103DBB2A2FB031225
:1023F000D20802EB8202A3EB420384F84831FEF7D5
:10240000B1BD00BFC02500206766666674880020E5
:10241000788800207C8800201F85EB51E04900204F
:10242000CDCCCCCC588800201C6F002094F8A4326E
:10243000C24AC4F8A08202EB8302926C42B314AD8C
:1024400004F2AB23BE4E45F8203D002104F2BD232B
:1024500031800D9380211523A52784F8AA322846C0
:1024600084F8A91284F8A872904728463188F8F7B2
:102470005BF90C9DB34804F52A716D1A152DA8BFA0
:1024800015252A462BF050FFAF4A94F8A432157058
:10249000AE4A013382FB0312A2EBE37202EB42026B
:1024A0009B1A84F8A432FEF78ABDA94AA94BD4F836
:1024B0001411DBF800001B88D77AA74A401A4FF4A2
:1024C0007A71DEB201FB07F11B0A96771675884216
:1024D0004FF00006D37753759670167180F0D18453
:1024E0009E4E9F4BD6F800C01B689E4E9E48DFF85C
:1024F000989201688068DFF894E286FB0376DB1728
:10250000C3EB661303F5FA739BB293761B0AD3767B
:1025100089FB0173C917C1EBA30189FB007911770E
:10252000C0170912C0EBA90051778E4982F820002C
:102530000CF5EA43001281FB0C71303382F8210064
:102540004FEAEC701B12C0EB6110884E9EF800E061
:1025500082F823307830864B82F824000CF1300169
:10256000307D03901EF0020F82F82210987600F062
:102570008584D6F800E07F4AD6F804A07E48DFF8CC
:1025800010C282FB0E194FEAEE7182FB0A72C1EB98
:10259000A9514FEAEA79C9EBA25200FB01E900FB1D
:1025A00002A009EB490900EB40004FEA490940004D
:1025B000049207468CFB0920801405908CFB072CA5
:1025C000F089049A3689079702EB820206F5FA76BB
:1025D00000EBC00002EB8202B6B204960892059EA0
:1025E0008200099201EB81014FEAE972B01A01EB16
:1025F0008101624E06910246039906FB1292069EE5
:1026000040B2052900EB86004FEAE7714FEAAC4C77
:102610005A4E0590ACEB0100014606FB1070089E77
:10262000504FDFF870C14FEADA7A49B201EB860108
:102630004FEADE7E87FB006983F80EA087FB026A03
:10264000099F83F809E0DFF850E13E468EFB066EF5
:10265000BCF8006003969DF810605E75049EBDF89E
:1026600014C083F80AC04FEA162689B204964FEACE
:10267000E2724FEAE777424ED973C2EB6A12C7EBB8
:10268000AE174FEA1C2A4FEA112E4FEAE070039969
:10269000368883F80BA0C0EB691083F810E04FEA8E
:1026A00022291A739DF810209A754FEA202CC7F33F
:1026B000072A4FEA112134BF4FF0320E4FF0330E8C
:1026C0009DF80C2083F80D90587483F812C0DF71C8
:1026D00083F808A0DA74197583F81BE01E77C4F834
:1026E0001081FEF7BBBBDFF8B490D9F80000F6F715
:1026F00069FD00283EF441ACD9F800000121F6F74D
:102700005DFD0222002386F874203B70FEF735BC85
:1027100094F82C1194F82D3138684A1C013384F850
:102720002C2184F82D31F6F761FDFEF7FABB154C2C
:10273000DFF86C904FF0000A3FE000BF081004087B
:10274000EC870020C43C0020D93C0020565555554C
:102750004C6D0020446D00205889002048880020DE
:10276000548800201F85EB51F08700207C880020D2
:10277000848900206BCA5F6B806967FF40420F004D
:10278000B25B0020B8250020676666667888002066
:1027900083DE1B43D6A90020D34D62107840002071
:1027A0002C0000201B2B00F06F820D2B00F04B81C2
:1027B0004FF0010389F801303868F6F713FD00285F
:1027C00039D03868F6F706FD83B27E2BDBF800209F
:1027D0002AD099F801100029EED194F82E21002A70
:1027E000E0D07D2B00F0368294F83CE1BEF1000F82
:1027F00004D080F02003DBB284F83C11511CC9B234
:102800002244092984F82E1182F8303100F0168212
:102810000829D1D8B4F83A21134403EB132303F069
:10282000FF03A4F83A31C7E784F82EA184F82FA15A
:1028300089F801A0C0E794F83D3133B194F8313103
:1028400084F83D01302B00F0C18594F82F21C54B51
:10285000C549DFF850A3DFF850E391464A46002A05
:102860003EF46FABDBF80020921B012A24D894F8C9
:102870003E21002A40F01E8294F83FC133F81C002C
:10288000F8B94FF0010284F83F210A689706E5D5B0
:102890009AF800209007E1D5B44EB549F2894FF47B
:1028A000F36303FB02F381FB0321DB17C3EB61112D
:1028B0004FF4036020F0D0FD002384F82F31FEF7A1
:1028C00040BB0CF1010C5FFA8CFCB0F5E06F84F8B2
:1028D0003FC100F098801BD8B0F5047F00F0238141
:1028E00035D8B0F5887F00F0CD80B0F5007F00F0DE
:1028F000B380B0F5807FB1D10A685207AED59D4B49
:10290000196820F0A9FD002384F82F31FEF719BBC8
:10291000B0F5026F00F05A816AD8B0F5E46F00F0AC
:102920008180B0F5006F00F0D680B0F5E26F95D1F0
:10293000914BDA6B998A642303FB02F393FBF1F169
:1029400020F08AFD002384F82F31FEF7FABAB0F5A3
:10295000826F00F05181B0F5C06F00F02781B0F5B3
:10296000806F7FF47BAF94F840310133DBB2032BEF
:1029700000F2AD8142F2107184F8403101FB03F1A5
:102980007E4B1B88002B40F0A08101317C4B1B78D3
:10299000DB077C4B1B8848BF0431DF0748BF0A3187
:1029A000980748BF14311A0648BF2831DF0548BFD1
:1029B0002831580748BF64311A0748BFC8319F05FE
:1029C00048BF01F5C871980648BF01F57A71DA066B
:1029D00048BF01F5FA615F0648BF01F57A614FF41F
:1029E000806020F039FD002384F82F31FEF7A9BA6A
:1029F000B0F5046F1AD0B0F5116F52D0B0F5036F77
:102A00007FF42CAF41E75C4B91469A6B998A642323
:102A100003FB02F393FBF1F120F01EFD84F82F91EC
:102A2000FEF78FBA544B91461A6CEFE7564BB3F949
:102A3000041001EB81019146490020F00DFD84F85E
:102A40002F91FEF77EBA4FF0010184F82E1184F821
:102A50003031A4F83A21AFE69EF80620002A3FF470
:102A6000FDAE4A4B4A491B6881FB0321DB17C3EBD0
:102A7000A1014FF4007020F0EFFC002384F82F3107
:102A8000FEF75FBA0A6852077FF5E8AE414B4FF494
:102A90008870196820F0E0FC002384F82F31FEF7DD
:102AA00050BA9EF80520002A3FF4D8AE3A4A107872
:102AB00000283FF4D3AE394B1B8803EB8303590046
:102AC00091FBF0F14FF4116020F0C6FC002384F874
:102AD0002F31FEF736BA0A6897067FF5BFAE9AF82F
:102AE000002090077FF5BAAE1CF0010F1F4E204961
:102AF00000F05C84726882EAE273A3EBE27303EB9A
:102B00005303A1FB0331C908002AACBF41F00041C7
:102B100041F040414FF4006020F09EFC002384F817
:102B20002F31FEF70EBA9EF80520002A3FF496AE2C
:102B3000194A107800283FF491AE194B5B7B002BAB
:102B400000F09484154B1B8893FBF0F000EB8000A1
:102B500041004FF4047020F07FFC002384F82F31F3
:102B6000FEF7EFB908100408748800207C88002064
:102B70001F85EB515488002000880020ECA900201C
:102B8000288A00207C5B002058880020F0870020E5
:102B900067666666488800205A6D0020446D0020F4
:102BA0004C6D002078880020608800209EF8062068
:102BB000002A3FF453AEC34B4FF4C060996820F035
:102BC0004BFC002384F82F31FEF7BBB90F68BF061A
:102BD0007FF544AE9AF800C01CF0020F3FF43EAE01
:102BE000B94E33896421914601FB03F120F034FC96
:102BF00084F82F91FEF7A5B90A68900640F1F1809C
:102C0000B24BB14E1878317D00F00203002B0CBF9F
:102C100000234FF47A7340F6B83208BF4FF4FA62DB
:102C200010F0010F18BF134619444FF4826020F0D2
:102C300013FC002384F82F31FEF783B9B4F83A214E
:102C4000C2F1FF0293427FF4B3AD4FF0010384F869
:102C50003D31ADE54FF0010384F83C31ACE5FBF7C5
:102C60000BFF9B4B1B68C01A40F6B833984200F22A
:102C70001E81DFF89CA29AF804303A2B00F0BA8249
:102C800000233B70FEF779B93868F6F7ABFA0028F5
:102C90007FF48EAD4FF0010384F82F318CE5C4F83A
:102CA000203184F818318B4F20F024FC94F8243123
:102CB000FEF71DB98849062020F0A2F9002384F808
:102CC0003E0184F82F31FEF73CB902315EE6012364
:102CD00084F8403142F2107152E6804B1B88D805CF
:102CE00013D4D90600F17A839A0600F1F1835806CD
:102CF00000F1F383190700F1F983DA0700F1148476
:102D000013F0020F0CBF04260C26754B754A1B7876
:102D1000D27803F001030AB143F002035320049375
:102D200020F062FB704A128802EB820202EB820200
:102D3000900080B220F03CFB002020F039FB6B4A71
:102D40006B4912883868C2EBC212520081FB023113
:102D500011444FEAE27ACAEB612A5FFA8AFA5146D5
:102D6000F6F744FA99F80020049B38681E438AEA73
:102D7000020A002189F800A0F6F738FA31463868CF
:102D8000F6F734FA99F8003038687340DBB2194628
:102D900089F80030F6F72AFA94F848A1FFF7F2BA5A
:102DA000013B84F85631FEF717BB013B84F85731DD
:102DB000FEF72BBC09F1FF3984F85F91FFF760BA89
:102DC000013F84F85E71FEF7FDBF013B84F85A3184
:102DD000FEF713BF47493A2020F012F92870FEF79A
:102DE000E2B8454A1268120600F1FA82434A127BA1
:102DF000002A3FF433AD94F84111032900F28A838D
:102E0000DFE801F0322819023D4B1B6859799A79A5
:102E1000DB7901F1407101EB022101EB0341002359
:102E200084F841314FF4826020F016FB002384F8CF
:102E30002F31FEF786B8334B1A68137A507992789F
:102E40001B0403EB002313444A1C84F8412103EBC9
:102E50000161E7E72B4B1A68D379107952781B048C
:102E600003EB00231344EFE7264B1A689379D078DD
:102E700012781B0403EB00231344E5E72D22DA76D6
:102E80002DE4214BDBF800101B78C4F81411013B32
:102E9000012B3FF625AB1021022391701371FFF730
:102EA0001FBB20F017FB01233370FDF7F3BF174A58
:102EB000B2F84A3100210133A2F84A313970FEF7E5
:102EC0005CB800BFF08700207C8800207888002054
:102ED000743F0020206F0020533403087C5B0020E7
:102EE000288A0020845B0020446D0020D2A90020A5
:102EF00003082080397F0308F46100204C6D002016
:102F0000D85C0020CC5B0020E0A90020B825002080
:102F10005C3F0020A64EA74B00930024A6F13F0182
:102F2000A54BA64A0A9106F8404CA5490B960CA859
:102F3000F7F7D2FC0A9E731C0A9334700A9B29226D
:102F4000591C0A911A700A9BEA22591C0A911A709C
:102F50000A9BC822591C0A910CA81A702AF020FC5E
:102F6000471C0CA93A460A982BF0DEF90A9AD319A5
:102F700001330A93D4550A9B5A1C0A921C700A9B6F
:102F80005A1C0A921C700A9B5A1C0A921C700A9BBB
:102F90005A1C0A921C700A9B5A1C0A921C700A9BAB
:102FA0005A1C0A921C700A9B5A1C0A921C700A9B9B
:102FB0005A1C0A921C700A9B5A1C0A921C700A9B8B
:102FC0005A1C0A921C700A9B5A1C0A921C700A9B7B
:102FD000FF22591C0A911A700A9B0122991814A801
:102FE0000A911A7050F8283D9B1B337024F074FF2F
:102FF0002C70FDF7D8BF8C46894608460491059190
:10300000069107910B46FEF719BA9FED6E7A13F001
:10301000140F08BFF0EE477A7EF4F0AEFEF7F7BE6D
:10302000694B1868FFF799B9684A614B12680D93AC
:10303000A3F14007002103F8401C2123D100BB70FD
:1030400040F13A8262490326624B1B885A0500F11F
:103050002982D80700F13E8203F002035E4A002B6A
:103060001CBF03261146DFF88891324648462BF0F4
:103070005BF906EB090314A80133A9F1020140F83A
:10308000203D00225B1A06F809207B7024F024FF03
:10309000FEF742B8C4F81C8186F80090FDF7FABE2E
:1030A000434A4E4B0D9214AEA2F13D0046F8200D5E
:1030B00019884B4FA2F1400300204FF00A0E02F88E
:1030C000400C082283F801E030469A70F7F706FBBF
:1030D0003B684449DA1781FB0313C2EBA30399B29F
:1030E0003046F7F7FBFA07F01FFCBF680C9B3A0C61
:1030F000591C0C911A700C9B3A0A591C0C911A70AD
:103100000C9B5A1C0C921F700C9B5A1C0C92187032
:10311000304624F0E1FEFDF7FCBF334F9FED338ACC
:10312000B7F9022022480D9007EE902AF8EEE77AD0
:1031300014AE67EE887AA0F13D01FDEEE77A46F81D
:10314000201D00F8403C0823CDED037A00F83F3CF9
:103150001E23BDF80C1000F83E3C3046F7F7BEFACF
:10316000B7F9003007EE903AF8EEE77A304667EEAE
:10317000887AFDEEE77ACDED037ABDF80C10F7F70B
:10318000ADFAB7F9043007EE903AF8EEE77A304638
:1031900067EE887AFDEEE77ACDED037ABDF80C1084
:1031A000F7F79CFA304624F097FEFDF7AFBF00BF5B
:1031B000D8880020726B00200043040808430408EC
:1031C000144304080000000054880020E4A90020F3
:1031D000EC4204087C5B0020FC420408446D0020A3
:1031E000F0870020676666665888002058A08B41EB
:1031F0009B8800209AF80240C4B1013CE4B201343B
:1032000054445146002211F8013B534083EA031312
:10321000DBB2120ADE0042EA03228C4286EA131372
:1032200082EA0302EFD1002A7FF42AADC04AC14EE0
:10323000C14B1288C149C24CF261DFF838931A6859
:1032400009689B68F262B4F84A21F066F364D9F821
:103250000000F163F265F4F78FFF039000287DF41E
:1032600087AE0221D9F80000F5F7A8FF94F84C3199
:103270009AF803200492642B4FF0040286F874201D
:1032800040F07C8194F84D31072B04BF9DF80C3041
:1032900084F84D3194F84D31079306EB031ADAF8B0
:1032A0000410039108462AF07BFADAF80810069118
:1032B0005FFA80FA08462AF073FAC0B205900AEB6A
:1032C0000002079B9F48039903900832C27123F0C4
:1032D0000F0286468272059803F00F0300EBCA00C6
:1032E0008EF80D3052468EF80E000EF10F002BF0C6
:1032F0001BF8954B059A06990AF1090018442BF022
:1033000013F80398C37903F1010ACBB1013B5FFACB
:1033100083FC0CF1080CDFF860E2844400230730E2
:1033200010F8011B59408B00CA0883EA410302F0E0
:1033300018024B404EFA02F253408445DBB2EFD103
:10334000814A04980AF8023027F052FC94F84D3173
:103350000022013384F84D3184F84C21039BDDF8C1
:103360000CA09B785BB11AF80510D9F80000F5F7AE
:103370003DFF01359AF80230EDB2AB42F3D894F834
:103380004C310322013384F84C3186F874203A70B2
:10339000FFF7ABB902213868F5F710FF94F8243134
:1033A000FDF7A5BD4FF0010AFEF7B2BF326882EA11
:1033B000E273A3EBE27303EB5303A1FB0331C908F0
:1033C000002AB8BF41F08041FFF7A4BB5F49881FC6
:1033D0001FF0BAFE84F83E01FFF737BA342694E4B2
:1033E00010230026042218460CA98DF830308DF8E1
:1033F00031208DF832608DF833608DF834608DF8AF
:10340000356020F00BF884F82F61FDF79ABD4B4B27
:103410001E6806EB86067600FEF7EFB94C4AD278B6
:10342000002A0CBF4FF0040C4FF0050CFEF710BE45
:10343000012338683370F5F7CDFE06463868F5F796
:10344000C9FE72067DF426AD8A2851D08E287DF4FF
:1034500021AD94F81831002B7DF438AD3D4BC4F804
:1034600020312D2384F82431FDF71BBD304B188803
:10347000FFF76CBB0127FEF7E1B82D499A790B885D
:1034800003EB830303EB83039F00BFB2002A00F02A
:103490001181294B1B680FFA83FA07F045FA40B2F5
:1034A000FDF7E0BE03262C49DDE59C46994618460B
:1034B00004930593FDF7C2BF284B294A1B6829498D
:1034C00003F48003002B16BF114604260326BBE538
:1034D00024261AE424490426C5E5102615E4138998
:1034E00007EE903AF8EE677AFEF791BC20260CE4DE
:1034F0001E4B1B689B067DF5CDAC94F81831002B54
:103500007DF4E4AC1A4BC4F820312D2384F8243127
:10351000FDF7C7BC4B1CDBB2042B84F841314FEAEA
:1035200001613FF47CAC7DE40826FFF7EEBB00BFF1
:10353000446D00202C000020F087002054880020DB
:10354000B82500200CA4002012A40020F0260020A2
:10355000845B002058890020F0420408F4610020B8
:10356000EC420408E4420408F44204087488002091
:1035700084890020784000200007090E96F875A085
:10358000574905951AF00F0F04BF0AF1010A5FFAB7
:103590008AFABAF1070F28BF4FF0010A4FEA0A1C56
:1035A00006EB0C03187C4F4B03930A18002392F888
:1035B00024104C4A93725FFA8CF31A464A4B964693
:1035C00006EB0C024EEA000001291870D26803F1E4
:1035D00001000CD90239C9B28D1C1D44034603F801
:1035E000012BAB424FEA1222F9D101310844B44415
:1035F00022F060030AF1010A9CF811205FFA8AFAAE
:103600001343BAF1080F037000F1010340D04FEAF1
:103610000A1C06EB0C01344A087C314901449A1A11
:1036200091F8241055180EF1100E132D5FFA8EFE2E
:10363000C6DD059D0398DFF8BCE0D2B2931DDBB276
:1036400043F04001C17103F1010CCBB10532D3B29B
:103650000833C31805930EF10100002310F8011B75
:1036600059408B0083EA4103CA084B401F4902F0CE
:10367000180241FA02F25340059A8242DBB2EDD1C0
:1036800004980CF80E3086F875A027F0B1FA65E6BC
:10369000154A059D9A1ACDE7154B6420B3F900A091
:1036A000FDF7E0BD9C4699461846049305930693A2
:1036B000FDF7C4BE4FF0FF33EDE69C46FDF7BEBEFE
:1036C0009C469946FDF7BABE9C4699461846FDF7BA
:1036D000B5BE9C46994618460493FDF7AFBE00BFA1
:1036E000081004080CA4002019A400200007090EEB
:1036F000F087002012A400202DE9F04F724B734A8E
:103700001C7893B000F59C412031814607911160EF
:10371000002C00F027856E4A1268904240F2278202
:103720006C4A6D491768DFF8E8B10492013C1C70DF
:103730006A4C039107F48057002F40F02582039BC9
:103740005B7D002B40F09B84049B1B681D0400F1F3
:103750007787634B9945A37800F27383002B40F081
:103760007383604B0693049B1F6817F4805940F0E5
:10377000FA83039BBBF906605B8B9E42B4BF0026B5
:103780000126594B1B6813F0805300F00782069AFC
:10379000127812F0010200F0088203985349408C1D
:1037A00091ED037A07EE900AF8EEE77AB4EEE77A45
:1037B000F1EE10FA81F20A80002E40F0FD814C4DAE
:1037C00095F8A010002940F0F7814A484A49056859
:1037D00095F82D5000200860486088604749002D0A
:1037E00040F0EB810D70002A40F0EC81444B1A78D8
:1037F000002A50D10399BBF900E04F8B898BBBF9AC
:103800000200BE45CCBF8025002545F040038E4513
:10381000A8BF2B469B0843F08005B842C8BF2B4683
:1038200043F040058842A8BF1D46BBF904E0BBF940
:103830000600AD0845F08003BE45C8BF1D4645F0F3
:1038400040038E45A8BF2B469B0843F0800E284DB1
:10385000B842C8BF734643F0400E95F8A270884244
:10386000B8BF73469F4201F04081A5F8A42085F8B7
:10387000A620244985F8A2300F78002F01F0B180EE
:103880005F2B01F018816F2B00F0F887069B1B78E7
:10389000D90740F1BA87049B1B4A1B68059203F0C5
:1038A0000403002B40F04A850DF14008174D00231A
:1038B000C8F8043005F15009109340F6330A19276F
:1038C00040F2833629E000BF28400020DC3D002084
:1038D00024400020F461002064630020845B002009
:1038E000404B4C00288A0020E4A900205C6D002099
:1038F0007C280020CC5B002010410020E82A00201A
:103900006D8A00201A020020748800206046002082
:10391000F4A7002004354D4520D0AA78EB789A42D0
:1039200017FB0261F6D26A78043217FB03633BF996
:1039300012205245A8BF5246B2F5617FB8BF4FF47E
:1039400061729142E6DA9A42E4DC29782429E1D8CE
:1039500040460435F7F72EFA4D45DED1B04B98E8D6
:1039600003001F78AF4B83E80300002F00F03C8476
:103970000121AC48F7F72EFA002840F09A81E3784D
:10398000002B40F09681A84C23881DB225F001053C
:10399000AEB2B342268000F0B286A44D02270E20BC
:1039A0004FF014094FF0FF082F7085F8019085F84B
:1039B000028014F09DFC39469A482688F7F70AFAE7
:1039C000002841F0458026F002039BB2B3422380D9
:1039D0000AD0964B1421FF2202250E201D7059702B
:1039E0009A7014F085FC2688914BDFF884A2197830
:1039F000DAF804000393B50708BF81F00201C1F3B0
:103A00004001F6F75DF824218648F7F7E3F930B96D
:103A1000069A1378590744BF23F004031370059BDB
:103A20001B6813F00A0F1DD005217E48F7F7D2F965
:103A3000002800F0988625886F0740F1B5877948FF
:103A40000621F7F7C7F9002800F07A866E0640F1E4
:103A5000888707217348F7F7BDF9002840F03083C5
:103A6000059B1B689D0600F13B8327886D480C2150
:103A7000F7F7B0F9002800F0388147F48073BB42B3
:103A8000238009D0694B02251421FF220E201D70CE
:103A900059709A7014F02CFC664B1B78082B00F0C0
:103AA00030810E2B00F02D81049B1B685E0544D5F0
:103AB000614B1B79002B00F0E18014215948F7F786
:103AC00089F9002840F0DF8024F076FA012014F014
:103AD00051FB90B3DFF89C8100254FF0CC0902E048
:103AE000DDB2022D29D809FB05F76B1C58F80760D9
:103AF000002EF5D1C378514A90F9020052F82330D4
:103B00000196032200920121324613F0D9FA0346AE
:103B100005EB450000EB0010049353B1314608EB70
:103B20008000CC222CF015FF049B48F807300135AB
:103B3000EDB21EF023FB0028D3D1069B1B78DD07D6
:103B400040F1F2803E493F4A01230B701370039B02
:103B5000DAF80000197801F00101F5F7B1FF059BD3
:103B60001B685A0700F1508113B0BDE8F08F364B47
:103B7000364A1F68049307F480570392DFF8F8B0C1
:103B8000334C002F3FF4DBAD00212648F7F722F934
:103B900000287FF4D4AD0AF009FFD0E578023FF5A4
:103BA000F6AD069A127802F001022A4D002185F83E
:103BB000A010002E3FF409AE274901200870002A0A
:103BC0003FF414AEF9067FF511AE244A1278D206FE
:103BD0003FF50CAEB9F1000F7FF408AE002B7FF477
:103BE00005AE7B023FF502AE1D4B1B78002B01F0AA
:103BF00021841C4B9B78002E41F059843BB11A4A1A
:103C00001A4B12681B689B1A002BC1F28B84102080
:103C1000104D14F06DFB012385F8A130E6E500BFDF
:103C2000A44C0020E4A900207C5B0020C4530020A9
:103C300000B400205C4600204C6D002024390408AC
:103C4000298A00205C590020F46100206463002070
:103C5000845B00207C280020E82A0020788800204F
:103C60001A020020FC5C002060AA0020F43B002027
:103C700004B4002034A40020F4A70020069B1B7885
:103C8000D8077FF521AF3C2026F006FE00283FF440
:103C900054AF07F0E9F83C2026F0A0FD00283FF4DF
:103CA0004CAF07F0E1F83C2026F098FD0028F0D159
:103CB00043E7059B1B689A077FF565AEBF4C2688D6
:103CC000F3073FF580AE46F001039E4223803FF4A8
:103CD0007AAEBB4B1421FF2202250E201D705970B5
:103CE0009A7014F005FB26886DE627F480739BB26A
:103CF000BB4223807FF4C6AEB24B1B78082B7FF407
:103D0000D0AE228822F040039BB29A4223803FF437
:103D1000CBAEAB4B02251421FF220E201D70597033
:103D20009A7014F0E5FABFE6A74B93F80090B9F14A
:103D3000000F5FD1DFF8E482A44F18F8030C3E783F
:103D40004146A8F103051AF067FE002800F0F08351
:103D5000002E40F0428405F1080168791AF05CFEFB
:103D6000002841F0E9819A49A87A1AF055FE002806
:103D700000F0F183022E41F0E3819649E87B1AF0CE
:103D80004BFE002841F0E0819349287D1AF044FE63
:103D9000002800F0F183042E41F0DA818F49687E1B
:103DA0001AF03AFE002841F0D7818D49A87F1AF019
:103DB00033FE002800F0F183062E41F0B9818949D5
:103DC00095F823001AF028FE002840F0588786490D
:103DD00095F828001AF020FE002800F0F183082E44
:103DE00040F03787814995F82D001AF015FE00281C
:103DF00040F0F1837E4B01221A701BF090F8059B76
:103E00001B685A077FF5B0AE03201AF02FFE00287A
:103E100000F06686238813F008047FF4A5AE08201E
:103E200014F0AEFB7348744D7449754A754BBBF87A
:103E3000066000682E80086014601C6013B0BDE846
:103E4000F08F0BB90123A3706F4B06931B201F78D3
:103E500094F821601AF00AFE012E07F0010982464B
:103E600000F0258607F00203059394F82030DFF870
:103E7000B081664D052B69D8DFE813F05B004F0079
:103E80000600DC00FF008D00012E04BF052384F82E
:103E90002030B9F1000F00F05281039B5C4FB3F961
:103EA0001810B8F80030002261F30F0263F31F42CC
:103EB000002361F30F0361F31F43CBF8042039683B
:103EC0006269CBF800308A42C0F06784012E41F06D
:103ED000FE82032294F820300592CBE71AF0F2FD1F
:103EE000012807D14A4FB8F802303A68642101FB33
:103EF00003232361BAF1000F04D098F80630002B99
:103F000040F09080012E21D0414F22693B689A42B7
:103F1000C0F03186012384F82030012E3BD098F880
:103F20000730012B00F0148112F05CFF94F8203070
:103F3000A0E7B9F1000FD1D14FF48060BAF1000FC2
:103F400000F0FB8314F01CFB00232361059B002B76
:103F50003FF409AC059814F0CBF9049B1F6817F4E3
:103F600080593FF406AC1D212A48F6F733FF00289C
:103F70007FF4FFAB284A039BD2881B8BBBF90660FA
:103F8000991A8E4240F3018613449E42B4BF002624
:103F90000126FFF7F6BB1E4F3A68B8F802306421DD
:103FA00001FB03234FF480600022236184F820206A
:103FB000E27014F0CDFA94F820305BE77C5B0020CF
:103FC000C45300205C460020298A0020A200002063
:103FD000B8520020BD520020C2520020C75200201B
:103FE000CC520020D1520020D6520020DB520020BB
:103FF0005C590020548800203C590020485900207A
:104000004059002038590020288A0020ECA90020BF
:1040100060AA0020E4A90020A0530020AE52002096
:10402000BC53002012F0DEFE03224FF47A7384F8B2
:104030002020E361A74F2B8843F002032B800AF076
:10404000B5FC3A68E36913440422A36184F8202094
:10405000012E40F09D853B68A2699A42BFF476AF7D
:104060009D4B187820B91AF001FD00287FF46EAF3F
:104070002B8823F002032B808EE7964FE8E7039A04
:10408000013BD27D3BF91330002A40F08183A3F538
:104090007A73B3F57A7FA8BF4FF47A7323EAE37398
:1040A00007EE903A9FED8D7AF8EEE77A67EE877A21
:1040B0008B4AFCEEE77A17EE903A1380FFF749BB84
:1040C000884B894AB3F90430884982FB0302DB1725
:1040D000C3EBA202059B0A801B689D067FF5C5AC59
:1040E000834B1B78980704D5824E337D042B00F256
:1040F0005585278817F0300F3FF4B8AC102014F026
:1041000027FA202014F024FA7B4B278800221A700B
:104110007A4A7B487B4E7C4D002111607B4A31609E
:104120000023296041608161036083604361C36152
:1041300013605160936053619161D36196E4654F60
:104140003B6847F230520323E26184F8203072E783
:1041500012F048FE032240F6B83384F82020E361D1
:104160005C4F68E76A4F3B78002B00F09887694BFB
:10417000DFF8B481DFF8B4B1DFF8B4A103934546AA
:104180005E46049099460EE019F804109847032CF7
:1041900028DC88B93B782AF8020F01349C4205F1EB
:1041A000040580F2EF80072CE1B23046DBF80430E2
:1041B000EADD984700B2EDE738F824206B88801AD2
:1041C0004FF47A719B1A01FB00F040F6CA0290FB93
:1041D000F3F00844904240F2EE23A8BF1046984204
:1041E000B8BF184600B2D5E7DFF848A1DFF848812C
:1041F000494D0AF15A064FF0010951461AF8010CCF
:104200001AF00AFCF8B19AF804009AF802309AF809
:1042100003E000EB400105EB8101013BD1F8B42044
:1042200003EB4303434493420DD095F8E02081F81B
:10423000B0E009FA00F022EA0000C1F8B430C1F899
:10424000B87085F8E0000AF1060A5645D5D1334921
:10425000204A334B334D09681B78D2F800900891FF
:104260000793A5F1B00A00266B685BB31F784FB3C4
:10427000AA68A9EB0202002A0ADB9AF8E0200121D1
:10428000B14022EA010209F5FA718AF8E020A9603A
:10429000079ABAB12A7859780432D2B2002940F08C
:1042A0009B8203993BF91220098B01F1C8008242DD
:1042B00040F333849AF8E0109A7841FA06F3D8076D
:1042C00040F1C2840136042E05F10C05CCD1FFF774
:1042D0004FBB00BF60AA00201A020020AAF1823F53
:1042E000D2A90020588800206766666630590020F1
:1042F000788800207C8800209E490020904A002079
:10430000404A0020BC2A0020B8590020684A0020FA
:104310007C400020646300207C280020D85C0020C2
:104320004D5B00202C29002090400020946F00203D
:104330007A280020C55100205C100408A84D95F88B
:10434000AA3053B1069B1B78DE0706D5039BBBF949
:1043500006205B8B9A4200F34D841121A148F6F7A9
:1043600039FD002800F0208295F8AE302BB995F881
:10437000A83013B93223A5F8AC30012385F8AE304C
:10438000FFF792BADDF81090974A04921146974AC7
:104390000968A2FB092A42F201020A404FEA9A1A6E
:1043A000059200F0FD81924D9248934C934A95F806
:1043B00000E0007884F800E01070BEF1000F04D037
:1043C0008E4A92F800E08EF0010E854D0F2085F8A0
:1043D0002400002B00F01283894B039E0C931B7862
:1043E000B6F826C00B931C463B78B78C039E854AD3
:1043F000368B0E962646A2FB0442520802EB42027E
:10440000B21AD2B2CDF824C001F48051089295F8C6
:104410002580DFF808B2DFF824C20A900AF5967208
:1044200076460F9105F1280400200692CDF83490CD
:10443000AE46002E00F037823EF910201FFA82F9B6
:10444000B9454FEA400103D3099DA94540F26F8267
:104450005CF82020924580F02F823BF90120059DD9
:10446000002D40F04382013098422BF8012004F1E6
:104470000604DEDB0A98644ADDF834908EF8258065
:104480000F280CBF012100218EF82400117000F0CC
:10449000BC825E4C5E4E5F4F35883868A1686268AA
:1044A000E06045F00405401A9042524F3580534D6C
:1044B0004FF0010188BF00223970297088BF84F84D
:1044C0002120002B00F0B382049A03991768524E02
:1044D000B1F824C0B1F818E0504817F480573546B9
:1044E00040F0C78239460EE06A7802EB820202EBA6
:1044F000820202F2EE2292B201318B4220F8022BAC
:1045000005F102050ED016F81120002A00F01382E2
:10451000022AE9D00131028820F8022B8B4205F1F2
:104520000205F0D10C9A137801331370FFF704B928
:1045300008F1050168791AF06FFA00283FF413AC0E
:10454000012E40F0F98505F10D01A87A1AF064FA00
:10455000002840F0F5853249E87B1AF05DFA002822
:104560003FF412AC032E40F0EF852E49287D1AF05F
:1045700053FA002840F0EC852B49687E1AF04CFA7B
:1045800000283FF412AC052E40F0E6852749A87FAD
:104590001AF042FA002840F0CB85254995F823000F
:1045A0001AF03AFA00283FF412AC072E40F0678365
:1045B000204995F828001AF02FFA002840F0498386
:1045C0001D4995F82D001AF027FA00283FF412AC87
:1045D000092E3FF40FAC4FF009094B463CE300BFF6
:1045E0007C280020E4A90020F4610020D34D621053
:1045F000B83D0020E40000204D5B0020E5000020D5
:1046000029400020ABAAAAAA15510020845B0020F3
:10461000ECA9002060AA0020C4400020F4A70020DC
:10462000BD520020C2520020C7520020CC520020B0
:10463000D1520020D6520020DB5200202C40002016
:10464000CC4DD5F88830A9EB0303002BFFF681A8E9
:10465000C94A95F88C30517C079AC5F888200133F7
:10466000C64A039E32F81120B17D03F00F0385F88E
:104670008C302B4492B292FBF1F283F8902095F8A3
:10468000901095F8912095F8923095F89C000A4486
:1046900095F89310134495F89420194495F89530A3
:1046A0000A4495F89610134495F89720194495F804
:1046B00098300A4495F89910134495F89A201944B3
:1046C00095F89B300A44134495F89D1095F89F2067
:1046D000184495F89E3001440B441A4442F30B12DF
:1046E000642AF17DA8BF642213B209B1C2F1640348
:1046F00007EE903A9FEDA27AF8EEE77AD6E402212F
:10470000A048F6F767FB00283FF45DA92580B707AE
:104710003FF56AA946F00203B34223803FF464A93F
:10472000994B02201421FF2218700E2059709A70A4
:1047300013F0DEFD2688FFF757B913F009FF03E4F5
:1047400025F040039BB2AB4223803FF482A98E4BFD
:1047500002251421FF220E201D7059709A7013F04B
:10476000C7FDFFF776B9238823F00405ADB2AB424D
:1047700025803FF464A9844B02251421FF220E20DA
:104780001D7059709A7013F0B3FD2588FFF757B963
:10479000C3F53B6308331BB279E403230593D0E4EC
:1047A0007A4A92F800E008E695F8A830002B3FF42A
:1047B0007BA8069B1B7813F001037FF475A80122E8
:1047C00085F8A83085F8A920FFF76EB8694D01215A
:1047D00085F8A010FFF7F0B9012900F002849AF8DB
:1047E000E0200123B34001361343042E8AF8E03061
:1047F00005F10C057FF438ADFFF7BAB8069B644AA3
:104800001B781060DF0700F1038295F8A6100029DD
:104810007FF441A8B5F9A430322B7FF73CA895F876
:10482000A2200120572A85F8A60000F09984049B55
:104830001B6813F0040302D05A2A00F0E8855D2AB1
:1048400000F0E6845B2A00F026855E2A00F06C8585
:10485000562A00F0CD85972A00F08785A72A40F0D8
:104860009E844C49049B0A781B6842F004020A703B
:10487000494A059203F00403FFF713B8B2F5FA7F33
:10488000FFF609A895F8A620002A7FF404A8069B45
:104890001B780121D80785F8A61000F1C48409F01F
:1048A000EBF9FEF7F8BF002F3FD05CF820209245CF
:1048B0004FEA4001FFF4D1AD384A384D525C05EB68
:1048C0000109002A00F0B880022A47D199F8012096
:1048D00002EB820202EB820202F2EE2292B2032883
:1048E00033DD059D12B2002D3FF4BDAD089D24F8C7
:1048F0001520B8F1000F03D10B9D022D7FF6B3AD4B
:104900002288B4F80290B4F804804A449044244ABF
:104910000FFA88F882FB0852224DA2EBE87225F8C4
:10492000018012B24FF001089DE53A464100069D14
:104930004CF8205093E5CAB2022A04D9032A7FF426
:10494000E9AD6246D8E57246D6E5012505FA00F9DB
:104950000A9D25EA090512B20A9580E53BF8012077
:10496000BDE745F04003AB4223807FF4F0AEFFF794
:1049700070B800BF7C2800205C64002078640020B0
:1049800014AE2341E4A90020C45300204D5B002055
:10499000F83B00207888002074880020C440002064
:1049A00056555555EC28002045F004039D422380C0
:1049B0000AD0B54B02251421FF220E201D7059701C
:1049C0009A7013F095FC2588B04BB14AB3F90430C6
:1049D000B04982FB0302DB17C3EBA2030B80FFF796
:1049E0002EB83946AC48F6F7F5F900283FF406AF83
:1049F00085F8A77009F040F9FEF748BFA749A84A13
:104A00000C91DFF8C0B2012111701B21A24805935F
:104A1000F6F7E0F9059B00287FF43BADA14CA24FCF
:104A2000E2683B68A3609B1AC82B00F25A83049B80
:104A30001F6807F4805775E5C2B2022A40F2CF82A0
:104A4000032A8BD10E9A0F9D002D08BF3A4646E7E8
:104A500026F001039BB2B34223803FF458AE0E20F0
:104A60002F7085F8019085F8028013F041FC2688AC
:104A70004DE600210FE06A7802EB820202EB82022F
:104A800002F2EE2292B20131994220F8022B05F196
:104A900002053FF447AD16F811201AB1022AEAD0F8
:104AA0000288F0E7CAB2032AFAD87246EBE700237D
:104AB0000593FFF7DAB9B2F5FA7FFEF6ECAE95F89A
:104AC000A630002B7EF4E7AE069B1B7801210B403D
:104AD00085F8A61000F0E78209F068FFFEF7DBBE5C
:104AE000082013F035FDFFF73FB8704A7049106891
:104AF000B5F9A420C76981FB07018911FF17781A4E
:104B000000F5FF407F3082423EF7B3AEC91B0A4436
:104B100012B2A5F8A420FEF7ACBEC8398A425CDA0E
:104B20009AF8E0109A7841FA06F3D9073FF5CAAB34
:104B300052420120099213F0F3FC7B1E099A162BB6
:104B400000F24281DFE813F0E301F901CA01220219
:104B50000F0236029D01880171015A014301400193
:104B60002202300136029D0188011A010401EE0083
:104B7000B201D600C00012F035F9032240F6B83376
:104B800084F82020E361FFF756BA0126FEF7F9BD4D
:104B90003A68E3691344A361FFF7D8B90A2019F012
:104BA00065FF27888046002800F05882F90640F10A
:104BB0004483404D95F8F080B8F1000F7EF456AF75
:104BC0000D2013F095FB012385F8F0302788B8F10C
:104BD000000F7FF49DAAFEF749BF9AF8E03001224A
:104BE000B24023EA020309F5FA728AF8E030AA60BB
:104BF000FFF768BB00212848F6F7ECF800287FF49F
:104C0000ACAB322385F8AA00A5F8AC30FFF7A5BB02
:104C1000294B1B78002B3EF43EAEE378002B7EF44C
:104C20003AAE95F8A7300133DBB2032B85F8A730F5
:104C30007EF631AE214B5B7813B9002E7EF42BAE9D
:104C400009F0B4FEFEF722BE002A0CBF01200220AC
:104C500070E74FF008094B4603EB83031D4487F8C8
:104C60000090A97868781FF0EFFB069B144A1B7828
:104C700001211170D9077FF5C0A8FEF768BF4FF07A
:104C800007094B46E8E700BFC453002058880020BE
:104C900067666666B04A0020E4A90020294000202B
:104CA00015510020845B002060AA0020108A00209B
:104CB000D34D62107C2800204D5B0020FC5C00205E
:104CC0005C590020F4A70020DAF8E400DFF81C8724
:104CD00090F8361098F8023011446429A8BF642176
:104CE00021EAE17180F83610002B40F04B8422F06D
:104CF000BDFA74E5DAF8E400DFF8F08690F83710D2
:104D000098F802301144FE29A8BFFE2121EAE17182
:104D100080F83710002BEAD0162019F005FFDAF8DA
:104D2000E400E4E7DAF8E400DFF8C08681781144B3
:104D3000C829A8BFC82121EAE171817098F8023022
:104D4000002BD4D0142019F0EFFEDAF8E400CEE7FF
:104D5000DAF8E400DFF8948641781144C829A8BF46
:104D6000C82121EAE171417098F80230002BBED0D1
:104D7000132019F0D9FEDAF8E400B8E7DAF8E40015
:104D8000DFF8688601781144C829A8BFC82121EA44
:104D9000E171017098F80230002BA8D0122019F0B0
:104DA000C3FEDAF8E400A2E7DFF84086089898F836
:104DB0000230417911446429A8BF642121EAE171DC
:104DC0004171002B40F09383DAF8E4008FE7DAF8C2
:104DD000E400DFF81886017A98F802301144C829F7
:104DE000A8BFC82121EAE1710172002B3FF47FAF17
:104DF0000B2019F099FEDAF8E40078E7DAF8E4001D
:104E0000DFF8E885C17998F802301144C829A8BFB5
:104E1000C82121EAE171C171002B3FF468AF0A207B
:104E200019F082FEDAF8E40061E7DAF8E400DFF86E
:104E3000BC85817998F802301144C829A8BFC821DF
:104E400021EAE1718171002B3FF451AF092019F083
:104E50006BFEDAF8E4004AE7DAF8E400DFF88C8564
:104E6000417998F802301144C829A8BFC82121EA25
:104E7000E1714171002B40F04183112F7FF456AF57
:104E800035E7DAF8E400DFF86485017998F8023054
:104E90001144C829A8BFC82121EAE1710171002B82
:104EA00040F07483102F7FF457AF20E70898DFF8A5
:104EB0003C8541781144B1F5967FA8BF4FF49671B7
:104EC00021EAE171417098F80230002B3FF47CAF89
:104ED000152019F029FEDAF8E40008E70899DFF850
:104EE0000C850F791744642FA8BF642727EAE7775A
:104EF0000F7119F033FE98F80230002B3FF464AFC5
:104F00000320394619F010FEDAF8E400EFE60898BD
:104F1000DFF8D88401781144FA29A8BFFA2121EAE0
:104F2000E171017098F80230002B3FF44DAF012081
:104F300019F0FAFDDAF8E400D9E60898DFF8AC8455
:104F4000817811446429A8BF642121EAE17181704C
:104F500098F80230002B3FF437AF022019F0E4FD3F
:104F6000DAF8E400C3E60898DFF88084C17998F89D
:104F70000230114481F30801C171002B3FF424AFCA
:104F8000052019F0D1FDDAF8E400B0E6089BDFF85F
:104F90005C84997998F8020011446429A8BF6421BF
:104FA00021EAE1719971002840F0B0820D2F7FF461
:104FB000FDAE09E7DAF8E400DFF83084C17898F84C
:104FC00002301144C829A8BFC82121EAE171C1708B
:104FD000002B40F084820F2F7FF4D4AE87E60E9A28
:104FE0007DE43BF912209978B2F5617F4FF4966326
:104FF00093FBF1F34ADB40F633019142A8BF11461F
:105000000C2FA1F5617191FBF3F100F08381182F52
:105010007FF4E5ABC9B2C8290B46A8BFC823DAF8AC
:10502000E400C27DDFB297423FF4D9AB9A1ADFF8B1
:10503000BC83C77548BF0732D71098F802300137D4
:10504000FFB23BB9002F3FF4CAAB384613F068FA01
:10505000FFF7C5BB182019F067FDF3E7FA0600F16A
:105060004F810B2019F002FD002840F01881BB068B
:1050700000F15281C34D95F8F030002B3FF4A0AD04
:10508000B8F1000F7FF444A8FEF7F0BC0C2F00F03D
:10509000EA80182F7FF4A3AB00210B46BFE7BA4A82
:1050A0000392FFF771B9B949096811F4003140F072
:1050B0003F810B46B648C65C0F2E03F10C031ED091
:1050C00001311529F7D1049BB2491B680591FA3AC1
:1050D000A5F8A420002203F0040385F8A620FEF71B
:1050E000E0BBAD4A049B1F68138823F004031380C0
:1050F000012307F4805784F82130FFF713BAA74E35
:10510000D6F800E04B00BEF1000F07D05F1800EBAF
:1051100087079EF801E07F787745D4D20B44A04FF3
:10512000A04900EB8300002330603B800B60CAE79E
:105130004FF006094B468FE54FF001094B468BE5D2
:105140004FF002094B4687E54FF003094B4683E5D4
:105150004FF004094B467FE54FF005094B467BE5D0
:10516000914B92491A684FF47A73B3FBF2F3C3EB95
:10517000431203EB8203049A1268DB001206A1F8C3
:10518000B43000F1E580834B05931B685F0700F1A5
:10519000D680049B1B6803F00403FEF782BB00214A
:1051A000BB2A109100F08081B72A00F07981BE2AD5
:1051B00000F07481BD2A00F04D81792A00F0DB8176
:1051C0007A2A00F0D1819E2A00F0C8819D2A00F041
:1051D000BE81AE2A00F00182AD2A00F0F781EF2AED
:1051E00000F0EE81FD2A00F0E581FB2A00F0DC8171
:1051F000FE2A00F0D381F72A00F08E817B2A7EF40C
:105200004AAB4FF4FA61022005F0A0FAFEF743BB67
:10521000674B00220120674D67492A700B6013F02D
:105220007FF9FEF738BB049B64491B680A60594A42
:10523000059203F00403FEF734BB102013F0A0F92D
:10524000202013F085F95E494E4D081F1FF002F82B
:105250005C4B02221A7095F8F030002B00F03B8175
:105260002788FEF755BF00273946524B09915B78D6
:10527000BB423FF4B4AADFF87481384605F040FB26
:1052800098F8023009991BB1C9B20C2019F04CFCF6
:105290000137FFB2D6E64C4B01220220BBE74B4A56
:1052A0004B4B528993ED007A07EE902AF8EEE77A9D
:1052B000B0EEC77AB4EEE77AF1EE10FA7FF5D7AE2A
:1052C00093ED017AB0EEC77AF4EEC77AF1EE10FAF8
:1052D0007FF7CDAEBB063FF5CDAE2A4D202013F0B3
:1052E0004FF929467268336841F8EC2F05F1E80060
:1052F000C5F8E8301EF0AEFF324B01221A70AAE763
:10530000102013F025F92F4B278883F800804FF0E9
:105310000108A6E6CFB2A8E7202013F019F9294B1F
:10532000184D00221A7096E72A4B0222032072E7DA
:1053300029490978032900F0C5801946BAE6049B7B
:10534000264A1B680A21118003F00403FEF7A9BA5C
:10535000234B1B789B077FF516AF224B1B7D042B3D
:105360007FF611AF1EF000FF0DE7049B1E4A1B687D
:105370004FF4C8711180074A059203F00403FEF749
:1053800090BA00BF7C28002064630020B851002040
:105390002C2D040874880020ECA90020942A0020F9
:1053A000322B0020342B0020E461002098AA00203A
:1053B000A27000206C6B0020CC5B0020F83B00202A
:1053C000E44900209E490020F0700020344A00206B
:1053D0005C6D00203E710020E0A90020F65C0020FA
:1053E000788800207C880020F85C0020CCA9002070
:1053F0000BF05EFCF4F734FF0BF042FCF9F75CF8BD
:10540000012013F08DF895F8A220FFF724BA95F843
:10541000A820002A40F0938095F8AA3083F0010379
:1054200085F8AA30002B40F085800C2012F060FF38
:10543000FEF731BA002E3EF4EAAB6B4D95F8A13081
:10544000002B3EF4D3A912F037FF002385F8A130DA
:10545000FEF7CCB94FF6FE73644A6548968905900D
:10546000D089334401449381D1810BF021FCF4F7BE
:10547000F7FE0BF005FCF9F71FF8012013F050F8C8
:10548000049BB5F8A4201B68FA3A0021A5F8A420D3
:1054900003F0040385F8A610FEF703BA0223DBE746
:1054A0000B464FF6FE71D7E70B460221D4E7002BDF
:1054B000C3D05049504A09684FF47A7000FB031377
:1054C0001360BAE712F0F8FEB5F9A420FBE5032358
:1054D0000593FEF73FBD4FF00108FFF771BB0F20AA
:1054E000099219F021FBDAF8E400099A73E50E201D
:1054F00019F01AFBDAF8E400FFF7F9BB1120099262
:1055000019F012FBDAF8E400099AB6E40D200992CA
:1055100019F00AFB099A49E50021042005F016F963
:10552000FEF7B9B9304D09F041FA002385F8A130F2
:10553000FEF75CB90B2012F0DBFEFEF7ACB92C4A8B
:1055400085F8A81085F8A9000592FEF7AAB90021F0
:10555000FF2028F09FFE95F8A2203AE6012028F0CF
:1055600099FE95F8A22031E6244A137A43F001030C
:105570001372FEF790B9214A137A23F001031372D4
:10558000FEF789B9172019F0CFFA1DE4102009920F
:1055900019F0CAFADAF8E400099A83E4002103203A
:1055A00005F0D4F8FEF777B90021022005F0CEF817
:1055B000FEF771B90021012005F0C8F8FEF76BB9BC
:1055C0000021084605F0C2F8FEF765B9FF2100206A
:1055D00028F060FE95F8A22001E60121002028F0C5
:1055E00059FE95F8A220F7E57C2800201440002001
:1055F0007488002060AA0020F43B002000510020A5
:105600002DE9F0478C4B1B78DB07074644D58B4BC5
:105610008B4D1C788B4E012C59D01CD3022C07D1FA
:1056200089498A4A09881288914201D901241C704B
:10563000EB7AE3B12B89D3B1854B1B78BBB105F075
:1056400073F9002800F09B802B7B83422CBF012143
:10565000002131700CE07C497E4A098810886A7B01
:10566000801A8842E2DAEB7A0024002BE2D131780A
:105670002A79632A06D8022C774E00F0BA80337854
:10568000002B5DD1754AAB7A8C4238BF0C46147042
:10569000002B4CD1BDE8F0876B4B694D19885B88B6
:1056A000E878CB1A83EAE3728142A2EBE3721DD35E
:1056B0002B788B421AD3614B1C78E01E012861D9EC
:1056C0006749097802294FD0012C5E4EA5D15F4A67
:1056D0005D491288687B0988121A914239DD5D4A5A
:1056E00012888A42A4D200241C70A1E7B1EB400FBB
:1056F000E1DC524B1C78E11E012940F29480022A21
:10570000DEDC57494F4E0878DFF84481DFF844C1AA
:10571000DFF838E100210324022834701C7088F877
:105720000010ACF80010AEF8001081D11FE0012C81
:1057300071D0022C0BD10720BDE8F04712F0D8BD84
:105740007068381A474B984258DD72709AE7BDE886
:10575000F08702241C706BE7022AD2DD40490978E9
:1057600002294FF0040464D13949364E09783E4885
:10577000022ACCBF00220122C28081804BE7022195
:10578000317075E7022A9BDC95F800C091FBFCFCA8
:105790000CF1010CBCF1080FDFF8B4A0304EA87872
:1057A00095F801E096F800802A4CDFF8A090254E8D
:1057B000A8BF4FF0080C8AF800C01FFA8CFA10FB43
:1057C0000AF01EFB0AFE80B2DFF88CA02080A9F848
:1057D00000E000244FF0640EB8F1020F34701C702A
:1057E000CAF804408AF801E07FF439AF0FFA8CF16F
:1057F000BDE73078A0B9012377603370C2F164024D
:105800001A4B00FB02F083FB0023C017A0EBA35050
:105810006430707036E70820BDE8F04712F068BDCC
:105820007368F81A8EE7032C96D10D49097802297E
:105830009AD0044EFCE600BF288A0020E42B00200A
:1058400060880020EA2B0020446D0020E82B002017
:105850005A6D0020E62B002028590020E0A90020E6
:10586000786C00207F9698007C6C00206BCA5F6B80
:105870002DE9F04F2DED0A8B484B1B7893B0012B8F
:10588000039001F02480464C94F80021002A41F056
:105890002C80072B01F033804FF0000ADFF810B1A5
:1058A000DBF8043058469847002800F0D680BBF853
:1058B000B47000228BF85520002F41F03982DBF8BC
:1058C0004C30BBF94060BBF93C70DBF82410BBF9ED
:1058D0003E50DBF82820A6EB030E8EEAEE70791A14
:1058E000A0EBEE70AA1ACBF830102E49CBF834207A
:1058F000B0F5804FDBF82C200191D8BF33460D4620
:10590000A3EB02039BF856102748D8BFCBF84C6096
:10591000CBF838300DF0DAFA2B68990040F1378770
:10592000DBED0D5ADBED0C7A204A94ED416AD4EDA3
:10593000426A94ED437AD4F810311268B8EEE58AE1
:10594000DBED0E5AF8EEE77AF8EEE58A013377EEF2
:10595000867A38EE268A78EE878A9342C4ED417AB9
:1059600084ED428AC4ED438AC4F8103101F02987DE
:105970000A4B1F78142F02F05E850023D4F81851CB
:105980000293062D00F2F686DFE815F0C9136712C0
:1059900005128C126006F712C61300BF786C002047
:1059A00070290020F4610020C8AA00208C4100204A
:1059B00098AA0020D24D0294DFF8B083DFF8B093AC
:1059C000019C05F2DC670026CE4BDBED087A1B78E4
:1059D000172B01F0D38095ED007AB8EEC78A082B1B
:1059E00028EE278A07D1B0EE480A019328F0A4FEDA
:1059F000019B29F81600226892000BD5002E04F0B6
:105A0000AB81B0EE480ADBF8783707F170009847B1
:105A1000B0EE408AB0EE480ADBF89836A7F1700085
:105A20009847DBF8083738469847B64B1B78032B66
:105A3000B0EE408A01F0AF80D5F85C06DBF8B830F4
:105A4000B0EE480A98470136032E07F12407A8EC68
:105A5000010A05F10405B7D1029CAA4B1D78072D58
:105A600001F0268294F828310493002B40F0BD8683
:105A7000A54B5B79002B40F0C2850123A14A84F835
:105A800028311278072A01F08786002306939F4B5E
:105A900094ED4C9A93ED007A9D4BDFF8D882D3F8C1
:105AA00000A09C4B0293F7EE007A37EEC9BA08F1DA
:105AB0001C032BEE07BA0025B4EEE7BAF1EE10FA9C
:105AC0000593D4ED4BBA944BDFF8ACB2DFED938A7B
:105AD0009FED93AADFED93AADFED939ADFF89C92F6
:105AE000924F019388BFB0EE67BA2E46904B98ED67
:105AF000008A2B44D3ED007AF5EE407AF1EE10FAED
:105B000017D08C4B2B44D3ED006A38EE667AB0EE9A
:105B1000C76AF4EEC67AF1EE10FA08D5B5EEC07A8F
:105B2000F1EE10FACCBF37EEA68A36EEE78A83EDA7
:105B3000008A814B1A8893073FD0022E3DD07F4BBD
:105B40009AF82E1033F9163007EE103A059B07EE3F
:105B5000901A2B44F8EEE76AB8EEC77AD3ED007AD4
:105B60004B42A6EEA77A700007EE903AF8EEE77A7D
:105B7000B4EEE77AF1EE10FA0AD407EE901AF8EED6
:105B8000677AF4EEC77AF1EE10FA88BFF0EE477A42
:105B90006B4B6C490344085EB3F90C30C01A07EE36
:105BA000100AB8EEC77AD007E7EE687A40F125868A
:105BB000654B93ED008A27EE888A029B94F8682152
:105BC0002B44D3ED01CA38EE6CCA002A3DD05F4B9E
:105BD000D4F86C2103991B688A1A9A4235DD9AF829
:105BE0004830022B01F0B086022E04F07E80584B24
:105BF0001B68990740F1A987514B5249DFF848E1EA
:105C000031F916C09EED008ADFF874E1C7ED00AAF5
:105C100003EB460028EE288AB0F90C00A0EB0C003C
:105C200007EE900AF8EEE77ADEF8000027EE888AA1
:105C3000904238EE6CCAC1F26C81F7EE007AB4EE95
:105C4000E79AF1EE10FA01F13B81424B2B4493EDC0
:105C5000000A019B2BEE800A022E20EE0C0AA3EC18
:105C6000010A019303F0FF873B4B9BED007AD3EDD4
:105C7000007A3A4BD7ED006A93ED006A384B67EE35
:105C8000277A2B4427EE8B7AD3ED007A67EE277ABA
:105C9000F0EE665AECEE275AB1EE467AF4EEC75AA9
:105CA000F1EE10FA08D4F4EEC65AF1EE10FA8CBFF9
:105CB000B0EE467AB0EE657A94ED4C6AF7EE007A73
:105CC000B4EEE76AF1EE10FAACBF0123002343B152
:105CD000F0EEE66AF0EEC77AF4EEE67AF1EE10FA4C
:105CE00001D587ED007A022E03F0B6871D4A1E4BC0
:105CF00052F826001B68B0EE6C0A984742E000BFDD
:105D0000C8AA0020786C0020D06100208486002082
:105D1000CC5B0020E461002004410020CDCCCC3DD0
:105D2000AE47813F000000000000C8421041002043
:105D300078860020B02A00207C5B0020BC2A00204E
:105D40001440002058880020608600208C860020A7
:105D50007488002034860020A4000020A88600203B
:105D600040860020DC810020D8810020E8610020EE
:105D70007C6C0020A42A0020D48100201C4100203B
:105D800088860020CC4ACD4B52F826001B689847E5
:105D90009AF8373023B1CA4B1B88002B00F0B4852A
:105DA000B0EE6A8AC74B9BED007A38EE400A2B446E
:105DB00093ED008A83ED000A9AF8483030EE480AE5
:105DC000C0EE077A2BB3C04B1B78DB0721D5B7EEAB
:105DD000007AB4EEC79AF1EE10FA04DB94F8683159
:105DE000002B00F05087D4F86C31039AD31AB74ACD
:105DF00012689A420DDDB64B93ED007AB0EECCCA34
:105E0000B4EEC7CAF1EE10FA41F19F80002384F886
:105E10006831B04B94F878212B4493ED007A2BEE47
:105E2000877A67EE277AC9ED007A32B9019BC7ED10
:105E300000AA43ED01AAC9ED00AA0136032E08F11C
:105E4000040809F1040907F1040705F104057FF4CA
:105E50004DAEA14B1B78072B01F02482012B01F0E2
:105E6000A0840023029394F88031002B40F09885A1
:105E70009A4B9B4A1B68126813F4805C92F82C20A2
:105E800040F08F869749984891ED006A408B97497A
:105E900084ED646A91ED007A954984ED657A07EEA8
:105EA000900AF8EEE76AD1ED037A924984ED626ACE
:105EB00037EE467A77EEE67AD1ED006A84ED617AC4
:105EC000012184F89811C7EEA65A8B488B4990EDB2
:105ED000005A8B489FED8B6A90ED004A8A48DFEDAF
:105EE0008B6AD0ED004A91ED007A35EE045AF7EE58
:105EF000007AF4EEE75A35EE245AF1EE10FA88BF34
:105F0000F0EE675A25EE065AF4EEE65AB1EE476A0D
:105F1000F1EE10FAB4EEC65AB8BFF0EE665AF1EEE2
:105F200010FAC4ED675A01F11F80B4EEC75AF1EEC2
:105F300010FA88BFB0EE475A6F49DFED726AD1EDB3
:105F4000017A6F4991ED014A6F4977EE847AD1ED7C
:105F5000014A77EEA47A67EEA67AB4EEE76AF1EE2C
:105F600010FA08DCB4EEE77AF1EE10FA8CBFB0EE6E
:105F7000676AB0EE476A6049DFED626AD1ED027A86
:105F80005F49D1ED024A624977EEA47A91ED007A39
:105F900067EEA67AB1EE473AF4EEC37AF1EE10FA64
:105FA00008D4F4EEC77AF1EE10FA8CBFB0EE473A9F
:105FB000B0EE673A5749497809B9B1EE433A002A39
:105FC00041F09282F7EE003ADFF850B19BF80020E2
:105FD000002A02F00F825049DFED4C7AD1ED024ADF
:105FE000D1ED016A91ED037A66EE244AE5EE264A88
:105FF000E3EE074A63EEA44AF4EEE74AF1EE10FA44
:10600000B4BFB0EE674AB0EE644A98BFF0EE647A6F
:10601000012ACDED0A4A02F01D8291ED067AD1EDFA
:10602000052AD1ED076A26EE077AA5EE227AA3EEBD
:10603000267A23EE877AB4EEE77AF1EE10FAB4EE20
:10604000C47A8CBFF0EE676AF0EE476AF1EE10FAA0
:1060500088BFF0EE676AB4BFF0EE447AF0EE477A9C
:10606000022A8DED0B7A00F0138191ED0A7AD1EDC1
:10607000092A91ED0B4A26EE077AA5EE227AA3EEC5
:10608000047A23EE877AB4EEE67AF1EE10FAB4EEF3
:10609000E77A8CBFB0EE664AB0EE474AF1EE10FAEE
:1060A00098BFF0EE446AA8BFF0EE477A032A8DED60
:1060B0000C7A00F0ED8033E0308200202C8200204A
:1060C0007C5B0020E02A0020288A00208C860020AB
:1060D000988600204C860020786C0020F461002017
:1060E000CC5B0020D844002064630020945300203F
:1060F0005C6D0020A853002004410020AC860020E5
:10610000104100206F12833A1C4100200000000063
:10611000B08600205C46002014530020596C0020FB
:1061200091ED0E7AD1ED0D2A91ED0F4A26EE077A08
:10613000A5EE227AA3EE047A23EE877AB4EEE67A0D
:10614000F1EE10FAB4EEE77A8CBFB0EE664AB0EE2C
:10615000474AF1EE10FA98BFF0EE446AA8BFF0EE9D
:10616000477A042A8DED0D7A00F0928091ED124A63
:10617000D1ED112A91ED137A26EE044AA5EE224ABA
:10618000A3EE074A23EE844AB4EEE64AF1EE10FA93
:10619000B4EEE74A8CBFB0EE667AB0EE447AF1EE28
:1061A00010FA98BFF0EE476AA8BFF0EE447A052ACD
:1061B0008DED0E4A6CD091ED164AD1ED152A91ED78
:1061C000177A26EE044AA5EE224AA3EE074A23EEEA
:1061D000844AB4EEE64AF1EE10FAB4EEE74A8CBF18
:1061E000B0EE667AB0EE447AF1EE10FA98BFF0EEB7
:1061F000476AA8BFF0EE447A062A8DED0F4A47D0D1
:1062000091ED1A4AD1ED192A91ED1B7A26EE044A36
:10621000A5EE224AA3EE074A23EE844AB4EEE64AEC
:10622000F1EE10FAB4EEE74A8CBFB0EE667AB0EE4B
:10623000447AF1EE10FA98BFF0EE476AA8BFF0EE8C
:10624000447A072A8DED104A22D091ED1E7AD1EDC5
:106250001D2A91ED1F4A26EE077AA5EE227AA4EEBA
:10626000037A27EE237AB4EEE67AF1EE10FAB4EE72
:10627000E77A8CBFB0EE666AB0EE476AF1EE10FACC
:106280008DED117A98BFF0EE466AA8BFF0EE477A1E
:1062900077EEE67AF7EE006AF4EEE67AF1EE10FABF
:1062A000C4ED4C7A43F3648386EEA77A022ADDEDCF
:1062B0000B7A67EE244A67EE877ACDED0A4ACDED78
:1062C0000B7A2DD0DDED0C7A67EE877A032ACDEDBF
:1062D0000C7A25D0DDED0D7A67EE877A042ACDEDB4
:1062E0000D7A1DD0DDED0E7A67EE877A052ACDEDA9
:1062F0000E7A15D0DDED0F7A67EE877A062ACDED9E
:106300000F7A0DD0DDED107A67EE877A072ACDED92
:10631000107A05D0DDED117A27EE877A8DED117AAE
:10632000BA49096811F0805800F09D87F6EE005ACE
:10633000C4ED675A002A02F0548094F99801D4ED14
:10634000654AB34DB34994ED646AB34EB34FDFF879
:10635000F8E2B5F81AA0C978B6F9069097ED005A98
:106360009EF800E0D4ED616AD4ED627A07EE100A7F
:10637000FDEEE44AAA4814EE905A0078FDEEC64AB3
:1063800003F0100603F4800300F00107B8EEC77AAB
:1063900014EE900A0193002941F0E680A149002EF5
:1063A00040F09B8791ED006A9DED0A5A9E4B25EEC9
:1063B000866AA5EE076AB0EE675AA6EE265ABDEECB
:1063C000C56A16EE10EA16EE106AAE45A8BF2E4654
:1063D0007045C8BF064606EE106AB8EEC66A012AC6
:1063E00083ED006A00F0DC8091ED046A9DED0B5AAC
:1063F00025EE866AA5EE076AB0EE675AA6EE265A23
:10640000BDEEC56A16EE10EA16EE106AAE45A8BFDC
:106410002E467045C8BF064606EE106AB8EEC66A3C
:10642000022A83ED016A00F0BB8091ED086A9DEDC0
:106430000C5A25EE866AA5EE076AB0EE675AA6EEFC
:10644000265ABDEEC56A16EE10EA16EE106AAE4583
:10645000A8BF2E467045C8BF064606EE106AB8EEC5
:10646000C66A032A83ED026A00F09A8091ED0C6AF5
:106470009DED0D5A25EE866AA5EE076AB0EE675AC5
:10648000A6EE265ABDEEC56A16EE10EA16EE106AA2
:10649000AE45A8BF2E467045C8BF064606EE106A38
:1064A000B8EEC66A042A83ED036A79D091ED106ACA
:1064B0009DED0E5A25EE866AA5EE076AB0EE675A84
:1064C000A6EE265ABDEEC56A16EE10EA16EE106A62
:1064D000AE45A8BF2E467045C8BF064606EE106AF8
:1064E000B8EEC66A052A83ED046A59D091ED146AA4
:1064F0009DED0F5A25EE866AA5EE076AB0EE675A43
:10650000A6EE265ABDEEC56A16EE10EA16EE106A21
:10651000AE45A8BF2E467045C8BF064606EE106AB7
:10652000B8EEC66A062A83ED056A39D091ED186A7D
:106530009DED105A25EE866AA5EE076AB0EE675A01
:10654000A6EE265ABDEEC56A16EE10EA16EE106AE1
:10655000AE45A8BF2E467045C8BF064606EE106A77
:10656000B8EEC66A072A83ED066A19D091ED1C6A57
:106570009DED115A65EE865AE7EE055AE6EEA57ACC
:10658000FDEEE77A17EE901A8D42A8BF0D468842BD
:10659000C8BF054607EE905AF8EEE77AC3ED077AD2
:1065A0002FB922B1920021491F4827F0BDFE204B90
:1065B0001B68002B40F0F0841E4B1B7893B19BF8B6
:1065C000000060B1184E1C4F0025E8B23B68B6ECE5
:1065D000010A98479BF8000001358542F5DB174B0F
:1065E0001B689847164B1B78072B00F06E8601231B
:1065F00084F8003113B0BDEC0A8BBDE8F08F114B6D
:106600001B78013BDBB2FFF739BA00BFE4A90020D9
:1066100064630020845B0020F4A70020F052002077
:10662000288A00201453002064410020F4520020E6
:10663000CC810020CC610020B85E0020C05E00202C
:10664000786C002030860020C45E0020BC4B1A7895
:10665000D4F81CE1BB4E9FEDBC7A4FEACE00331854
:1066600083ED007A002A7BD0B849B0EE476AF0EE9D
:10667000476A0023F1EC017A013367EEA77A05EE51
:10668000903AB4EEE77AF1EE10FAF8EEE55AB8BFB8
:10669000B0EE677A9A4276EEA76AA7EEA56AE9D1CC
:1066A000F5EEC06A3318F1EE10FA83ED007A57DD8B
:1066B000C6EE265AA64BA74A1288B7EE000AD3EDBB
:1066C000007A75EEC05A65EEA77AFDEEE77A17EE0E
:1066D000903A812B41F3DB879342A8BF134607EE24
:1066E000903AF8EEE77A9C4B00EB0E0103EB810346
:1066F00093ED057AD3ED003A93ED066A93ED014AE6
:10670000D3ED046AD3ED034A93ED025AA3EEA77AC0
:10671000A4EE276A66EEC76AA7EE646ABDEEC77A82
:10672000E5EE276A17EE101A812983ED056AC3ED9D
:10673000066A41F3A9878A42A8BF0A4607EE902A53
:10674000F8EEE77AFCEEE77ACDED047ABDF810308A
:1067500032189380BEF1000F02D1132F03F0FC809A
:10676000152F41F06D8330447C4E838826F81E300F
:10677000D4F818517A4B013583FB05235A19EB17CE
:10678000C3EBA203C3EBC303ED1AC4F81851754B56
:106790001B78002B7FF40EA9734EDFF8008206F2FF
:1067A0004C7506F5F767F6EC017A9BED080ADBF805
:1067B0007837F8EEE77A284627EE800A9847A5F161
:1067C000E000DBF898369847A5F17000DBF8083751
:1067D0009847D6F85806DBF8B83098472435AF42CA
:1067E000A8EC010ADFD1FFF738B9013B84F8283162
:1067F00013B0BDEC0A8BBDE8F08F94ED577AB1F978
:106800000000D4ED586AB1F902E0584AF4EEC76AC4
:1068100080EAE0738EEAEE71A3EBE073F1EE10FA1A
:10682000A1EBEE71B4BFB0EE476AB0EE666A8B4280
:10683000B8BF0B4607EE103A1378B8EEC77A27EECA
:10684000287A002B40F0F081494BD3ED005AF4EE4A
:10685000CA5AF1EE10FA40F19A87B7EE005A75EE77
:10686000654ADFED446A9FED445A444B36EEC77AE1
:1068700024EE855AD3ED006AE7EE055A65EEA65A76
:10688000F5EEC05AF1EE10FA40F2E984C9EEA56ABD
:10689000B7EE007AF0EE475AE6EE665AF0EE656A19
:1068A000F4EEC76AF1EE10FA88BFF0EE476AF5EE33
:1068B000C06AF1EE10FAB8BFF0EE6A6A304B93EDA1
:1068C000007A67EE877AA7EEA68AFFF776B92D4B96
:1068D0001E4C19682C4A214E94F80031C96912885F
:1068E00031807280002B3EF4D7AF11F04FFF0023B0
:1068F00084F80031254B1B78072B7EF4CDAFF8F7D9
:10690000BBF88246FEF7CABF214B224A2B4493EDC7
:10691000007AD2ED007A204B67EE277AF7EE006A14
:10692000F4EEE67AF1EE10FA93ED007A88BFF0EE1D
:10693000667A67EE877A27EE888AFFF733BA00BF58
:1069400092410020B0430020000000007029002088
:106950009441002090410020C84300207C6C00201E
:106960009324499284410020C8AA00206C8600200C
:106970007486002000003443610BB63B688600201B
:1069800064860020108A0020E43A0020786C002001
:10699000CC2A00205C86002058860020E861002078
:1069A000CE4BDFF888B31B789BF80020DD077FF51E
:1069B000F8AD002A3FF4FBADD4ED583A94ED574AB8
:1069C000C74BD4ED627A93ED005A94ED617AD4ED21
:1069D000555A94ED546AC349C34BF4EEC43AF3EEEE
:1069E000046AF1EE10FA77EEA64A00F1E58791ED20
:1069F000026A26EE656AB0EE674AA6EE074AB4EE72
:106A0000E44A34EE666AF1EE10FA48BFB0EE456A29
:106A1000012A83ED006A3FF4CAAD91ED066A26EEC5
:106A2000656AB0EE674AA6EE074AB4EEE44A34EE71
:106A3000666AF1EE10FA48BFB0EE456A022A83EDAD
:106A4000016A3FF4B4AD91ED0A6A26EE656AB0EED4
:106A5000674AA6EE074AB4EEE44A34EE666AF1EEFF
:106A600010FA48BFB0EE456A032A83ED026A3FF48C
:106A70009EAD91ED0E6A26EE656AB0EE674AA6EE0F
:106A8000074AB4EEE44A34EE666AF1EE10FA48BF03
:106A9000B0EE456A042A83ED036A3FF488AD91EDB8
:106AA000126A26EE656AB0EE674AA6EE074AB4EEB1
:106AB000E44A34EE666AF1EE10FA48BFB0EE456A79
:106AC000052A83ED046A3FF472AD91ED166A26EE55
:106AD000656AB0EE674AA6EE074AB4EEE44A74EE81
:106AE000666AF1EE10FA48BFF0EE456A062AC3ED79
:106AF000056A3FF45CADD1ED1A6A66EEE56AB0EE68
:106B0000674AA6EE874AB3EE046AB4EEE44A74EE2E
:106B1000466AF1EE10FA48BFF0EE456A072AC3ED67
:106B2000066A3FF444ADD1ED1E6A66EEE55AE5EE25
:106B3000877AF4EEE74A77EEC67AF1EE10FAC8BF2C
:106B4000F0EE457AC3ED077A31E5684BC7ED00AA50
:106B50001B689342BFF671A8654B1A88002384F81E
:106B60006831002A41F03384624A634B1178186817
:106B700081F00101F2F7A4FFFFF767B895ED007A05
:106B80000BEB4602B8EEC78A928F29F8162028EE42
:106B9000278AFEF730BF27F0CFFD29F81600FEF751
:106BA0004BBF4E490978C80703D45449098BA4F850
:106BB0008C1153495348098890ED037A07EE901AD7
:106BC000F8EEE77AB4EEE77AF1EE10FA40F2CD860D
:106BD0004D48008807EE900AF8EEE77AB4EEE77ABF
:106BE000F1EE10FAC0F2798648484949D0ED006AC2
:106BF00091ED006A4748C4ED646ABCEEC75A76EE70
:106C0000665A15EE101AC4ED626AC4ED615A84ED3D
:106C1000656AA4F88C110121D0ED006A84F89811FE
:106C200077EE677AFFF74FB93B4B93ED005AB5EE1D
:106C3000C05AF1EE10FA40F31283384BD3ED006ADC
:106C4000F5EEC06AF1EE10FA40F3098336EEC77A2A
:106C500066EE695A87EE266AC5EE856AB7EE007A57
:106C6000B4EEC76AF1EE10FA88BFB0EE476AB5EE2F
:106C7000C06AF1EE10FA76EE876AB8BFB0EE6A6AC3
:106C800066EE266A0CE6264A92ED007AF0EEE76A96
:106C9000F4EEC76AF1EE10FA7FF7A5A8214A92ED4B
:106CA000007AF0EECC6AF4EEC76AF1EE10FA7FF7E4
:106CB0009AA81D4A98ED007AD2ED006AB0EEC77A24
:106CC000B4EEE67AF1EE10FA7FF58DA80122039971
:106CD000C4F86C1184F86821FFF789B8288A00206D
:106CE000F0520020145300206441002088860020C8
:106CF00010B4002012B4002014B4002064630020FB
:106D0000AC5300205C6D0020AE530020985300204F
:106D100094530020B4530020688600207086002021
:106D20009C86002098860020A0860020596C0020B8
:106D30008F49904B91F801908F4902930D781B6811
:106D40008E4E4FF47A71B1FBF3F3C3EB431803EBB0
:106D500088034FEAC3081FFA88F84745B6F90600CA
:106D600001F0FE85DBF88810BBF93CE0DBF86C3005
:106D70004A1C07EE90EA7344012ACBF88820CBF82E
:106D80006C30F8EEE77A01F0F885DBED1E5ADBEDAA
:106D9000206A07EE102A37EEE56AB8EEC75A012FCF
:106DA00086EE057A37EE257A77EEC77A8BED1F7A75
:106DB000E7EE866A8BED1E7AF0EE667ACBED216AFD
:106DC000CBED206A02F01084DBF89C10BBF93EE0AA
:106DD000DBF870304A1C07EE90EA7344012ACBF8C6
:106DE0009C20CBF87030F8EEE77A01F0E185DBED1E
:106DF000235ADBED256A07EE102A37EEE56AB8EE76
:106E0000C75A012F86EE057A37EE257A77EEC77AD4
:106E10008BED247AE7EE866A8BED237AF0EE667AC4
:106E2000CBED266ACBED256A02F00884DBF8B010C2
:106E3000BBF940E0DBF874304A1C07EE90EA73447B
:106E4000012ACBF8B020CBF87430F8EEE77A01F0E5
:106E5000CA85DBED285ADBED2A6A07EE102A37EEE9
:106E6000E56AB8EEC75A012F86EE057A37EE257A25
:106E700077EEC77A8BED297AE6EE276A8BED287AD2
:106E8000F0EE667ACBED2B6ACBED2A6A02F09F8397
:106E9000F080BBF8B430384A013B1578ABF8B43019
:106EA00002990023072D4B608B60CB607EF4DAAD36
:106EB000F7F7E2FD314EA0EB0A003080FEF7D2BDBD
:106EC00002992F4BD1ED017A93ED007AF0EEE77A3B
:106ED000F4EEC77AF1EE10FA7EF5B7AED1ED027A94
:106EE000F0EEE77AB4EEE77AF1EE10FA7EF7ADAEA7
:106EF000D1ED037AF0EEE77AB4EEE77AF1EE10FA2C
:106F00007EF7A3AE1F4B1B689A077FF525AE1E497F
